:020000040800F2
:1040000000500020616C0008716B0008756B00089F
:10401000796B00087D6B0008816B000800000000D0
:10402000000000000000000000000000896B000894
:10403000856B0008000000008D6B00083D780008CB
:10404000916B0008956B0008996B00089D6B000848
:10405000A16B0008A56B0008A96B0008AD6B0008F8
:1040600000000000B16B0008B56B00080000000004
:104070000000000000000000000000000000000040
:104080000000000000000000D56B0008657D0008FE
:10409000057C0008B57C0008E56B00080000000006
:1040A000E96B0008000000000000000000000000B4
:1040B0000000000000000000ADA30008ED6B000848
:1040C000F16B0008F56B0008F96B000879A3000894
:1040D000016C0008DD830008096C00080D6C000805
:1040E000116C0008156C0008196C00080000000035
:1040F00000000000000000000000000000000000C0
:0C41000000000000000000005FF800005C
:1041100030BF704720BF704740BF7047BFF36F8FFD
:104120007047BFF34F8F7047BFF35F8F704701DF5A
:104130007047EFF31480704780F31488BFF36F8FDC
:104140007047EFF30980704780F309887047EFF3F9
:104150000880704780F30888704772B6704762B66F
:10416000704771B6704761B6704780F31188704729
:10417000EFF31280704740BA704700BA70470000F2
:1041800008B501214FF0007001F0ACFABDE808401D
:1041900000214FF0007001F0A5BA00BF01232F4AA3
:1041A0001360536813F0010356D0037810B4012B49
:1041B000136841890CBF43F0800323F08003136030
:1041C0004378264A012B136801F1FF310CBF43F0FD
:1041D000400323F0400313608378204A012B1368C7
:1041E0000CBF43F0200323F020031360C3781B4A65
:1041F000012B13680CBF43F0100323F0100313606E
:104200000379164A012B13680CBF43F0080323F00F
:10421000080313604379114A012B13680CBF43F064
:10422000040323F004031360C3798279047A1B0624
:1042300043EA8273427A43EA044343EA0253074A59
:104240000B43D361136810BC23F001031360506863
:10425000C04300F0010070471846704700640040FA
:1042600001220378F0B59A4092B2D143374DD5F888
:10427000004244F00104C5F80042D5F81C420C404D
:10428000C5F81C428478002C46D14489C688D5F8EC
:104290000C72B0F808E046EA0446DB00848803F1BB
:1042A000804303F5C8430F4044EA0E44C5F80C723E
:1042B000C3F84062C3F844424378244C33BBD4F87B
:1042C00004320B40C4F804328389B3B91F4BD3F8CE
:1042D00014422140C3F81412837B012B05D11B4BE0
:1042E000D3F81C120A43C3F81C22184AD2F8003231
:1042F00023F00103C2F80032F0BD012BECD11349C9
:10430000D1F814321343C1F81432E5E7D4F804327B
:104310001343C4F80432D7E7012CCDD18488C68872
:10432000D5F80C72B0F808E046EA0446DB00448990
:1043300003F1804303F5C843174344EA0E44C5F82C
:104340000C72C3F84062C3F84442B5E70064004011
:10435000002310B40221032401220472417242811D
:10436000037043708370C370037143718371C371B1
:1043700010BC7047044A536919B923EA0000506120
:104380007047184350617047006400402E4BF0B4F2
:104390009A68510105D49A6812014BD501210C4647
:1043A00001E000210C46090101F1804303F5C843F7
:1043B000D3F8802102F00102C3F88021027A72B39F
:1043C0004568477AED00D3F880612A433A43324387
:1043D0004560C3F88021827A01F1804102F00F022A
:1043E0008272D3F8845101F5C84125F00F05C3F856
:1043F0008451D3F884512A43C3F88421D0F80B2088
:10440000C1F88821D0F80F202046F0BCC1F88C21DB
:10441000D3F8802142F00102C3F88021704705687B
:10442000427AD3F880616D052A4332430560C3F8B0
:104430008021D0E79B68DB0002D502210C46B2E761
:1044400004242046F0BC704700640040012825D0B9
:1044500014D3022810D11A491A488B688A689B0B1A
:104460008968120C02F0020203F004031343C1F343
:1044700000721343C05C7047022070471049114816
:104480008B688A6889689B00C1F3806103F004032C
:104490000B4302F002021343C05C7047084909480D
:1044A0008B688A689B098968120A02F0020203F08D
:1044B00004031343C1F3C0621343C05C704700BFE1
:1044C00000640040EC23010801280FD008D3022823
:1044D00005D1094A936843F400039360704770471D
:1044E000054A936843F0800393607047024A9368DB
:1044F00043F4004393607047006400402022034B64
:1045000008B11A617047DA60704700BF006400406C
:1045100038B1012803BF054B186900F003000020E3
:104520007047024BD86800F00300704700640040F9
:10453000030103F1804202F5C84230B4D2F8B04121
:1045400004F004040C72B4BBD2F8B041640D0C60EA
:10455000D2F8B0511C4C05F002054D72D2F8B4519E
:10456000234405F00F058D72D2F8B421120ACA74E3
:10457000D3F8B821CA72D3F8B821120A0A73D3F853
:10458000B821120C4A73D3F8B821120E8A73D3F8EB
:10459000BC21CA73D3F8BC21120A0A74D3F8BC2117
:1045A000120C4A74D3F8BC311B0E8B74202338B123
:1045B000236130BC7047D2F8B041E4084C60C7E7D3
:1045C000E36030BC704700BF00640040044B1A68D1
:1045D00042F002021A601868C0F34000704700BF42
:1045E00000640040054B1A6822F002021A60186845
:1045F00080F00200C0F34000704700BF006400403C
:10460000034B9B69034214BF01200020704700BF89
:1046100000640040024A936923EA000090617047F9
:104620000064004020283DD00ED9B0F5007F20D096
:1046300029D9B0F5803F21D0B0F5003F3CD0B0F58E
:10464000806F43D000207047062844D008D907283F
:1046500023D00828F6D1224BD868C0F30010704749
:1046600004282ED00528EDD11D4B986800F00100DC
:1046700070471B4B9869C0F340007047184B58684F
:10468000C0F3C0007047402811D0B0F5807FD9D169
:10469000134B986900F001007047114B9868C0F304
:1046A000004070470E4B1869C0F3C00070470C4BB8
:1046B0001869C0F300107047094B5868C0F3001028
:1046C0007047074BD868C0F3C0007047044B986927
:1046D000C0F380007047024B9868C0F30020704719
:1046E0000064004020283BD00DD9B0F5007F1DD0DC
:1046F00026D9B0F5803F1FD0B0F5003F47D0B0F5C8
:10470000806F3ED07047062836D007D9072822D0C0
:10471000082842D11022214BDA607047042827D0A4
:10472000052838D101221D4B9A6070471B4A9369B6
:1047300023F00203936170470822184B5A607047B8
:10474000402811D0B0F5807F26D1144A936923F018
:104750000103936170474FF48032104B9A607047A9
:1047600008220E4B1A61704710220C4B1A617047D9
:1047700008220A4BDA6070474FF48072074B9A6048
:104780007047064A936923F004039361704710222F
:10479000024B5A60B6E770477047704700640040AC
:1047A000044B1A6802F038021A601A681043186045
:1047B000704700BF00200240044B1A6822F0080234
:1047C0001A601A6810431860704700BF002002404A
:1047D000044B1A6822F010021A601A68104318601D
:1047E000704700BF002002400022044B04491A60B9
:1047F0005A609A60DA605961704700BF0004014056
:10480000FFFF0700837933B330B404681B4BE143E7
:104810001D6802790D401D605D6802F180422940EB
:10482000596002F58232156841792C4314600268A0
:104830009C68D04304409C60DC68102900EA0400B6
:10484000D86013D030BC01F1804303F5823319687E
:104850000A431A6070470379016803F1804303F546
:1048600082331A6822EA01021A607047996830BCE4
:1048700011439960D9680A43DA6070470004014027
:1048800000230C220360427103718371704700BFE3
:10489000024A136918431061704700BF00040140C9
:1048A000034B5B69034214BF01200020704700BF27
:1048B00000040140014B5861704700BF00040140F3
:1048C000054B1A685B69034004D0024214BF012003
:1048D000002070471846704700040140014B5861A2
:1048E000704700BF0004014008B5184B984220D023
:1048F00003F5A053984210D0A3F5C053984200D0BE
:1049000008BD01214FF4007000F0E0FEBDE8084052
:1049100000214FF4007000F0D9BE01214FF4004097
:1049200000F0D4FEBDE8084000214FF4004000F044
:10493000CDBE01214FF4806000F0C8FEBDE8084004
:1049400000214FF4806000F0C1BE00BF002801408C
:10495000436830B423F470230C790A6823F480731D
:1049600043EA04231343436085688C68CB68094A93
:1049700023432A404C79134343EA440383600A7C6F
:10498000C36A013AD2B223F4700343EA0253C3620A
:1049900030BC7047FDF7F1FF002301220360027471
:1049A000037143718360C360704700BF836819B9A6
:1049B00023F001038360704743F001038360704775
:1049C000836819B923F480738360704743F480735C
:1049D00083607047C9B243681AB923EA0101416094
:1049E0007047194341607047836843F00803836050
:1049F000704700BF8068C0F3C0007047836843F011
:104A000004038360704700BF8068C0F38000704774
:104A1000836819B923F4A0038360704743F4A003AB
:104A2000836070478068C0F38050704743680139E5
:104A300023F4604343EA413343607047436819B944
:104A400023F400634360704743F40063436070479E
:104A5000092970B41DD90726A1F10A0404EB440406
:104A6000C568A640A34025EA06042343062AC3607E
:104A70004FF01F041BD90C2A25D90D3A02EB8202F4
:104A8000C36A9440914023EA04021143C16270BC9E
:104A90007047072501EB41060469B54024EA050487
:104AA000B3402343062A03614FF01F04E3D8013AC1
:104AB00002EB8202436B9440914023EA04021143CB
:104AC000416370BC7047073A02EB8202036B94406B
:104AD000914023EA04021143016370BC704700BF98
:104AE000836819B923F480138360704743F48013FB
:104AF00083607047C06C80B2704700BF014B18687C
:104B0000704700BF4C240140436819B923F4806307
:104B10004360704743F4806343607047436819B94A
:104B200023F480534360704743F4805343607047DD
:104B3000836823F4E043194381607047836819B99F
:104B400023F400438360704743F40043836070475D
:104B5000836819B923F402138360704743F4021386
:104B6000836070478068C0F340507047092970B473
:104B70001AD8072501EB41060469B540B34024EA81
:104B80000504234303611F24836B0232C3F30155E1
:104B9000521BD2B202EB8202944023EA04039140FA
:104BA0001943816370BC70470726A1F10A0404EB26
:104BB0004404C568A640A34025EA06042343C36015
:104BC000E1E700BF836B013923F4401343EA01534B
:104BD00083637047425070472830405880B2704716
:104BE000436823F4400323F4007319434160704782
:104BF00041628262704700BF436823F01F0319437C
:104C000041607047054A936818B923F40003936024
:104C1000704743F400039360704700BF00240140D5
:104C20000368194214BF012000207047C943016086
:104C3000704700BF4368006810EA112004D0C9B271
:104C4000194214BF01200020704700BF6FEA1121F4
:104C500001607047002302683D4922F0010288424A
:104C60000260036043608360C3604AD00DD9394B52
:104C7000984226D031D9384B984228D014339842E4
:104C80005DD0283B984254D07047344B98424AD06C
:104C90000BD9334B98422ED01433984257D1314A16
:104CA000536843F4702353607047283B984234D0D4
:104CB0001433984249D12B4A536843F0F0035360B0
:104CC0007047294A536843F0F00353607047264AFF
:104CD000536843F4704353607047A3F56773984279
:104CE00015D003F56273984230D11F4A536843F0E0
:104CF0000F03536070471B4A536843F4704353607B
:104D00007047184A536843F4700353607047154A5C
:104D1000536843F0706353607047124A536843F01E
:104D20000F03536070470F4A536843F47063536036
:104D300070470D4A536843F47063536070470A4AE2
:104D4000536843F4702353609EE770477047704781
:104D50006C0002401C040240440402403000024047
:104D60004400024000000240000402408B6830B45E
:104D70000C6A0A6923434C6913438A692343CC694B
:104D80004D6A1343026823438C6A2B4322F4FF428B
:104D9000CD68234322F070020C6849681343036016
:104DA00045608460C16030BC704700BF0023036071
:104DB00043608360C360036143618361C3610362D5
:104DC00043628362704700BF036819B923F001038F
:104DD0000360704743F001030360704703681AB92A
:104DE00023EA01010160704719430160704700BF69
:104DF000406880B2704700BFC3004CBF034B044BF8
:104E00001B68034214BF01200020704700040240C9
:104E100000000240FFF7F0BFC3004CBF014B024B44
:104E2000586070470004024000000240FFF7F4BFE2
:104E300008B5324B984256D00BD9314B984234D0FA
:104E400003F5806398421AD0A3F50063984236D0E8
:104E500008BDA3F5006398423BD003F580639842F8
:104E600019D0A3F500639842F2D10121042000F08B
:104E70002DFCBDE808400021042000F027BC0121E2
:104E80004FF4807000F022FCBDE8084000214FF490
:104E9000807000F01BBC0121102000F017FCBDE861
:104EA00008400021102000F011BC0121802000F0FA
:104EB0000DFCBDE808400021802000F007BC012166
:104EC000402000F003FCBDE808400021402000F035
:104ED000FDBB0121082000F0F9FBBDE808400021DE
:104EE000082000F0F3BB0121202000F0EFFBBDE81B
:104EF00008400021202000F0E9BB00BF0014014061
:104F0000001C0140012108B5084600F0DFFBBDE8A8
:104F100008400021012000F0D9BB00BF2DE9F0417D
:104F2000CD78EB0648BF8B78098805F00F0E48BF97
:104F30004EEA030E11F0FF0F20D0002301274FF09F
:104F40000F08066802E00133082B16D007FA03F2B7
:104F500032EA0104F7D19C0008FA04FC26EA0C06A8
:104F60000EFA04F4282D46EA040632D0482D03F147
:104F7000010308BF0261082BE8D10660FF2924D98C
:104F80000022082301274FF00F08466804E0013390
:104F9000102B02F1040217D007FA03F434EA010CD3
:104FA000F5D108FA02FC26EA0C06282D0EFA02FCBE
:104FB0004CEA06060BD0482D03F1010308BF04613B
:104FC000102B02F10402E7D14660BDE8F081446194
:104FD000DDE74261B7E700BF4FF6FF71022204230D
:104FE00001808270C37070478368194214BF01202A
:104FF00000207047806880B2704700BFC3681942C4
:1050000014BF012000207047C06880B2704700BF05
:1050100001617047416170470AB9416170470161A0
:10502000704700BFC160704741F480338361816184
:10503000836183698369704710B44FF68074044AB2
:1050400013682340194341EA0011116010BC7047F6
:1050500000000140014B1860704700BF1C00204257
:1050600030B4164C00F44015B5F5401F82B26368A9
:105070001CD0C40211D50324C0F30345AC4023EA7D
:10508000040343F0706321B1400D000102FA00F007
:1050900003430A4A30BC53607047440D240102FAAE
:1050A00004F423EA040343F07063ECE7656823F03B
:1050B000706325F070656560E5E700BF00000140A2
:1050C00010B40F2401F0FC0303F1804303F5803397
:1050D00001F003019A6889008C4022EA04029A6078
:1050E0009A6800FA01F11143996010BC704700BF43
:1050F00000230C4A30B44FF0FF356FF07044104677
:105100001946C2F88050C2F88440C2F88051C2F8F3
:10511000844103F1C00201330F2B40F82210F8D173
:1051200030BC704700E100E010B400224FF0FF31C6
:105130004FF02064074B08485C609A6010BCD86050
:105140001A615A619A61DA611A625A629962D96285
:105150001963704700ED00E00000FA0540F0BF6001
:10516000024B40F40030D860704700BF00ED00E013
:10517000C3785BB9012103781C485A0903F01F0367
:10518000203201FA03F340F822307047184BF0B593
:10519000D9680F26C943FF25012402784378877810
:1051A000C1F3022126FA01F0C1F1040E02F0FC0164
:1051B000384003FA0EF301F16041034301F5614108
:1051C00002F00300D1F80063C0001B01834085405A
:1051D00073402B40054802F01F0573405209AC4054
:1051E000C1F8003340F82240F0BD00BF00E100E00C
:1051F00000ED00E00023037043708370C3707047BC
:10520000FEF7ABBFFEF7ABBFFEF7ABBFFEF7ABBF22
:105210000001FEF7AABF00BFFEF7AABF024B586805
:10522000C0F30930704700BF00ED00E001234209E0
:105230000649403251F8222000F01F0003FA00F026
:1052400030EA02030CBF01200020704700E100E0BB
:10525000014B1860704700BF00EF00E001224309D6
:10526000044900F01F00603302FA00F041F8230007
:10527000704700BF00E100E0024B5868C0F309002E
:10528000704700BF00ED00E001234209064980326B
:1052900051F8222000F01F0003FA00F030EA020368
:1052A0000CBF01200020704700E100E0014B1868AE
:1052B000704700BF00ED00E021F0604121F07F0168
:1052C000014B01439960704700ED00E0014B024A39
:1052D000DA60704700ED00E00400FA05014B024A75
:1052E000DA60704700ED00E00100FA0529B9054ACF
:1052F000136923EA000010617047024B1A691043DA
:105300001861704700ED00E00123064A00F01F001D
:105310008340506A19B920EA03035362704703437C
:105320005362704700ED00E0124BF0B4DB68FF25DC
:10533000DB43C0F38114A40004F1604404F56D4420
:10534000C0F30120A669C000C3F3022305FA00F7E9
:10535000DD40C3F10403154026EA070601FA03F312
:10536000A6612B43A2691B0183401343A361F0BCD8
:10537000704700BF00ED00E00123054AC0F3832021
:10538000526A834093430CBF01200020704700BF46
:1053900000ED00E00123044A00F01F005168834043
:1053A0000B435360704700BF00ED00E00123044A47
:1053B00000F01F005168013883400B435360704771
:1053C00000ED00E00123054AC0F38330526A8340B8
:1053D00093430CBF01200020704700BF00ED00E0A8
:1053E000C0F3814323B1012B084B04D0186B7047E5
:1053F000064BD86A7047C0F301509B6AC200D34085
:10540000022814BF03F00F00D8B2704700ED00E08F
:10541000024B420254BF586B986B704700ED00E09E
:1054200000200C4B0C4A196841F0010119605968C1
:105430000A405A601A6822F0847222F480321A609C
:105440001A6822F480221A605A6822F4FE025A6016
:1054500098607047001002400000FFF80C4BB0F558
:10546000803F1A6822F480321A601A6822F480227F
:105470001A6008D0B0F5802F04D11A6842F4A02237
:105480001A60704770471A6842F480321A60704799
:105490000010024040F2FF100A4B0B4902E05A682C
:1054A000824209D00A68C2F340421A705A68013237
:1054B0005A601A78002AF2D0034B1868C0F34040B3
:1054C000704700BF8800002000100240034A1368A4
:1054D00023F0F80343EAC000106070470010024058
:1054E000014B1860704700BF00004242034A5368F6
:1054F00023F47C13194301435160704700100240AC
:10550000014B1860704700BF60004242034A536875
:1055100023F0030318435060704700BF001002409F
:10552000024B586800F00C00704700BF00100240AA
:10553000034A536823F0F00318435060704700BFDC
:1055400000100240034A536823F4E063184350609C
:10555000704700BF00100240034A536823F46053B1
:1055600043EAC0005060704700100240044A1378BC
:1055700019B923EA00001070704718431070704783
:1055800009100240014B1860704700BFD80042422A
:10559000034A536823F4404318435060704700BFE8
:1055A000001002400022064B01281A701A7005D024
:1055B000042802D105221A7070477047187070478E
:1055C00020100240014B1860704700BF8004424227
:1055D000024A136A18431062704700BF001002406D
:1055E000014B1860704700BF3C044242214A10B48E
:1055F000536803F00C03042B06D0082B25D01BB1F5
:105600001D4A1346026001E01B4B036019491B4A07
:105610004C68C4F30314145DE34043604C68C4F366
:105620000224145D23FA04F484604C68C4F3C22499
:10563000145DE340C360496810BCC1F381310A4482
:10564000127CB3FBF2F30361704753685168C3F3F4
:105650008343C90303F1020307D55268920304D4BC
:10566000054A02FB03F30360D0E7054A02FB03F39C
:105670000360CBE70010024000127A00F423010817
:1056800000093D00044A536919B923EA000050613A
:10569000704718435061704700100240044A9369F4
:1056A00019B923EA00009061704718439061704770
:1056B00000100240044AD36919B923EA0000D061FE
:1056C00070471843D061704700100240044AD36805
:1056D00019B923EA0000D06070471843D0607047C2
:1056E00000100240044A136919B923EA000010614E
:1056F000704718431061704700100240014B18605A
:10570000704700BF40044242014B1860704700BF21
:105710004C004242014B1870704700BF0710024016
:105720004309012B0BD0022B094B00F01F000CBFCB
:105730001B6A5B6A23FA00F000F001007047044B1B
:1057400000F01F001B6823FA00F000F00100704712
:1057500000100240024A536A43F08073536270475C
:1057600000100240034B9B68184214BF0120002028
:10577000704700BF00100240014B1870704700BF17
:105780000A10024008B53A4B984265D016D9394BF9
:10579000984257D034D9384B984225D003F500634E
:1057A000984263D101214FF40050FFF78FFFBDE80D
:1057B000084000214FF40050FFF788BFA3F50063B5
:1057C00098422BD003F58063984203D0B0F1804F0C
:1057D0002ED008BD01210420FFF784FFBDE808405A
:1057E00000210420FFF77EBF01214FF40060FFF786
:1057F0006DFFBDE8084000214FF40060FFF766BF71
:10580000A3F58063984232D101211020FFF76AFF8F
:10581000BDE8084000211020FFF764BF01210220ED
:10582000FFF760FFBDE8084000210220FFF75ABFE4
:1058300001210846FFF756FFBDE80840002101207E
:10584000FFF750BF01212020FFF74CFFBDE80840C3
:1058500000212020FFF746BF01210820FFF742FF6B
:10586000BDE8084000210820FFF73CBF08BD08BD87
:10587000000C004000140040002C01400288CB883E
:1058800002F08F02028030B44C8802882343134315
:105890000A4A8D880C889BB29042038085850485D6
:1058A00006D0074B984203D030BC01238382704757
:1058B0000B7A30BC0386012383827047002C0140A1
:1058C00000340140028CF0B422F001021204120CE8
:1058D0000E890284038C8488028B0D8822F070026A
:1058E00023F0020312041B04120C1B0C2A43114D5B
:1058F0004F883343CE88A842A4B243EA0703868682
:1059000008D005F50065A84204D084800283F0BC6D
:105910000384704747F6FF454E898F8923F00803BB
:1059200033432C408E88C98923F004033C4333431E
:105930000C43EAE7002C0140028CF0B522F0100283
:105940001204120C0C890284038C4D88868823F083
:105950002003028B1B042C4322F4E0421B0C0F8813
:1059600043EA04131204174C120CCD8842EA0722B2
:10597000A042B6B29BB292B2058707D004F500648C
:10598000A04203D0868002830384F0BD4FF6BF752A
:1059900047F2FF344F8923F08003B1F80EE043EA69
:1059A00007138F891D408B8806EA040147EA0E041D
:1059B00045EA031341EA84019BB28EB286800283DA
:1059C0000384F0BD002C0140028CF0B422F48072FC
:1059D0001204120C0D890284038C4E8823F4007388
:1059E00084881B04828B35431B0C43EA052322F079
:1059F0007002154D0F881204CE88120CA842A4B272
:105A00009BB242EA0702868708D005F50065A842E6
:105A100004D084808283F0BC038470474FF6FF3645
:105A200044F6FF754F8923F4006343EA07231E40C1
:105A30008F898B88C9892C40394346EA032344EA7D
:105A400001149BB2A4B2E4E7002C0140028CF0B434
:105A500022F480521204120C0D890284038C4E88A9
:105A6000848823F40053828B1B04354322F4E042E4
:105A70001B0C0F8843EA053312040E4D120CCE881E
:105A800042EA0722A842A4B29BB292B2A0F84060B8
:105A900008D005F50065A84204D084808283F0BC5C
:105AA000038470478989C4F30D0444EA8114A4B2C5
:105AB000F3E700BF002C01400B88F0B5002B2FD07E
:105AC000042B53D0082B7DD040F6FF42048C4D8828
:105AD00024F480542404240CB1F804E00E890484D6
:105AE000878B038C34039BB223F4005344EA0E24C7
:105AF0003A4043F48053224343EA053392B29BB2C7
:105B000082830384828BC98822F440621204120CBF
:105B10008283838B9BB243EA01239BB28383F0BDD4
:105B2000028C4C8822F001021204120C8B880E8920
:105B30000284058B028CADB225F0F30592B22B43A3
:105B400022F0020243EA061322439BB242F0010212
:105B500003830284038BCA8823F00C031B041B0CF1
:105B60000383038B9BB213430383F0BD40F6FF42D4
:105B7000048C4D8824F010042404240C8E88B1F881
:105B800008E00484078B038C34029BB223F02003CB
:105B900044EA0E343A4043F01003224343EA05132B
:105BA00092B29BB202830384028BC98822F44062C2
:105BB0001204120C0283038B9BB243EA01239BB2B3
:105BC0000383F0BD048C4D8824F480742404240CD9
:105BD0008A880E890484848B038CA4B29BB224F03F
:105BE000F30423F40073224343F4807342EA061261
:105BF00043EA052392B29BB282830384838BCA88D3
:105C000023F00C031B041B0C8383838B9BB2134375
:105C10008383F0BDF0B54F888E88002F0B880CBFB2
:105C200002220022012E0CBF02240124002B4CD0A2
:105C300040F6FF4E038C0D8923F010031B041B0C50
:105C40000384B0F818C0038C36029BB223F0200303
:105C500046EA05360EEA0C0E43F010034EEA06063D
:105C600043EA0713B6B29BB206830384038BCE8844
:105C700023F440631B041B0C0383038B9BB243EA96
:105C800006239BB20383038C23F001031B041B0C2C
:105C90000384038B018C9BB223F0F30389B243EAA4
:105CA000051321F002019BB241F0010123430A4395
:105CB00003830284038B23F00C031B041B0C03835C
:105CC000038B9BB21E430683F0BD038C40F6FF4C52
:105CD00023F001031B041B0CB1F808E00384058BBF
:105CE000038CADB225F0F3059BB22E4323F00203E3
:105CF00046EA0E163B4343F00103B6B20683038423
:105D0000058BCB8825F00C010904090C0183018B5C
:105D100089B219430183018C21F010010904090C97
:105D20000184058B018C0CEA050C89B24CEA0E3E0D
:105D300021F020011FFA8EFE41F0100141EA02120B
:105D40004EEA042404830284028B22F4406212048B
:105D5000120C0283028B92B242EA03239BB20383AA
:105D6000F0BD00BF10B40B884C888A882343CC88D0
:105D700013430A8923434C8913438A8923431343DA
:105D80009BB2A0F8443010BC704700BF00234FF610
:105D9000FF7203808280C38043800372704700BF1C
:105DA0000023038043808380C380038143818381F8
:105DB000C381704700230122038082804380C38017
:105DC000038170470023038043808380C380038165
:105DD00043818381704700BF29B940F2FE330288B6
:105DE00013400380704703889BB243F00103038094
:105DF000704700BFB0F8443021B9C3F30E03A0F8D8
:105E0000443070476FEA43436FEA53439BB2A0F8B4
:105E100044307047818270470A43A0F84820704799
:105E200083899BB21AB923EA010181817047194322
:105E300081817047FFF7F4BF038923F007031B0438
:105E40001B0C0381704700BF038923F070031B0400
:105E50001B0C1943018103899BB243F007030381A3
:105E6000704700BF602970B427D0068C42F0010251
:105E700026F001063604360C0684058B068C25F0C8
:105E8000F3042404240C26F0020544EA03142D0430
:105E900044F001042D0CA4B2154304830584038946
:105EA00070BC23F070031B041B0C19430181038990
:105EB0009BB243F007030381704740F6FF44058C13
:105EC00025F010052D042D0C0584068B058C34401F
:105ED00025F020052D042D0C44EA033345EA021277
:105EE00043F4807342F010029BB292B203830284A7
:105EF000D5E700BF10B4048942EA03231943E4B292
:105F0000214389B20181038910BC23F077031B046C
:105F10001B0C43F077030381704700BF10B4048962
:105F200042EA03231943E4B2214389B20181038980
:105F300010BC9BB243F480430381704710B40489C2
:105F400042EA0323E4B21943214389B2018110BC20
:105F5000704700BF01858282704700BF40F28F33D7
:105F60000288134019430180704700BF038923F062
:105F700070031B041B0C19430181704770B4068920
:105F8000048B058C24F4407424F0030425F02205CE
:105F900026F0070624042D0442EA03133604240CD9
:105FA0002D0C360C44F480741D43314344F001043D
:105FB000ADB201810483058470BC7047038B23F06C
:105FC00070031B041B0C194301837047038B23F4DC
:105FD000E0431B041B0C43EA012189B20183704793
:105FE000838B23F070031B041B0C194381837047C0
:105FF000838B23F4E0431B041B0C43EA012189B289
:106000008183704729B940F27F33028813400380AF
:10601000704703889BB243F080030380704700BF42
:10602000838829B923F004031B041B0C8380704769
:106030009BB243F004038380704700BF838829B973
:1060400023F008031B041B0C838070479BB243F0B2
:1060500008038380704700BF838829B923F00103B8
:106060001B041B0C838070479BB243F001038380A9
:10607000704700BF038B23F008031B041B0C19435C
:1060800001837047038B23F400631B041B0C43EA5A
:10609000012189B201837047838B23F008031B041D
:1060A0001B0C194381837047838B23F400631B040B
:1060B0001B0C43EA012189B281837047038B23F0D3
:1060C00004031B041B0C194301837047038B23F447
:1060D00080631B041B0C43EA012189B201837047D2
:1060E000838B23F004031B041B0C1943818370472B
:1060F000838B23F480631B041B0C43EA012189B2C8
:1061000081837047038B23F080031B041B0C19430E
:1061100001837047038BC3F30E0343EA012189B265
:1061200001837047838B23F080031B041B0C1943EE
:1061300081837047838BC3F30E0343EA012189B245
:1061400081837047038C23F002031B041B0C19434B
:1061500001847047038C23F008031B041B0C1943B4
:1061600001847047038C23F020031B041B0C43EABB
:10617000011189B201847047038C23F080031B0452
:106180001B0C43EA011189B201847047038C23F48C
:1061900000731B041B0C43EA012189B20184704780
:1061A000038C23F400631B041B0C43EA012189B216
:1061B00001847047038C23F400531B041B0C43EA37
:1061C000013189B20184704710B40124038C8C40E2
:1061D0009BB223EA04030384038C02FA01F11943FE
:1061E00089B2018410BC704710B40424038C8C4025
:1061F0009BB223EA04030384038C02FA01F11943DE
:1062000089B2018410BC704710B40124038C8C4007
:106210009BB223EA040321F0080403847CB148F60E
:10622000FF740439C1F34E0118300B581202234099
:106230000B500B5892B21A430A5010BC70474FF6DD
:106240008F74490818300B5823400B500B5810BC62
:106250001A430A50704700BF29B940F2FD33028843
:1062600013400380704703889BB243F0020303800E
:10627000704700BF29B940F2FB3302881340038006
:10628000704703889BB243F004030380704700BF4C
:10629000838829B923F080031B041B0C838070477B
:1062A0009BB243F080038380704700BF40F2F73316
:1062B00002881340038003889BB219430180704712
:1062C000838823F070031B041B0C838083889BB29C
:1062D00019438180704700BF038923F007031B0423
:1062E0001B0C038103899BB219430181704700BFD6
:1062F000038923F080031B041B0C038103899BB2D9
:1063000019430181704700BF8184704781857047C0
:10631000818670470187704781877047A0F84010D9
:10632000704700BF038B23F00C031B041B0C03837B
:10633000038B9BB219430183704700BF038B23F487
:1063400040631B041B0C0383038B9BB243EA0121B4
:1063500089B20183704700BF838B23F00C031B04B9
:106360001B0C8383838B9BB219438183704700BFCF
:10637000838B23F440631B041B0C8383838B9BB2AE
:1063800043EA012189B28183704700BF0388DBB2F1
:10639000038003889BB2194301807047808E80B2CE
:1063A000704700BF008F80B2704700BF808F80B2FF
:1063B000704700BFB0F8400080B27047808C80B258
:1063C000704700BF008D80B2704700BF038A19423A
:1063D00014BF012000207047C94389B20182704771
:1063E000038A828911EA030092B203D0114214BFDA
:1063F00001200020704700BFC94389B20182704765
:1064000008B5284B984241D013D8A3F500639842B1
:1064100030D003F5806398421FD101214FF48020D2
:10642000FFF760F9BDE8084000214FF48020FFF736
:1064300059B91D4B984211D003F5684398420BD1CE
:1064400001214FF48040FFF741F9BDE808400021E9
:106450004FF48040FFF73AB908BD08BD01214FF461
:106460008010FFF73FF9BDE8084000214FF480108D
:10647000FFF738B901214FF40030FFF733F9BDE8D9
:10648000084000214FF40030FFF72CB901214FF4F0
:106490000020FFF727F9BDE8084000214FF4002055
:1064A000FFF720B9004C00400050004030B50D46C9
:1064B0000446038ACA889BB223F4405313430382E1
:1064C0008289888822F4B05323F00C031B040989C5
:1064D0001B0C6A8903430B4313439BB2A381A38A1A
:1064E000AA899BB223F4407387B01343A38201A807
:1064F000FFF77CF80499039A0F482B68844208BF81
:106500000A4602EB82029B0002EB8202B2FBF3F22C
:1065100064230A48A0FB0251490903FB11231B0114
:106520003233A0FB0323C3F3431343EA01139BB2AB
:10653000238107B030BD00BF003801401F85EB51FB
:1065400000234FF416510C22016042818380C380E6
:1065500003818381704700BF30B40B884D888C88DD
:10656000028A2B43C988234392B20B4322F4706200
:1065700013439BB2038230BC704700BF00230380EB
:1065800043808380C3807047838929B923F40053F3
:106590001B041B0C838170479BB243F4005383811F
:1065A000704700BF012310B401F01F04C1F3421172
:1065B000012903FA04F30FD002290CBF1030143064
:1065C0002AB9026810BC22EA03030360704702681C
:1065D00010BC1343036070470C30F1E7838A9BB211
:1065E0001AB923EA010181827047194381827047F9
:1065F000038A23F00F031B041B0C0382038A9BB244
:1066000019430182704700BF838923F400631B0490
:106610001B0C838183899BB219438181704700BF22
:10662000838929B923F002031B041B0C8381704763
:106630009BB243F002038381704700BF038A23F0BB
:1066400020031B041B0C0382038A9BB219430182A3
:10665000704700BF038A29B923F480431B041B0C35
:10666000038270479BB243F480430382704700BFAC
:10667000C1F30801818070478088C0F3080070472B
:1066800083899BB243F0010383817047038BDBB2A4
:106690000383038B9BB243EA01210183704700BF50
:1066A000038B03F47F430383038B9BB21943018362
:1066B000704700BF838A29B923F020031B041B0CF9
:1066C000838270479BB243F020038382704700BFF0
:1066D000838A29B923F010031B041B0C83827047A3
:1066E0009BB243F010038382704700BF838A29B9AD
:1066F00023F008031B041B0C838270479BB243F0FA
:1067000008038382704700BF838A23F004031B04BD
:106710001B0C8382838A9BB219438182704700BF1E
:10672000838A29B923F002031B041B0C8382704760
:106730009BB243F002038382704700BF0388194273
:1067400014BF012000207047C94389B201807047FF
:106750000123C1F3421210B4012A01F01F0403FA0D
:1067600004F315D0022A0CBF028A828A92B2134027
:10677000028892B24BB10123090A03FA01F10A42DD
:1067800014BF1846002010BC7047184610BC704754
:10679000828992B21340EBE70123090A8B40DB4365
:1067A0009BB20380704700BF08B5184B984220D0B9
:1067B00003F57443984210D0A3F57843984200D073
:1067C00008BD01214FF48040FEF78CFFBDE8084072
:1067D00000214FF48040FEF785BF01214FF4805027
:1067E000FEF774FFBDE8084000214FF48050FEF72B
:1067F0006DBF01214FF40040FEF774FFBDE8084073
:1068000000214FF40040FEF76DBF00BF003C004088
:106810004A880B8830B48C881343CA8823430C8978
:1068200013434A898D8923431343CC8902882B4320
:10683000234302F4415213439BB20380838B0A8AA1
:1068400023F400631B041B0C838330BC028270475B
:10685000F0B505460220AA8B0B8922F47B6222F058
:106860000F021204120CAA832884AE8B834287B0D5
:106870000C46B6B234D08B8801A8002B14BF022777
:106880000127FEF7B3FEE188B1F5007F2AD0238906
:106890007F0103FB07F7019B03EB83035B00B3FB63
:1068A000F7F305339BB2154AA2FB0323DB085A0812
:1068B000901EFD2803F001038CBF022342EA03234C
:1068C00060882288A788024342F4006260893A43C4
:1068D000024316430B43B6B22B84AE8307B0F0BD20
:1068E000C988EDE7019B208903EB83035B0002026B
:1068F000B3FBF2F305339BB2D5E700BFCDCCCCCCD4
:10690000002307220380028243808380C3800381A7
:1069100043818381C3817047002302220380028167
:1069200043808380C3804381704700BF038829B9B7
:1069300023F040031B041B0C038070479BB243F001
:1069400040030380704700BF838B29B923F4806321
:106950001B041B0C838370479BB243F480638383C7
:10696000704700BF012309098B4081889BB289B21F
:106970001AB921EA0303838070470B438380704771
:1069800083889BB21AB923EA0101818070471943B9
:106990008180704781817047808980B2704700BFD5
:1069A0004FF6FF639942038804D09BB243F480738F
:1069B0000380704723F480731B041B0C0380704713
:1069C000838829B923F004031B041B0C83807047C0
:1069D0009BB243F004038380704700BF038823F415
:1069E00000631B041B0C038003889BB219430180C6
:1069F000704700BF03889BB243F480530380704705
:106A0000038829B923F400531B041B0C038070472F
:106A10009BB243F400530380704700BF012914BFA9
:106A2000008B808A80B27047008A80B2704700BFB6
:106A3000B1F5804F038805D023F480431B041B0C61
:106A4000038070479BB243F480430380704700BFCC
:106A50000389194214BF012000207047202909D062
:106A6000402905D0082903D0C94389B20181704764
:106A700003897047038903889BB243F04003038076
:106A8000704700BF012210B48488008901F00F0311
:106A900080B202FA03F3184006D00909A4B28A4072
:106AA000144214BF0120002010BC704755290ED09D
:106AB00056290AD0532908D0012301F00F0103FA07
:106AC00001F1C94389B20181704703897047038985
:106AD00003889BB243F0400303807047044A0428B4
:106AE00013680CBF43F0040323F0040313607047E2
:106AF00010E000E0014B5860704700BF10E000E07C
:106B0000012805D0023009D00022074B9A60704757
:106B1000054A136843F0010313607047024A136883
:106B200023F001031360704710E000E0054A13688A
:106B300018B923F002031360704743F00203136097
:106B4000704700BF10E000E0014B9868704700BF3D
:106B500010E000E0C308022B044B0CBF1B68DB688D
:106B600023FA00F000F00100704700BF10E000E0E1
:106B7000704700BFFEE700BFFEE700BFFEE700BFB3
:106B8000FEE700BF704700BF704700BF704700BFFF
:106B9000704700BF704700BF704700BF704700BF1D
:106BA000704700BF704700BF704700BF704700BF0D
:106BB000704700BF704700BF704700BF704700BFFD
:106BC000704700BF704700BF704700BF704700BFED
:106BD000704700BF704700BF704700BF704700BFDD
:106BE000704700BF704700BF704700BF704700BFCD
:106BF000704700BF704700BF704700BF704700BFBD
:106C0000704700BF704700BF704700BF704700BFAC
:106C1000704700BF704700BF704700BF704700BF9C
:106C2000704700BF704700BF704700BF704700BF8C
:106C3000704700BF704700BF704700BF704700BF7C
:106C4000704700BF704700BF704700BF704700BF6C
:106C5000704700BF704700BF704700BF704700BF5C
:106C6000684620F007018D46134B144A01B5934244
:106C70000CD2D843104420F003000430104A1844CA
:106C800052F8041B43F8041B8342F9D10D4B0E4804
:106C900083420AD2DA430021024422F00302043282
:106CA0001A4443F8041B9342FBD10BF0C3F8BDE830
:106CB00001408546704700BF00000020840000208E
:106CC0002827010888000020582A002030B400221C
:106CD0000725082401200221094B1D705C715870A2
:106CE0009970DA701A719A711A755A759A75DA75FF
:106CF0001A769860D9601A61DA611A6230BC7047FE
:106D00009C2100202DE9F84F4FF48054404B002285
:106D10005C624FF0C8044FF47A714FF4FA704FF48C
:106D20007A6C4FF4FA6E32261C84012548F2E8078B
:106D30004FF0030B4FF0040A40F214541A765A76BF
:106D40009A76DA761A851A7783F82A2083F82B2028
:106D5000DA6283F8322083F8302083F8352083F814
:106D6000362083F837201A8783F83B201E64D863C7
:106D7000C3F800C0C3F80CC083F817B083F816A09E
:106D80009C82C3F804E0C3F808E083F83A501F82FD
:106D90005F82D983A3F8440083F85C2083F86020E5
:106DA00083F8562083F8552083F8542083F8332045
:106DB00083F8342083F8682083F8692083F86A20F8
:106DC0004FF480325A6646F2A8124FF014091A6541
:106DD0004FF04B084FF06402A3F84C600D4EA3F83F
:106DE0004600A3F85E10A3F85A1083F861503046AD
:106DF00083F8589083F85780A3F84820A3F84A20D6
:106E000008F09CFF4FF6FF733383BDE8F88F00BF97
:106E10002C21002004210020704700BF704700BFD4
:106E200001212DE9F04F084685B0FEF737FC01211E
:106E30005748FEF715F901210420FEF72FFC032621
:106E400010274FF43F43534C03A920464FF400480A
:106E50004FF4807B4FF40079ADF80C308DF80E6064
:106E60008DF80F70FEF75AF84FF480620F2300255B
:106E7000C4F810B003A9C4F8109020466261C4F8A9
:106E80001080ADF80C308DF80E608DF80F50FEF7C5
:106E900045F801210820FEF701FC49F61C52DFF8F5
:106EA00004A103A95046ADF80C208DF80E608DF8B2
:106EB0000F70FEF733F804224FF40060CAF8102078
:106EC0000823CAF810B04FF48051CAF810004FF4EC
:106ED0008060CAF81010CAF8148003A9CAF8140018
:106EE000CAF814705046CAF814308DF80F20019279
:106EF000ADF80C908DF80E60FEF710F8504603A91F
:106F0000ADF80C608DF80E608DF80F50FEF706F8A6
:106F100038460121FEF7C2FB4FF46043019A03A9F2
:106F20001D488DF80F20ADF80C308DF80E60FDF780
:106F3000F5FF01212020FEF7B1FB29464046FEF770
:106F40008FF801211548FEF78BF8294620460A23C1
:106F50004FF400524261846802616604846858BF3D
:106F60000135640448BF0131013BF3D10A2D08D03B
:106F70000B4A012106481370FEF772F805B0BDE810
:106F8000F08FA1F10A03B3FA83F35B09F0E700BFC6
:106F900000023000000801400010014000043000F1
:106FA000C1210020000C014010B500F08DFC04460A
:106FB00000F08AFC001B0028B8BF40426328F7DDC0
:106FC00000221146104609F01DFB00220A2110463E
:106FD00009F018FB6C4A0921002009F013FB00227C
:106FE0006A4C1046012109F00DFB1B21002008F01E
:106FF0007DFFA37DE27D1B2143EA0242002008F0D1
:1070000097FF00221721104608F092FF40F69F726A
:107010001821002008F08CFF40F60F721921002083
:1070200008F086FF07221A21002008F081FF584A45
:107030000A21002008F07CFF4FF0101204210020EC
:1070400008F076FF4FF080520521002008F070FF15
:1070500000220621104608F06BFF4E4A072100204F
:1070600008F066FF228A092142F08072002008F0B1
:107070005FFF628A082142F08072002008F058FF0A
:10708000236D454A1821B2FBF3F29200013A002029
:1070900008F04EFF002007F0A5FDE27E2521120337
:1070A000002008F045FF626A2621002008F040FF1A
:1070B000228D29211204002008F03AFF94F82B00B9
:1070C00002F0CAFF03F0F8F8A08D03F049F903F0CD
:1070D0000BF9B4F84620B4F84410002009F032FA55
:1070E000B4F84A20B4F84810002009F03BFA002216
:1070F000B4F84C10104609F03BFAA37D22686021D9
:1071000002FB03F2002008F013FF62682021002038
:1071100008F00EFF4FF4FA425D21002008F008FF4E
:1071200047F6FF725C21002008F002FFE268A18AA6
:10713000002009F033F800222421104608F0F8FE60
:1071400000224A21104608F0F3FE00224B2110468F
:1071500008F0EEFE00222121104608F0E9FE4FF66D
:10716000FF722021002008F0E3FE00224C2110468F
:1071700008F0DEFE094B94F83A202068616883F835
:1071800024201860596110BD0F0F13132C2100200B
:10719000000100214E014E0140787D0104210020B4
:1071A0000121F0B5084691B0FEF76CFA01214FF4C9
:1071B0000070FEF773FA3748FDF74CFD80234FF45B
:1071C00080714FF48060002404264FF4005520277E
:1071D000314A0A93314B0B910C9005A92D48059229
:1071E00006930E95079409940F9408960D97FDF752
:1071F000BDFD01212748FDF7E7FD01254FF4602380
:10720000694627480293009403948DF810608DF826
:1072100004508DF80550FDF79BFB2A4603230221FD
:107220001F48FDF715FC0323022219461C48FDF7F1
:107230000FFC032308211A461948FDF709FC032314
:10724000324609211648FDF703FC22464FF4FC6143
:107250001348FDF7BFFB29461148FDF7B1FB104865
:107260002946FDF7A3FB0E48FDF7BEFB0C48FDF7D2
:10727000C1FB0028FAD10A48FDF7C0FB0848FDF71A
:10728000C3FB0028FAD101210548FDF7C1FB11B06D
:10729000F0BD00BF080002404C24014090000020D7
:1072A00000240140704700BF00B17047012170B554
:1072B000044688B00846FEF7F1F901212648FDF79B
:1072C000CFFE01212548FDF7CBFE01210820FEF766
:1072D000E5F9082618220323694621488DF8032082
:1072E0008DF80230ADF80060FDF718FE0121084668
:1072F000FEF7E0F901A8FEF749FD48224FF47A7342
:1073000001A94FF08040ADF80420ADF80830ADF889
:107310000640ADF80A40FEF7B1FA04A8FEF740FDBA
:107320000125602304A94FF08040ADF81030ADF87E
:107330001640ADF81840ADF81250FEF7FDFA314690
:107340004FF08040FEF79EFE29464FF08040FEF74A
:1073500043FD08B070BD00BF0002300000031800FC
:10736000000C014000B1704701EB810149004FF072
:107370008040FEF7CFBF00BF48B919B94FF0804039
:10738000FEF7F0BE02214FF08040FEF7EBBE7047E3
:1073900000B1704770B510220323044608260A4D39
:1073A00082B001A928468DF807208DF80630ADF887
:1073B0000460FDF7B3FD21464FF08040FEF70CFD61
:1073C0006E6102B070BD00BF000C01404FF48052EE
:1073D000014B5A61704700BF000C01404FF48052CE
:1073E000014B1A61704700BF000C014010B9042224
:1073F000014B5A61704700BF000C014010B90422D4
:10740000014B1A61704700BF000C014018B94FF4DE
:107410008072014B5A6170470008014018B94FF45F
:107420008072014B1A617047000801401022014B25
:107430005A617047000801401022014B1A617047E1
:10744000000801401022014B5A61704700080140BA
:107450001022014B1A617047000801404FF400628E
:10746000014B1A61704700BF000C01404FF40062ED
:10747000014B5A61704700BF000C0140704700BFCC
:10748000704700BF18B94FF40042014B1A617047B2
:107490000008014018B94FF40042014B5A6170478F
:1074A0000008014020B9034B9868C0F3C030704712
:1074B000002070470008014008B9014B197070475F
:1074C000C02100204FF48062014B1A61704700BF59
:1074D000000801404FF48062014B5A61704700BFC1
:1074E00000080140024AD36883F48063D360704788
:1074F000000801404FF40072014B1A61704700BF51
:10750000000801404FF40072014B5A61704700BF00
:1075100000080140704700BF704700BF704700BFC0
:10752000704700BF704700BF00207047704700BF22
:10753000704700BF00207047032817D8DFE800F02D
:10754000110C07020A4B9868C0F340207047094BA2
:107550009868C0F340307047064B9868C0F380309D
:107560007047044B9868C0F3C030704700207047E4
:10757000000C014000100140012908B510D009D3CA
:10758000022905D1762108F0B1FCC0F3403008BDD6
:10759000002008BD762108F0A9FCC0F3003008BD2A
:1075A000762108F0A3FCC0F3803008BD40B101286B
:1075B00004D1064B9868C0F38020704700207047C4
:1075C000024B9868C0F30010704700BF000C0140E8
:1075D00038B1012804D14FF48062044B5A617047DE
:1075E00070471022014B5A61704700BF000C0140E8
:1075F00038B1012804D14FF48062044B1A617047FE
:1076000070471022014B1A61704700BF000C014007
:10761000032821D8DFE800F01C1806020F4B588819
:1076200080B2704700204FF6FF7300B583B000931F
:10763000019001230322022108F0A0FFA0F51040D1
:10764000EC3803B05DF804FB044BD88880B2704777
:10765000024B988880B2704700207047900000204D
:10766000174B184A70B592689C689868C4F3403408
:10767000C2F340229B68640144EA8214C0F3803064
:10768000C3F3C03344EA00147621002044EAC30463
:1076900008F02CFC76210646002008F027FC762115
:1076A0000546002008F022FCC0F300300443C6F376
:1076B000403644EA8604C5F3803044EA400070BD99
:1076C00000100140000C0140704700BF00B170473E
:1076D000012110B5084682B0FDF7E0FF01210B48FB
:1076E000FDF7BEFC01210820FDF7D8FF0824102279
:1076F000032301A90648ADF804408DF807208DF852
:107700000630FDF70BFC02B010BD00BF00023000D8
:10771000000C014018B90822024B09B95A617047A0
:107720001A617047000C0140704700BF704700BFEE
:10773000134B1B7813B370B44FF400754FF480648F
:107740002E4600200F49104A83B00E614C61019013
:10775000019B934205D8019B01330193019B934206
:10776000F9D94D610C610190019B9342EDD8019BC9
:1077700001330193019B9342F9D9E6E7704700BFBB
:10778000C1210020000801401FA1070070B500249E
:10779000224DFDF745FE4FF480302C70FDF75EFE64
:1077A000FDF778FE012810D001210846FDF776FF8D
:1077B0004FF480414FF00060FDF77EFD4FF44070C4
:1077C000FDF7CCFC72B662B670BD06461020FCF721
:1077D000FFFF0220FCF7E4FF2046FDF7A9FE20464C
:1077E000FDF7BAFE4FF48060FDF7ACFE4FF4403079
:1077F0004FF4E011FDF77AFE3046FDF781FE3920A7
:10780000FDF78EFF0028FAD00220FDF77FFEFDF77E
:1078100087FE0828FBD101232B70C5E798210020A3
:10782000034B10B9034ADA607047034ADA607047C5
:1078300000ED00E00100FA050400FA0510B5124A57
:10784000124C127823789A4215D86368104A013393
:10785000636013683BB11368013B1360136813B98D
:1078600001220C4B1A7000F065FE00232370A36800
:107870000133A36010BD23780133DBB22370A3680A
:107880000133A36010BD00BF080000209800002055
:10789000D8220020D422002008B50420FFF71EF9CA
:1078A00048F6A040FFF726F90120FFF729F905481F
:1078B00000220321FDF738FDBDE808400120FFF755
:1078C00035B900BF9AC30200014B5868704700BF2A
:1078D00098000020014B9868704700BF9800002076
:1078E0002DE9F04304468BB003A80D461746FCF77C
:1078F0002FFD601E072809D8DFE810F0FA00FC0011
:10790000FE00000102010800F80004010820032223
:1079100000230C218DF815208DF81330ADF81600DA
:107920008DF81410FCF72CFC01214FF00070FDF7CE
:10793000C1FE01210846FDF7B1FE01210420FDF73B
:10794000ADFE00210420FDF7C1FE00214FF4EA1036
:10795000FDF786FB4FF48051032218230DF1280810
:1079600028F8241D414668488DF806208DF8073018
:10797000FDF7D4FA4FF400630422002401264FF6E9
:10798000FF7941466048ADF804308DF80720FDF7D7
:10799000C5FA03A88DF812408DF80C408DF80E4002
:1079A0008DF80F408DF80D608DF810608DF8116026
:1079B000FCF7F4FB6B0106A88DF818408DF8194010
:1079C0008DF81A60ADF81E40ADF824408DF82660A1
:1079D000ADF82090ADF82290ADF81C30FCF740FCDB
:1079E000002F6CD14FF00008022301244FF6FF76E0
:1079F000ED002A1406A845F00405ADF81C20ADF8EA
:107A00001E508DF818308DF81980ADF824808DF84F
:107A10001A408DF82640ADF82060ADF82260FCF7E2
:107A20001FFC474519DD03239F403A1406A847F081
:107A300004078DF819808DF81A40ADF82060ADF874
:107A40002260ADF824408DF82640ADF81C20ADF83A
:107A50001E708DF81830FCF703FC01240726002562
:107A6000142302A88DF808308DF809608DF80A50AB
:107A70008DF80B40FDF77CFB152302A88DF808302C
:107A80008DF809608DF80A508DF80B40FDF770FBFA
:107A9000132302A88DF808308DF809608DF80A507C
:107AA0008DF80B40FDF764FB21460220FCF762FCD9
:107AB00021461020FCF75EFC0BB0BDE8F0837B0193
:107AC00006A88DF818608DF819408DF81A60ADF889
:107AD0001E40ADF82090ADF82290ADF824608DF8EE
:107AE0002660ADF81C30FCF7BBFB7BE704200EE7FB
:107AF000C8200CE764200AE7282008E7142006E7DE
:107B0000102004E7022002E700080140FFF7E8BE6A
:107B1000F0B5437887B004462BB3042100224368B4
:107B20008DF80C1001920293A378CBB102238DF84B
:107B30000D30234613F8081B0DF10F028DF80E10BF
:107B400004F1100013F8011B834202F8011BF9D164
:107B500001A8FCF71BFC04280BD0012007B0F0BDE6
:107B60008DF80D30E5E742688DF80C3002930192F4
:107B7000DAE70E4E0E4B35681B680135082D08BF3D
:107B800000259D420FD094E80F003768094C04EBA4
:107B9000071484E80F00012108463560FCF7EAFB72
:107BA000012007B0F0BD002007B0F0BDC8210020C3
:107BB000CC2100205422002070B40F4B0F4C2268BF
:107BC0001B689A4214D0054622680D4B511C216057
:107BD00003EB02130FCB266885E80F00082E02D0B6
:107BE00070BC0120704700230120236070BC7047E7
:107BF000002070BC704700BF50220020C42100202C
:107C0000D0210020684620F007018D4671B5264C32
:107C1000264B26681B680136082E08BF00269E42A8
:107C200087B034D001A90020FCF782FC9DF80C300D
:107C3000042B34D0002123681D4D019A05EB03135A
:107C40005970236805EB03135A609DF80D30022B21
:107C50000CBF01220022236805EB03139A70002257
:107C600023689DF80E101B01E9540DF10F012368E4
:107C700011F8010B05EB031313440132082A1872A3
:107C8000F5D1266007B0BDE87140854670470020F9
:107C9000FCF734FC07B0BDE8714085467047012110
:107CA0002368034D029AC9E750220020C421002016
:107CB000D0210020684620F007018D4671B5264C82
:107CC000264B26681B680136082E08BF00269E42F8
:107CD00087B034D001A90120FCF72AFC9DF80C30B4
:107CE000042B34D0002123681D4D019A05EB0313AA
:107CF0005970236805EB03135A609DF80D30022B71
:107D00000CBF01220022236805EB03139A700022A6
:107D100023689DF80E101B01E9540DF10F01236833
:107D200011F8010B05EB031313440132082A1872F2
:107D3000F5D1266007B0BDE8714085467047012047
:107D4000FCF7DCFB07B0BDE87140854670470121B8
:107D50002368034D029AC9E750220020C421002065
:107D6000D0210020684620F007018D462C4B11B52C
:107D70002C4987B00A681B689A424BD00B682A4C82
:107D800004EB03135B7803F0FF02002B34D10B6884
:107D90008DF80C2004EB03135B68029201930B68CF
:107DA00004EB03139B7803F0FF02002B2FD0022378
:107DB0008DF80D3000220B680DF10F001B01E35C04
:107DC0008DF80E300B6804EB031313441B7A013259
:107DD000082A00F8013BF5D10B6801A801330B60BC
:107DE0000B68082B04BF00230B60FCF7CFFA07B029
:107DF000BDE8114085467047042000220B688DF8CD
:107E00000C0004EB03135B6801920293C7E78DF843
:107E10000D20CFE700210120FCF7ACFAE7E700BF17
:107E2000C8210020CC21002054220020704700BF30
:107E300070B506460D46FFF7C9FA0D4C02212046E3
:107E4000FEF706FE0028F9D031460948FEF7A2FDEC
:107E5000074C01212046FEF7FBFD0028F9D00DB1AB
:107E6000FFF7BCFA0248FEF797FDC0B270BD00BF35
:107E70000038004010B5044600210320FFF7D8FF6A
:107E8000C4F307200021FFF7D3FFE0B20021FFF782
:107E9000CFFFBDE8104001210020FFF7C9BF00BFA0
:107EA00038B504460D4606200121FFF7C1FF002129
:107EB0000520FFF7BDFF01210020FFF7B9FF820772
:107EC000F5D500210220FFF7B3FF0021C4F30720FE
:107ED000FFF7AEFF0021E0B2FFF7AAFF284601211D
:107EE000FFF7A6FF00210520FFF7A2FF01210020D8
:107EF000FFF79EFFC307F5D438BD00BF38B54FF478
:107F0000006501210620FFF793FF00210520FFF700
:107F10008FFF01210020FFF78BFF8207F5D500219D
:107F20000220FFF785FF0021C5F30720FFF780FF40
:107F30000021E8B2FFF77CFF0024A4F13F01B1FA71
:107F400081F1002049090134FFF772FF402CF4D180
:107F500000210520FFF76CFF01210020FFF768FFDB
:107F6000C307F5D44035B5F5804FCAD138BD00BF41
:107F7000F0B5C0EBC00083B000F500640D460320EF
:107F80000021FFF755FFC4F307200021FFF750FF42
:107F9000E0B20021FFF74CFF00210846FFF748FF41
:107FA000002106460846FFF743FF00210446084625
:107FB000FFF73EFF002107460846FFF739FF002183
:107FC0008DF804000846FFF733FF00218DF8050007
:107FD0000846FFF72DFF01218DF806000020FFF76E
:107FE00027FF8DF800608DF80140BDF800202B8838
:107FF0008DF807009A4202D0002003B0F0BDAB78A4
:10800000BB42F9D16B680198C01AB0FA80F0400900
:10801000F3E700BF38B50D46C0EBC00404F50060BF
:108020000978FFF73DFF697804F60100FFF738FF94
:10803000A97804F60200FFF733FF297904F603005C
:10804000FFF72EFF697904F60400FFF729FFA979ED
:1080500004F60500FFF724FFE97904F60600BDE801
:108060003840FFF71DBF00BFC0EBC00038B50C465D
:1080700000F5006500210320FFF7DAFE0021C5F3BB
:108080000720FFF7D5FE0021E8B2FFF7D1FE00215F
:108090000846FFF7CDFE002120700846FFF7C8FE16
:1080A000002160700846FFF7C3FE0021A07008465B
:1080B000FFF7BEFE002120710846FFF7B9FE002140
:1080C00060710846FFF7B4FE0121A0710020FFF7A0
:1080D000AFFEE07138BD00BF2DE9F04105460E4608
:1080E000062001211746FFF7A3FE00210520FFF718
:1080F0009FFE01210020FFF79BFE8207F5D500219E
:108100000220FFF795FE0021C5F30720FFF790FE40
:108110000021E8B2FFF78CFE002F40D00024013E82
:1081200007F1FF3809E0A8EB0401B1FA81F1490930
:10813000FFF77EFE0134A74231D00135AB0616F8B9
:10814000010FF0D10121FFF773FEA045F2D9002104
:108150000520FFF76DFE01210020FFF769FEC10732
:10816000F5D401210620FFF763FE00210520FFF76B
:108170005FFE01210020FFF75BFE8207F5D500219D
:108180000220FFF755FE0021C5F30720FFF750FE40
:1081900001340021E8B2FFF74BFEA742CDD1002108
:1081A0000520FFF745FE01210020FFF741FEC30730
:1081B000F5D4BDE8F08100BFF8B5044616460D467B
:1081C00003200021FFF734FE0021C4F30720FFF74E
:1081D0002FFEE0B20021FFF72BFE76B10024013D17
:1081E000771E391BB1FA81F100204909FFF720FE03
:1081F0000134A64205F8010FF3D1F8BD10B540F2E5
:10820000FF70FFF737FE702802D1164B1B78ABB119
:10821000002140F2FF70FFF743FEFFF76FFE2422BC
:1082200011490020FFF758FF104940206C22FFF74A
:1082300053FF702140F2FF70FFF732FE0A4C2422F8
:1082400021460020FFF7B8FF607808F0DFFA4020F1
:108250006C220649FFF7B0FF6078BDE8104008F0D7
:10826000E1BA00BFC12100209C2100202C21002068
:1082700070B5544B544C86B0054618462360FEF743
:10828000BFF801210920FDF709FA01214FF48040D0
:10829000FDF704FA01210420FCF7E2FE402103224D
:1082A000182306AE26F8181D314648488DF80220DE
:1082B0008DF80330FCF732FE4822802331464348D4
:1082C0008DF80320ADF80030FCF728FE02A8FEF779
:1082D00037F9681E0A2807D8DFE800F055606B6E92
:1082E000585B6568635E71004FF4965302A920687D
:1082F000002501260293FEF7D9F80523252201A8BF
:108300008DF805308DF804208DF806508DF8076043
:10831000FCF72EFF206840F2FF31FEF715FA2A46DF
:1083200020682821FEF73EF93246206840F2277186
:10833000FEF738F93246206840F22661FEF732F93E
:108340003246206840F22551FEF72CF92A46206873
:1083500040F22441FEF726F92A46206840F64601FD
:10836000FEF720F92A46206840F66A11FEF71AF94E
:108370002A4620686021FEF715F931462068FEF78D
:1083800003F906B070BD4FF4E153AFE74FF4E1439A
:10839000ACE74FF41643A9E70D4BA7E74FF416538C
:1083A000A4E70C4BA2E74FF461439FE74FF4E1339E
:1083B0009CE74FF4615399E74FF4964396E7064BD9
:1083C00094E700BF003801400C000020000C014081
:1083D00090D0030048E8010020A10700684620F083
:1083E00007018D4631B5294D28680388990627D4A1
:1083F00003881A0611D5264C226B636B9A423BD038
:10840000FFF794F8636B28685A1C6263234493F85F
:1084100038308380636B202B35D003885B0603D410
:10842000BDE831408546704740F22661FEF7B4F959
:10843000174B5A6B1B6B9A42F2D1FFF779F8EFE7B3
:10844000FFF778F8A8B9124A286813685168013311
:10845000202B08BF00238B4205D01168848811446B
:10846000E4B20C7213600A210A4B1960936AD3625A
:10847000BEE728688388BBE7002240F22771FEF739
:1084800091F82868C9E700236363C6E70C00002061
:10849000A4000020D822002070B40C4C236B626B27
:1084A0000133202B08BF002393420DD00646256BD5
:1084B000074A254485F8386010682363012270BCA0
:1084C00040F22771FEF76EB870BC7047A400002020
:1084D0000C0000200A4B59681A6891420ED05A6865
:1084E000511C59601A44117A5A680170202A01D02F
:1084F00001207047002201205A6070470020704719
:10850000A4000020014B9862704700BFA400002027
:10851000044A137803F0FF0013B100230120137005
:10852000704700BFD4220020014BD86A704700BFBB
:10853000A4000020034BDA6A12B1DA6A013ADA6267
:10854000704700BFA400002030B4054B054C1D68E7
:108550006278A0786560052130BC02F02BBE00BFB8
:108560002424002008230020094B9A7842B95B7824
:10857000142B09D80749084A096842F823107047A4
:108580000422064B1A7070470322044B1A7070477E
:10859000082300202424002014230020FC24002091
:1085A000034A044B126809205A6004F0D1BB00BF93
:1085B00024240020082300200120054B05495A7877
:1085C0000870824202D15A68034B1A60704700BF9C
:1085D00008230020BD240020582400200222014B43
:1085E0001A707047BD240020F0B400254FF0FF340E
:1085F0002B4629460D4F0E4E0E4A0F483D703570E2
:10860000C15401332F2B42F8044FF9D10B4F0C4CBE
:108610000C4E0D4D0D480E4A0E4B397021703160D5
:108620002960016011601960F0BC7047FC220020D5
:10863000BC24002064230020C8240020BD24002086
:108640000423002058240020C424002024240020D7
:1086500008250020102300200022014B1A707047CB
:10866000BD24002070B42A494B78032B44D8DFE89E
:1086700003F0371407020A22264B5A6070BC704779
:1086800000222548254B1146026003F1280243F8D9
:10869000041B9342FBD170BC70471F4E306800280A
:1086A000ECD01E4A4D681368AB422FD01146002310
:1086B00001338342E2D051F8044FAC42F8D1411E5D
:1086C0008B420BD200F18040013802EB800002EBBC
:1086D00083035A6843F8042B8342FAD13160CDE713
:1086E0000D4A1368092B0CD84C680C48591C40F8EB
:1086F0002340116070BC70470322064B1A7070BC97
:1087000070470922034B1A7070BC70470023D6E7EC
:1087100008230020FC240020C02400205C2400202A
:108720002B4A5378092B50D8DFE803F010161C238E
:108730002A33393F45055368264A1360264A002BE1
:108740003ED0136823F00803136070472149536833
:108750000A6813440B60F1E71E4952680B689B1AC4
:108760000B60EBE71B4952680B6803FB02F30B60DD
:10877000E4E7184952680B6893FBF2F30B60DDE7FE
:1087800014495268086890FBF2F302FB13030B6074
:10879000D4E7104953680A6813400B60CEE70D49CF
:1087A00053680A6813430B60C8E70A4953680A68AC
:1087B00053400B60C2E7074A1368DB431360BDE711
:1087C000136843F0080313607047024B1B68B5E75A
:1087D000082300202424002010230020354B5B7840
:1087E0000A2B63D8DFE803F0141B222A323C434AE9
:1087F00051580600304A314910680B680860136010
:108800002F4A002B4DD0136823F0080313607047E4
:10881000294A2A4B11681B680B441360F0E7264A6B
:10882000264B11681B68CB1A1360E9E7224A2349DB
:108830001368096801FB03F31360E1E71E4A1F4B4D
:1088400011681B6891FBF3F31360D9E71A4A1B49BF
:108850001368096893FBF1F001FB10331360CFE755
:10886000154A164B11681B680B401360C8E7124A83
:10887000124B11681B680B431360C1E70E4A0F4B84
:1088800011681B684B401360BAE70C490A4B0A6831
:108890001B68D2430A60B3E7074B084A1B681360A2
:1088A000AEE7136843F0080313607047024B1B6880
:1088B000A6E700BF0823002024240020082500206C
:1088C00010230020164B5B78052B09D8DFE803F056
:1088D000090F151B2103134A136823F480731360D7
:1088E0007047104A136803F00F03136070470D4A76
:1088F000136823F01003136070470A4A136823F0CB
:10890000200313607047074A136823F04003136085
:108910007047044A136823F080031360704700BF58
:108920000823002010230020104A114B11685B68B7
:10893000104A8B42136809DA23F0030343F004035F
:10894000136079B123F00803136070470BBF23F065
:10895000060323F0050343F0010343F00203136011
:108960000029EFD143F0080313607047242400204E
:108970000823002010230020830703D50822054B7D
:108980001A7070470422044B04495868044B08606D
:108990001A707047FC2400200823002000230020C8
:1089A000BD2400200022014B1A707047BD24002016
:1089B00008B50C4B196821F07F4121F0FF0121B966
:1089C00040F2D2425B68934200D008BD40F2FF7093
:1089D000FFF766FAFFF792FABDE808400120FEF7BC
:1089E0001FBF00BF0823002010B4124B5B78032B7D
:1089F0000FD8DFE803F01C0216100F4B0F48104988
:108A00001A6800780F4B0978140A5C711A71D871D2
:108A1000997110BC70470C4A0A4B12685A6010BC1E
:108A200070470A4A074B12685A6010BC7047084BDF
:108A3000E4E700BF0823002058240020BD240020C4
:108A400004230020FC2400200825002024240020EA
:108A5000002300200222014B1A70704728240020B6
:108A6000024A034B52681A60704700BF0823002077
:108A700058240020284A53780C2B0CD8DFE803F048
:108A8000071E141923282E33383D42470C00234B70
:108A90001B68180704D47047204B1B68DB05FAD508
:108AA00052681F4B1A6070471C4B1B68DB07F7D4DA
:108AB00070471A4B1B68D807F2D57047174B1B68D5
:108AC0001907EDD57047154B1B685907E8D4704757
:108AD000124B1B6813F0050FE2D170470F4B1B6858
:108AE0009B07DDD470470D4B1B689807D8D17047A2
:108AF0000A4B1B68D906D3D47047084B1B689B06EA
:108B0000CED47047054B1B685806C9D47047034B39
:108B10001B681906C4D470470823002010230020C6
:108B200058240020084A1368072B0BD870B4074953
:108B300007480D684668074C581C10600E6044F8E2
:108B4000235070BC704700BFC4240020582400206C
:108B50000823002038240020F0B501241E4B1F4AB2
:108B60005B681F4DB3F5006F83B01470287001DC93
:108B70000C400AD000211B4BDA1D03F8011B934265
:108B8000FBD12B782B7203B0F0BD18466946FFF776
:108B90006BFA9DF801309DF8050021469DF80020F4
:108BA0009DF802709DF807609DF80640AB709DF837
:108BB0000430A871EB716A70EF702E716C71AB1C90
:108BC00005F1080001E013F8012B1144C9B28342FA
:108BD0002972F8D103B0F0BD08230020282400201A
:108BE0002C2400202D240020054A136833B10549A8
:108BF000013B51F82300044913600860704700BF2F
:108C0000C4240020382400205824002030B5144DFE
:108C100083B06C7884B1012C04D00322114B1A70FC
:108C200003B030BDAB782A2BF7D1291D042240F2C6
:108C3000FB70FFF751FAF3E7042240F2FB700DEBF3
:108C40000201FFF7B9FA6A68019B9A4203D0054B0B
:108C50005C6003B030BD0122024B5A60E0E700BF08
:108C600008230020FC2400200022014B1A707047CA
:108C7000BD24002070B5114E114D3068114C2A787A
:108C80006B68B0F5006F6270636005D90721002240
:108C90000D4B21701A7070BD2946FFF7BBF92946AC
:108CA0003068FFF765F928B1652233682270013317
:108CB000336070BD0723237070BD00BF0023002008
:108CC00008230020FC240020BD24002070B52A4E7B
:108CD0002A4C33786BB963685A1C2BD003EB83039F
:108CE000274A5B001360FEF7EFFD0122254B32702F
:108CF0001860657885B1012D0DD1A07800F08CFE4B
:108D000010F4804530D11E4C2368DBB91E4A13682D
:108D1000013B136070BD70BDFEF7D6FD194B184ABC
:108D20001B681268C01A0028B8BF40429042EDD9B3
:108D3000357070BD154B124A1B6803EB83035B0053
:108D40001360D0E7FEF7C0FD0E4B22681B68C31A04
:108D5000002BB8BF5B429342D8D90D4A35701368D7
:108D600043F01003136070BD0023094A3370136889
:108D700023F01003136070BD04230020082300209B
:108D80000C290020842400205824002024240020C2
:108D900010230020094B9A783AB95A78142A08D837
:108DA0005968074B43F8221070470422054B1A708C
:108DB00070470322034B1A70704700BF082300203E
:108DC00014230020FC240020144B9A785AB95A78B6
:108DD000142A19D81249134B51F822205A60124A0A
:108DE00012783AB9704704220E4B1A700E4A127864
:108DF000002AF7D00D4A5B6813600D4A43B113682F
:108E000023F00803136070470322064B1A70EDE746
:108E1000136843F008031360704700BF0823002065
:108E200014230020FC240020892400202424002076
:108E3000102300200A4B987838B910B55C78142CB0
:108E400007D90322074B1A7010BD0422054B1A7074
:108E5000704705F0B5FB044B43F8240010BD00BF7C
:108E600008230020FC24002014230020074B5B78FB
:108E70002E2B07D9FF2B0BBF01220322044B054BDE
:108E80001A7070470121044AD1547047082300200A
:108E9000FC220020FC240020C8240020074B5B7823
:108EA0002E2B07D9FF2B0BBF00220322044B054BAF
:108EB0001A7070470021044AD154704708230020DB
:108EC000FC220020FC240020C8240020064A5378FD
:108ED0002E2B03D90322054B1A7070475168044AA0
:108EE00042F82310704700BF08230020FC24002014
:108EF00068230020F0B5114B114E1F685D68114CBE
:108F0000376025609F68DD681A7F0F4E0F4C10494F
:108F10003760D3F810E025605E699C690D4F0E4DF7
:108F20000E4B885C87F800E02E601C6008B10123BE
:108F30008B5400220A4B1A70F0BD00BFDC220020C7
:108F4000242400200825002058240020102300207D
:108F5000C824002004230020842400200C290020A1
:108F6000BC240020564B5A68FF2A22DC10B45978E2
:108F70000B2900F29980DFE801F08C8175695B5064
:108F8000453A31291D0699784E4B53F8211053F874
:108F900022304D4A9942136800F38B800BBF23F0B7
:108FA000060323F0050343F0010343F0020310BC62
:108FB000136070479978434B53F8224053F82100CF
:108FC00043F8214043F8220010BCF2E73D499B786A
:108FD00051F8222010BC41F82320EAE7394998785B
:108FE00051F8223010BCDB4341F82030E1E799789A
:108FF000344B10BC53F8220053F82120424043F870
:109000002120D6E799782F4B10BC53F8220053F853
:109010002120024343F82120CBE79978294B10BC4B
:1090200053F8220053F82120024043F82120C0E7E2
:109030009978244B53F8214053F8220094FBF0F226
:1090400000FB124210BC43F82120B2E799781D4B77
:1090500010BC53F8220053F8212092FBF0F243F8A1
:109060002120A6E79978174B10BC53F8222053F81B
:10907000210002FB00F243F821209AE79978114B76
:1090800010BC53F8220053F82120121A43F8212073
:109090008FE799780B4B10BC53F8220053F821202E
:1090A000024443F8212084E70322084B1A7010BCC5
:1090B0007FE723F0030343F00403136010BC78E759
:1090C000082300200C25002010230020FC24002071
:1090D00010B44D4A53780B2B00F28C80DFE803F07C
:1090E0001B26303B46535D67717980069178474B6C
:1090F000474A1B6852F821209A42464A13687DDC91
:109100000BBF23F0060323F0050343F0010343F0F4
:109110000203136008E091783C483D4A006852F829
:109120002130034442F8213010BC70479178374811
:10913000374A006852F821301B1A42F82130F3E711
:109140009178324B324A1B6852F8210003FB00F33E
:1091500042F82130E8E791782C482D4A006852F80F
:10916000213093FBF0F342F82130DDE79178274B73
:10917000274A186852F8214094FBF0F300FB134390
:1091800042F82130D0E791782048214A006852F80F
:109190002130034042F82130C6E791781B481C4A31
:1091A000006852F82130034342F82130BCE791783F
:1091B0001648174A006852F82130434042F82130DF
:1091C000B2E7124B91781B68114ADB4342F8213019
:1091D000AAE70E4B927819680D4B43F82210A3E7CB
:1091E00092780B4B094953F8224008680C6043F809
:1091F000220099E70322084B1A7095E723F0030336
:1092000043F0040313608FE7082300202424002088
:109210000C25002010230020FC24002030B45C4AE0
:1092200053780B2B00F2A080DFE803F01C2D3844AC
:10923000505E69747F8992069178564B564A53F86E
:1092400021301268554993420B6880F2958023F0D3
:10925000030343F004030B6082B130BC23F0080326
:109260000B60704791784C4B4A4A52F821001A68BB
:109270004A4902441A600B68002AEED130BC43F020
:1092800008030B6070479178434B424A186852F8C4
:1092900021204249821A1A600B68DDE792783E4825
:1092A0003C4B3E4953F82230026802FB03F20B6844
:1092B0000260D1E792783848364B384953F822306B
:1092C000026892FBF3F20B680260C5E792783248BD
:1092D000304B324953F82230026892FBF3F403FB1F
:1092E00014220B680260B7E791782B4B294A52F899
:1092F00021001A68294902401A600B68ACE791788E
:10930000254B244A52F821001A68244902431A6066
:109310000B68A1E79178204B1E4A52F821001A6889
:109320001E4942401A600B6896E71A4B92781A4819
:1093300053F822201949D2430B6802608CE79178D8
:10934000144A154B52F8212014491A600B6883E720
:10935000114B94780F481D6850F824200F491A606B
:1093600040F824500B6877E703240B4B0B490C485B
:109370001A6804700B686FE70BBF23F0060323F035
:10938000050343F0010343F002030B6064E700BFF1
:10939000082300200C250020242400201023002076
:1093A000FC24002010B44D4A53780B2B00F28C8023
:1093B000DFE803F01B26303B46535D67717980067A
:1093C0009178474B474A1B6852F821209A42464AF7
:1093D00013687DDC0BBF23F0060323F0050343F085
:1093E000010343F00203136008E091783C483D4AD2
:1093F000006852F82130034442F8213010BC704715
:1094000091783748374A006852F821301B1A42F8E1
:109410002130F3E79178324B324A1B6852F8210031
:1094200003FB00F342F82130E8E791782C482D4AFD
:10943000006852F8213093FBF0F342F82130DDE769
:109440009178274B274A186852F8214094FBF0F393
:1094500000FB134342F82130D0E791782048214A9D
:10946000006852F82130034042F82130C6E7917875
:109470001B481C4A006852F82130034342F821304F
:10948000BCE791781648174A006852F821304340EB
:1094900042F82130B2E7124B91781B68114ADB4346
:1094A00042F82130AAE70E4B927819680D4B43F829
:1094B0002210A3E792780B4B094953F82240086821
:1094C0000C6043F8220099E70322084B1A7095E7D5
:1094D00023F0030343F0040313608FE70823002005
:1094E000082500200C25002010230020FC2400204B
:1094F000494A53780B2B00F28580DFE803F01B24E8
:109500002D37414D565F687077069178434B444A3A
:109510001B6852F821209A42424A136876DB0BBF3F
:1095200023F0060323F0050343F0010343F0020395
:109530001360704791783A4B384A53F821301168DC
:109540000B44136070479178354B344A53F821101F
:1095500013685B1A136070479178314B2F4A53F8A8
:109560002110136803FB01F31360704791782C4BB3
:109570002A4A53F82110136893FBF1F313607047E4
:109580009178274B254A53F82110106890FBF1F38E
:1095900001FB1303136070479178214B1F4A53F866
:1095A000213011680B401360704791781C4B1B4AA7
:1095B00053F8213011680B43136070479178184BB2
:1095C000164A53F8213011684B4013607047917868
:1095D000134B124A53F82130DB43136070479178E4
:1095E0000F4A0E4B52F821201A60704710B40C4BF2
:1095F00092780A4953F8224008680C6043F8220028
:1096000010BC70470322084B1A70704723F0030305
:1096100043F004031360704708230020082500204E
:109620000C25002010230020FC240020434B5A78F6
:109630000B2A78D8DFE802F01A232C36404E576008
:109640006971770699783E4A5B6852F821209A4200
:109650003C4A13686BDC0BBF23F0060323F00503C1
:1096600043F0010343F00203136070479978344AD2
:10967000586852F82130034442F8213070479978F5
:109680002F4A586852F821301B1A42F8213070478F
:1096900099782B4A5B6852F8210003FB00F342F8EB
:1096A000213070479978264A586852F8213093FB48
:1096B000F0F342F82130704710B4214A9978586885
:1096C00052F8214094FBF0F300FB134310BC42F826
:1096D0002130704799781A4A586852F8213003406F
:1096E00042F8213070479978154A586852F821306D
:1096F000034342F8213070479978114A586852F86C
:109700002130434042F82130704799780C4A52F892
:109710002130DB4342F8213070479978084A5B6872
:1097200042F8213070470322074B1A70704723F02C
:10973000030343F004031360704700BF08230020B5
:109740000C25002010230020FC240020034A044B99
:10975000126898785A6001F041BC00BF24240020B0
:1097600008230020F0B400254FF0FF342B46294693
:109770000F4F104E104A11483D703570C1540133DF
:109780002F2B42F8044FF9D101270D4A0D4B526897
:109790000D4E0E4C1A600E4D0E480F4A0F4B37708F
:1097A00021702960016011601960F0BC704700BF32
:1097B000FC220020BC24002064230020C8240020B8
:1097C0000823002058240020BD240020042300206A
:1097D000C424002024240020082500201023002079
:1097E0000648074A417852F82130013B002B42F8E5
:1097F000213002DD4268034B1A60704708230020C5
:109800000C25002058240020024A034B12685A609D
:1098100001F0CCBB2424002008230020024A034B83
:1098200012685A6001F0CABB2424002008230020DB
:10983000044B1B68FF2B04D80349044A496842F8CB
:109840002310704708250020082300200C25002045
:109850000B4B1B68FF2B0CD80A4A0B4952F82330DC
:109860000A4A0B6053600A4A23B1136823F00803C5
:1098700013607047136843F008031360704700BF1C
:10988000082500200C25002024240020FC24002092
:1098900010230020044B1B68FF2B04D80349044A03
:1098A000096842F82310704708250020242400206E
:1098B0000C2500202E4A1368072B1BD870B42D48A6
:1098C00041780C2915D8DFE801F04E49443F3A347D
:1098D0002F2A25201B16070027490968C90508D526
:1098E000264946680D68264C581C0E6044F82350E3
:1098F000106070BC7047204909680C06F9D5EFE785
:109900001D4909684D06F4D5EAE71B4909688E062A
:10991000EFD5E5E718490968C906EAD5E0E7164931
:1099200009688C07E5D0DBE7134909688D07E0D5A6
:10993000D6E71149096811F0050FDAD0D0E70E49D2
:1099400009684E07D5D5CBE70B490968C907D0D4BC
:10995000C6E709490968CC07CBD5C1E706490968BC
:109960000D07C6D4BCE7044909680E07C1D5B7E79F
:10997000C4240020082300201023002058240020A5
:1099800038240020034A52F82030194342F82010AE
:10999000704700BF1C290020024A1368184310605A
:1099A000704700BF1C290020034A52F8203023EAE8
:1099B000010142F8201070471C290020024A136858
:1099C00023EA0000106070471C2900203AB9074ABA
:1099D00052F8203023EA010142F820107047034A70
:1099E00052F82030194342F8201070471C290020FB
:1099F000034B53F820300B4214BF01200020704766
:109A00001C290020034A52F8203023F0610342F859
:109A1000203070471C2900200246054B53F82000D7
:109A200053F8221021F0610143F82210704700BF63
:109A30001C2900200246064B53F8200053F8221040
:109A400000F06B0021F0610143F82210704700BF65
:109A50001C29002000232DE9F041454C82B00193E0
:109A600023786568013B042B7FD8DFE803F01E43B1
:109A70002640030001AAE9B2280E01F0C9FA0198B4
:109A80002269237D1040E268D840237A9042CCBFFF
:109A9000012400248CBF01210021062B63D8DFE8BC
:109AA00003F05A534C4740392E0001ABEAB2280E5E
:109AB000062101F07FFB0198E2E72E0EC5F3072790
:109AC0003946304606F012FAC5F307428046394659
:109AD000304606F02DFAE9B2304606F007FA424663
:109AE00001903946304606F023FA0198C8E7FDF7A1
:109AF000EBFEC5E7E9B2280E06F0F8F9C0E71D4B0A
:109B00009A788A4201D002221A705C70997002B071
:109B1000BDE8F081174B9D78002DF6D09042F2D928
:109B2000F3E7144B9D78002DEFD19042EBD8ECE792
:109B3000104B5A78A242E6D1E7E70E4B5D78002D34
:109B4000E3D09042DFDDE0E70A4B5D78002DDCD109
:109B50009042DADDD7E70222064B1A705C709970EA
:109B600002B0BDE8F081034BCFE7002088E700BFDB
:109B700040290020FC000020024B1B78012B00D064
:109B8000704767E7FC0000202DE9F04F3F4C85B09F
:109B9000E3784BB12378012B27D03D4E63683268C0
:109BA00001339342636002D205B0BDE8F08F002715
:109BB00023786760022BF7D1364D05F120092B7809
:109BC0001BB90835A945FAD1EEE7D4F80880013B66
:109BD00008F101020397A260D5F804A0042B53D822
:109BE000DFE803F0473F1F1B0600FFF733FFD4E712
:109BF00003AA5FFA8AF14FEA1A6001F009FAA26833
:109C00000398736804EB88089342C8F80C00D8D80E
:109C1000032200232270E370C6E7FDF755FEA26819
:109C2000EFE74FEA1A6BCAF3072319465846019328
:109C300006F05CF9019BCAF30742194600905846AA
:109C400006F076F95FFA8AF1584606F04FF9019B63
:109C5000009A03901946584606F06AF9A2680398DC
:109C6000CFE75FFA8AF14FEA1A6006F03FF9A2687F
:109C7000C7E75FFA8AF203AB4FEA1A60062101F0E8
:109C800099FAA2680398BCE70020BAE7FC0000201C
:109C90001000002020290020F0B50024134822469F
:109CA0000346134903F8084BC47043F8042F8B4252
:109CB000FBD14FF0010E4FF4FA674FF0FF360D491C
:109CC0000D4B0E4C0E4D0A758260C4F800E06760C3
:109CD0000E610A704A60C5F8542E1A705A601A72E2
:109CE000DA601A745A611A76DA61F0BDFC0000205D
:109CF00044200020402900202029002010000020BE
:109D0000F4110020B0F5FA6F28BF4FF4FA60014B50
:109D10005860704710000020014B1860704700BF6A
:109D20001000002005280FD80B4B1B7863B930B406
:109D30000A4A12F8334002EBC3053CB10133042B4D
:109D4000F7D130BC002070470020704702F8330084
:109D50006960012030BC7047FC00002020290020F1
:109D60000528034607D8054A127822B9044A01207B
:109D70001370516070470020704700BFFC00002046
:109D800040290020014B18611975704740290020B7
:109D900006281AD82DE9F043354D83B02B7883B9C6
:109DA000344C237800B193B10022013B2072E16072
:109DB00001926668042B58D8DFE803F02932385343
:109DC0000D00002003B0BDE8F08300207047184666
:109DD00003B0BDE8F083F1B201AA300E01F018F92A
:109DE000E16801982269237D1040D8408842C8BFAD
:109DF00001224FF00100D8BF00228CBF01230023B5
:109E00006A70AB702870E87003B0BDE8F08306217B
:109E100001ABF2B2300E01F0CDF9E1680198E1E753
:109E2000F1B2300E06F062F8E168DBE7370EC6F3F8
:109E300007284146384606F059F8C6F307428146DE
:109E40004146384606F074F8F1B2384606F04EF84E
:109E5000414601904A46384606F06AF8E1680198A2
:109E6000C0E7FDF731FDE168BCE70020BAE700BFBD
:109E7000FC00002040290020014B1878704700BFEB
:109E8000FC000020054B9A68824205D903EB800351
:109E9000DB6801200B60704700207047FC00002049
:109EA00003280ED8DFE800F0020A070404207047F8
:109EB000054B9868704742F2107070474FF4FA6093
:109EC00070474FF0FF307047FC000020FF2803462A
:109ED00009D0032805D8064A012012F833300B7048
:109EE000704700207047034B01201B780B707047B0
:109EF0002029002040290020FF2803460AD00328FB
:109F000006D8074A012002EBC3035B680B60704769
:109F100000207047034B01205B680B60704700BF57
:109F20002029002040290020F0B5012187B04FF4FE
:109F30008040FBF7BFFB01210820FBF7AFFB182493
:109F400003254FF420431D4E69463046ADF80030DE
:109F50008DF802508DF80340FAF7E0FF4FF480438C
:109F6000694630468DF80250ADF8003001268DF874
:109F700003400227FAF7D2FF00234FF4827E4FF40A
:109F800000720F4D01A92846ADF80430ADF8083035
:109F9000ADF81230ADF81430ADF806E0ADF80E2093
:109FA000ADF81040ADF80A70ADF80C60FCF730FC6D
:109FB00031462846FCF7BAFC07B0F0BD000C014062
:109FC00000380040F8B50E4615460746FDF70EFA74
:109FD0000D4C02212046FCF73BFD0028F9D031460C
:109FE0000948FCF7D7FC084C01212046FCF730FD5E
:109FF0000028F9D00448FCF7CFFCC4B215B13846AC
:10A00000FDF7FCF92046F8BD00380040704700BF5E
:10A01000F8B50E4615460746FDF7F8F90D4C022136
:10A020002046FCF715FD0028F9D031460948FCF719
:10A03000B1FC084C01212046FCF70AFD0028F9D0AC
:10A040000448FCF7A9FCC4B215B13846FDF7E6F99F
:10A050002046F8BD003800402DE9F041684D044627
:10A060002B78002B7BD1032C2C707ED04BD8012C6D
:10A0700000F09F80022C40F0948000234FF0320CBF
:10A080000A264FF47A7710200E224FF00D0E5D490C
:10A090000B805D49A1F800C05C490E705C4E5D49C3
:10A0A00037805D4E087033705C485D495D4B5E4E95
:10A0B00002705E4F0A705E481C705E4986F800E0D0
:10A0C0005D4B5E4E02705E4C5E485F4A3B605F4F88
:10A0D0000E6017605E495F4E5F4F20605F480E6004
:10A0E00007605F4A5F4E6049604F16606048614E8E
:10A0F000614A0F6061490660116098472B78002B18
:10A1000053D1BDE8F081042C72D0C82C49D102276C
:10A1100032260A244FF47A7E00223A493A480F80C8
:10A12000574B068039493A480C7093F86860A0F89C
:10A1300000E093F869403749374893F86A70374B25
:10A140000E7004703649374E374C39481F700A700C
:10A15000364F3270384B3749384E2270B2E73A4B9F
:10A160001B689847032C2C7080D14FF0010E3224CD
:10A170000A274FF47A761223002222482249A0F8B7
:10A1800000E022480C8007702149224C2248234FCE
:10A190000E80237022490270224E234C24483B70CB
:10A1A000D5E700232B70BDE8F0812368BDE8F041BE
:10A1B00018471E4F334B1F49334E3448224A204C18
:10A1C0003B60334F0E6017602149324E324F2060A2
:10A1D00022480E600760224A304E2349304F1660F5
:10A1E0002348304E244A0F602F490660116084E7EF
:10A1F0004FF0010E32240A274FF47A761323BBE77F
:10A200004C2000209629002090290020AB29002016
:10A21000A82900209A29002093290020AF29002096
:10A22000AD290020AC290020B229002058290020A7
:10A2300092290020742900201DA90008B1AB000854
:10A2400064290020D5AB00087829002019AC00084B
:10A250007029002009AC0008FDAB00086C29002023
:10A260007C29002051AC0008602900205DAC00086A
:10A270005C290020A5AC00086829002041AE000838
:10A280002C2100206DA4000839A6000861A6000852
:10A29000ADA600089DA6000891A60008E5A6000846
:10A2A000F1A6000839A7000895A80008014B187806
:10A2B000704700BF4C200020034B1B7803B9704748
:10A2C000024B1B68184700BF4C2000205829002073
:10A2D000034B1B7803B97047024B1B68184700BF3C
:10A2E0004C20002074290020034B1B7803B97047D1
:10A2F000024B1B68184700BF4C2000206429002037
:10A30000034B187800B97047024B1B68184700BF11
:10A310004C2000206C290020034B187800B97047AE
:10A32000024B1B68184700BF4C20002070290020FA
:10A33000034B1B7803B97047024B1B68184700BFDB
:10A340004C20002078290020034B187800B9704772
:10A35000024B1B68184700BF4C20002060290020DA
:10A36000034B1B7803B97047024B1B68184700BFAB
:10A370004C2000207C290020684620F007018D46F3
:10A38000562101B50648FCF791FB064B1B7813B12B
:10A39000054B1B689847BDE801408546704700BFE4
:10A3A000003001404C2000205C290020684620F04D
:10A3B00007018D46012101B50648FCF71DF8064B43
:10A3C0001B7813B1054B1B689847BDE801408546D3
:10A3D000704700BF000800404C2000206829002082
:10A3E00010B5FDF723F8072400BF013CFCD1102174
:10A3F0001348FCF7CFFA1248FCF7CEFA012260218D
:10A400000F48FCF7AFFA01210E48FBF7F5FF214694
:10A410000C48FBF779FF4FF4AF710A48FBF776FF62
:10A4200001210848FBF7D8FC012206481146FBF73A
:10A4300001FD0121044A054B11701C7010BD00BFC5
:10A4400000300140000800408C29002086290020AF
:10A4500000EBC0030448DB00A0FB0323DB0802D0B1
:10A4600000BF013BFCD17047CDCCCCCC2DE9F047EF
:10A470008AB0FCF7F3FF01214FF48050FBF70EF98F
:10A4800001210420FBF70AF90126A02218234FF02E
:10A4900004094FF0400A1027DFF8888169464046DA
:10A4A000ADF800208DF803308DF80260FAF736FD24
:10A4B00069464046ADF800A08DF80390FAF72EFDEE
:10A4C000694640468DF80260ADF800708DF8037063
:10A4D000FAF724FD4FF4827100244FF40072282310
:10A4E000484DC8F810702846ADF8161005A9ADF80B
:10A4F0001E20ADF820304FF00608ADF81440ADF83E
:10A500001840ADF81A40ADF81C40ADF82240ADF847
:10A510002440FCF77DF923230DEB09008DF804306E
:10A520008DF807608DF806408DF80580FAF720FE5B
:10A5300051462846FCF792FA28462021FCF78EFA6D
:10A5400039462846FCF78AFA39462846FCF786FA47
:10A55000224628467121FCF705FA2246284660214A
:10A56000FCF700FA224628465021FCF7FBF9314659
:10A570002846FCF7DBF9A5F5943531464846FBF74C
:10A5800099F821462846FBF727FC4FF6FF7348222F
:10A59000284602A9ADF80C30ADF80820ADF80A4005
:10A5A000ADF80E408DF81040FBF768F928460821F9
:10A5B000FBF77CFE31462846FBF75CFE224631461F
:10A5C0002846FBF737FC1E230DEB09008DF80760CA
:10A5D0008DF804308DF805808DF80640FAF7C8FD37
:10A5E000094F0A4D0A480B490B4A0C4B0C4E3C7064
:10A5F00034802C8004800C7014701C700AB0BDE88C
:10A60000F08700BF003001408C2900208A290020FB
:10A6100082290020882900208729002086290020FF
:10A620008429002000080140024B1B7803B17047C9
:10A63000D6E600BF8C290020064A137803F0FF01FC
:10A640002BB9054B054801701970137803B1704799
:10A65000C6E600BF8C290020872900208829002019
:10A66000084A137853B9012010B403F0FF01064CD7
:10A67000064B2170187013780BB110BC704710BCDA
:10A68000AEE600BF8C290020882900208729002001
:10A69000014B188880B270478A2900200022024BA3
:10A6A00018781A70704700BF8829002010B50A4C2E
:10A6B000002260210948FCF755F9002220460121BB
:10A6C000FBF7B8FB20460021FBF786FBFCF7B4FE46
:10A6D0000022034B1A7010BD0008004000300140FA
:10A6E0008C290020014B1880704700BF842900206E
:10A6F00010B50E4B93F8300050B90D4B1C8804F088
:10A70000A3F90C4B1B889BB200FB134080B210BD19
:10A71000002004F099F9074B054A1B8812889BB268
:10A7200000FB03F0801A80B210BD00BF2C21002076
:10A730008429002082290020F8B54D48FCF72CF927
:10A7400005464B4C80212046FCF782F90028F9D1C0
:10A75000152300BF013BFCD1FCF76EFE2B2400BF8C
:10A76000013CFCD1434E3378DBB2032B36D0042BB3
:10A7700018D0022B00D0F8BD102D40D03E4A1378DF
:10A78000322B57D013780133DBB21370FCF74EFE37
:10A79000072300BF013BFCD1BDE8F840002134484D
:10A7A000FCF7F8B80127354B354A1B78DFF8E0E0B5
:10A7B00045EA03239BB21380138860219BB21B01DF
:10A7C0009BB222462A48AEF80030FCF7CBF82D4A5F
:10A7D0002D4B17701B78ABB93470F8BD0423274A92
:10A7E000EDB215703370FCF721FE072300BF013B6B
:10A7F000FCD1BDE8F84000211D48FCF7CBB803238D
:10A800003370C3E739462148FBF7F6FD21461F4860
:10A81000FBF77AFD64211D48FBF778FD39461B489C
:10A82000FBF7DAFA3A4639461848FBF703FB0523EB
:10A830003370F8BD224660210D48FCF793F80121E2
:10A840001248FBF7D9FD21461048FBF75DFD642156
:10A850000E48FBF75BFD01210C48FBF7BDFA012216
:10A860000A481146FBF7E6FA05233370F8BD00BF2E
:10A87000003001408C2900208629002080290020FA
:10A880008A2900208829002087290020000800400C
:10A890008229002038B5154D2C78E4B2012C07D060
:10A8A000052C04D100232B702B78DBB138BD38BDCB
:10A8B000002221460E48FBF7BDFA00210C48FBF7A9
:10A8C0008BFAFCF7B3FD602122460A48FCF74AF8F0
:10A8D000072100BF0139FCD10648FCF75BF80223D1
:10A8E0002B7038BDBDE838407AE500BF8C290020C8
:10A8F00000080040003001400723C2B28008013B3D
:10A90000424013F0FF03D2B2F8D102F00300A0F1ED
:10A910000300B0FA80F04009704700BF2DE9F04F06
:10A920008BB0FCF7A3FD01214FF48050FAF7B6FE7F
:10A9300001210420FAF7B2FE012618234FF0200B64
:10A940004FF004094FF0400A10275B4C694620463F
:10A950005A4D8DF803308DF80260ADF800B0FAF76B
:10A96000DDFA69462046ADF800A08DF80390FAF7AD
:10A97000D5FA694620468DF80260ADF800708DF872
:10A980000370FAF7CBFA276128460021FBF7CEFFC8
:10A99000022100244FF4827E4FF4007228232846BF
:10A9A000ADF81A1005A9ADF816E0ADF81E20ADF807
:10A9B0001C60ADF820304FF00608ADF81440ADF83B
:10A9C0001840ADF82240ADF82440FBF721FF2323C7
:10A9D0000DEB09008DF804308DF807608DF8064006
:10A9E0008DF80580FAF7C4FB51462846FCF736F887
:10A9F00059462846FCF732F839462846FCF72EF827
:10AA000039462846FCF72AF8224628467121FBF7EA
:10AA1000A9FF224628466021FBF7A4FF22462846CC
:10AA20005021FBF79FFF31462846FBF77FFFA5F536
:10AA3000943531464846FAF73DFE21462846FBF755
:10AA4000CBF94FF6FF734822284602A9ADF80C3027
:10AA5000ADF80820ADF80A40ADF80E408DF8104072
:10AA6000FAF70CFF28460821FBF720FC3146284660
:10AA7000FBF700FC224631462846FBF7DBF91E2394
:10AA80000DEB09008DF807608DF804308DF8058016
:10AA90008DF806400026FAF76BFB0027084D0948A1
:10AAA00009490A4A0A4B2C700460C1E90067147016
:10AAB0001C700BB0BDE8F08F000801400030014071
:10AAC000AA290020B4290020A0290020AE290020B6
:10AAD000B129002038B5FCF7B5FC20232C4A002111
:10AAE000536113682B4823F4700343F4401313603D
:10AAF000FBF772F901212748FBF77EFC002125486E
:10AB0000FBF702FC012207212248FBF723FA4FF64C
:10AB1000FF712048FBF7FAFB01211E48FBF75CF9A7
:10AB2000002201211B48FBF785F91B4D194C2046DB
:10AB3000FBF744FC2B789842F9D300211548FBF72A
:10AB4000E3FB2023124A002113611368134823F406
:10AB5000700343F430031360FBF71CFF0F48FBF74F
:10AB60001BFF012260210D48FBF7FCFE01240020A1
:10AB700000210B4A0B4B1470C3E900010A4B0B4A2E
:10AB80001B780733DB10013BDBB2137038BD00BF0D
:10AB90000008014000080040AB29002000300140BF
:10ABA000AA290020A02900209A290020B0290020ED
:10ABB000054B1B7803F0FF0203B170470349044BB8
:10ABC0000A701A70FFF786BFAA290020AE2900205C
:10ABD000B1290020064B1B7803F0FF0203B1704738
:10ABE00001210448044B02701970FFF773BF00BFC6
:10ABF000AA290020AE290020B1290020014B1868A5
:10AC0000704700BFB42900200022024B18781A7048
:10AC1000704700BFAE29002010B50A4C0022602109
:10AC20000948FBF79FFE002220460121FBF702F9AD
:10AC300020460021FBF7D0F8FCF70AFC0022034B6A
:10AC40001A7010BD0008004000300140AA29002001
:10AC5000014B1880704700BF9429002010B50E4B9F
:10AC600093F8300050B90D4B1C8803F0EDFE0C4BEF
:10AC70001B889BB200FB134080B210BD002003F084
:10AC8000E3FE074B054A1B8812889BB200FB03F0CA
:10AC9000801A80B210BD00BF2C2100209429002012
:10ACA00098290020F8B55848FBF776FE574D584CC8
:10ACB0002B78D4E90067DB009840064347EAE07749
:10ACC000C4E900672B78002B40F08B8003F0FF0273
:10ACD00060214D48FBF746FEFCF7BAFB4D4A4E4D4E
:10ACE00013781278073323F007039B1AC3F120026D
:10ACF000D4E9006707FA02F226FA03F01043A3F141
:10AD0000200227FA02F227FA03F11043C4E90001F6
:10AD10002B889BB2C3B9D4E90023072391B2D2B2E6
:10AD20008908013B4A4013F0FF03D2B2F8D102F088
:10AD30000302032A08D0394B1B7803F0FF02002BD3
:10AD40002BD1374B1A70F8BD01223649364B0A70A9
:10AD500030CC1B78354EDBB23778C3F1200024FAB3
:10AD600003F105FA00F0203B25FA03F3BA40014352
:10AD70001943013A2E4B0A401A603278102A39D909
:10AD80001B6832782B49103AD3409BB20B80234B7F
:10AD90001B7803F0FF02002BD3D000212648FBF7DD
:10ADA0001BF801212448FBF727FB00212248FBF771
:10ADB000ABFA012248212048FBF7CCF81F4B1E4874
:10ADC000198889B2FBF7A2FA01211B48FBF704F8A6
:10ADD000012219481146FBF72DF80222104B1A7078
:10ADE000F8BD00210848FBF7D5FD2B78013BDBB20D
:10ADF0002B70F8BD1B6832780E49C2F110029340E7
:10AE00009BB20B8097E700BF00300140B0290020C3
:10AE1000A02900209A29002096290020B12900208D
:10AE2000AA290020AE29002093290020AF29002064
:10AE3000B429002098290020000800409029002013
:10AE40000022024B1A70FFF745BE00BFAA2900205E
:10AE500038B500242046FCF71DFB104B204683F834
:10AE60005C4004F069FE72B6FAF742F90C4D0D4BE6
:10AE700021461C602846F9F7A7FF2846F9F7EAFEA5
:10AE80000948F9F731FDF9F7AFFC0848FAF77AFC01
:10AE90002046BDE83840FCF7C3BC00BF2C21002091
:10AEA0000800024010E000E000240140002C0140B6
:10AEB000FFF788B8FFF7ACB810B5144605F016F8E0
:10AEC000206010BD05F034B810B5144605F078FBCD
:10AED000206010BD05F096BB0022F8B52648274F2C
:10AEE000274E284D284C294B11463A6032602A6083
:10AEF0002260027003F5806243F8041F9342FBD185
:10AF0000234D2B7E73B940F21A7440F2FA77214E2A
:10AF10000422A4F21A71204631441444FDF74CF97E
:10AF2000BC42F5D100234FF0FF311C461A4A1B48A2
:10AF3000C45401332F2B42F8041FF9D10024184EBA
:10AF4000E0B2FCF7F9FA0134082C06F8010FF7D14A
:10AF500001210020FCF710FB0021124C2072084652
:10AF6000FCF70AFB6B7D207313B90F4A1370F8BD11
:10AF700001220D4B1A70F8BD042300205824002034
:10AF8000242400200825002010230020082500206C
:10AF90009C2100200C25002064230020C8240020D0
:10AFA0004F20002050200020BD240020024B596873
:10AFB0009878494203F0D0BC08230020024B59681E
:10AFC000987803F0C9BC00BF08230020024B002181
:10AFD000987803F0C1BC00BF082300200A4B9A7880
:10AFE00032B95A7862B1012A06D1596803F008BD16
:10AFF0000422064B1A7070470322044B1A707047E4
:10B00000596803F0CDBC00BF08230020FC240020B9
:10B0100030B5044683B01546392900F2C780DFE811
:10B0200001F0C1BCB7B3ADA6A09B968E888172C556
:10B03000C5C5C5C5C5C5C5C5C5C5C5C5C5C5C5C5C0
:10B04000C5C5C5C5C5C5C5C5C5C5C5C5C5C5C5C5B0
:10B05000C5C5C5C56C664D4B49472B1D18226F21D0
:10B06000204604F065FF20466E2104F03FFF642374
:10B070002860184603B030BD0621204604F0A2FF28
:10B0800020224E21204604F053FF2A684D212046FD
:10B0900004F04EFF21224E21204604F049FF2046B5
:10B0A00001224D2104F044FF6423184603B030BD53
:10B0B0001522D4E70521E0E71622D0E7042104F0A9
:10B0C00081FF20224E21204604F032FF2A684D21C4
:10B0D000204604F02DFF21224E21204604F028FFB7
:10B0E00020460A224D2104F023FF6423C1E72421D6
:10B0F00004F0FCFE64232860BBE71268242104F0FE
:10B1000017FF6423B5E7002302A941F8043DFEF7C9
:10B11000F3FE002814BF642309231846019A2A600D
:10B1200003B030BD002302A941F8043DFEF7CEFE76
:10B13000EFE71068FEF7B4FE6423286099E7002368
:10B1400002A941F8043D1068FEF79CFEE1E7FEF716
:10B1500093FE642328608CE71168FEF719FE6423D0
:10B1600087E701461068FEF70DFE642381E711684A
:10B17000FEF7F6FD002897D109237AE71168FEF75C
:10B18000D1FD002890D1F7E71068FEF7C5FD8BE7E9
:10B190001368002B88D004236BE71068FEF7B2FD1C
:10B1A000642366E7FEF778FD642362E7032360E724
:10B1B000704700BF30B51C4683B0002840F00581C1
:10B1C000FF2A00F27687DFE812F030012D0628060C
:10B1D0001D060906340521057407740774073E0629
:10B1E0000F05C605B305A0058D0517040E0451060D
:10B1F0000504C704A704740774077407B50495040D
:10B200007407740774076D046404590450047407C8
:10B2100074077407740774077407F204E904E00400
:10B22000CE0480036E0374077407740774077705F0
:10B2300065034207980685065B064E077407740788
:10B240007407740774077407740774077407740726
:10B25000740774077407EE060107FD0461072607EB
:10B2600038078305C803B803BE06A403FF057407A7
:10B270007407740774077407740774077407EC0580
:10B28000DB06D905C80644047407740774077407FD
:10B2900074073204200464055A0514074705AB06F9
:10B2A000460339032D037F0274077407740774077C
:10B2B000740774077407740774076D0292035B02C6
:10B2C000F501E301E5027407740774077407740756
:10B2D0007407740774077407740774077407740796
:10B2E0007407D10112030003740724037407740761
:10B2F0007407740774077407740774077407740776
:10B3000074071C02740774077407F303C102E10396
:10B3100093017407530349023702740774077407D3
:10B320007407740774077407740774077407740745
:10B330007407740774077407740774077407740735
:10B340007407740774077407740774077407740725
:10B350007407740774077407740774077407740715
:10B360007407740774077407740774072502BF0114
:10B37000A401D3021201170274077407740774073B
:10B3800074070F02F70274077407740774077407D1
:10B390007407740774070702D203AF0274077407B7
:10B3A00074077407740774077407B7028A01810170
:10B3B0005D016F014B017801540166014201740780
:10B3C00074077407740774073701042306290BD127
:10B3D000C64A127842B12268C5490A60FAB1C54925
:10B3E0000A6822F008020A60184603B030BD062938
:10B3F0001ED1C14D95F8333013F0040001F0728373
:10B4000002210020FCF7B8F8012800F09280002209
:10B41000B64B22601B785BB16423B5490A60B5491D
:10B420000A6842F008020A60DEE7062901F05E8140
:10B430006423184603B030BD052900F09E87062915
:10B44000F6D10020FCF72EF820606423C0E7052920
:10B4500001F031820629EBD105F00EFA2060F4E705
:10B46000052901F01C820629E2D105F0D5F92060FA
:10B47000EBE7052901F02B820629D9D105F0E4F983
:10B480002060E2E7052901F09E800629D0D105F071
:10B49000ABF92060D9E7052901F013820629C7D14D
:10B4A00005F0DEF92060D0E7052901F0FE810629CC
:10B4B000BED105F0A5F92060C7E7052901F00D828E
:10B4C0000629B5D105F0B4F92060BEE7052901F0E1
:10B4D00097810629ACD105F07BF92060B5E70529F5
:10B4E00001F059810629A3D105F066F92060ACE787
:10B4F000052901F09581062900F09E87072901F0B2
:10B50000FE82082994D104227C496C20FCF754FE69
:10B510008EE706298CD1784D95F8333013F0010170
:10B5200001F0D38200210846FCF726F801287FF4B9
:10B530006EAF01226D4B22601B78002B3FF478AF79
:10B540006B4964230A604AE7052900F0038706294E
:10B5500000F0FC87072901F0498308297FF468AFD0
:10B56000012267497320FCF727FE61E7052901F0F6
:10B570002D81062900F04E87072901F08A820829CB
:10B580007FF456AF01225F499C20FCF715FE4FE780
:10B59000052901F02E80062900F05F87072901F0B8
:10B5A0007F8208297FF444AF012257499420FCF799
:10B5B00003FE3DE7052901F05D81062900F0418782
:10B5C000072901F04A8208297FF432AF02224F494D
:10B5D0009A20FCF7F1FD2BE706297FF429AF05F04F
:10B5E0006FF864232060F3E606297FF421AF02F0B0
:10B5F000E1FE64232060EBE6052900F0D986642390
:10B60000E4E606297FF414AF0020FEF705FA642370
:10B610002060DDE6052900F0A786062900F0768780
:10B62000072901F01B8308297FF402AF0122384962
:10B630007420FCF7C1FDFBE6052901F025810629F0
:10B6400000F00587072901F0D78108297FF4F0AEC3
:10B6500001223049AA20FCF7AFFDE9E6052901F0F7
:10B66000E880062900F0CA86072901F079820829B6
:10B670007FF4DEAE01222849A920FCF79DFDD7E624
:10B68000052901F0C380062900F0D086072901F0C2
:10B69000CF8108297FF4CCAE012220499820FCF705
:10B6A0008BFDC5E6052901F09E80062900F0B886CD
:10B6B000072901F0C48108297FF4BAAE0122184994
:10B6C0009620FCF779FDB3E6052900F015860629DA
:10B6D00000F04887072901F0308308297FF4A8AEDD
:10B6E000042210499020FCF767FDA1E68924002080
:10B6F00024240020102300202C2100205821002089
:10B700005F21002088210020802100208621002048
:10B710006021002096210020952100208421002016
:10B72000822100207C21002006297FF481AE05F0D3
:10B7300023F8642320604BE6052900F0548706298E
:10B740007FF476AE05F02CF820607EE6052900F047
:10B75000E985062900F00B87072901F040820829B6
:10B760007FF466AE0122D5497220FCF725FD5FE625
:10B7700006297FF45DAED24D95F8333013F0020008
:10B7800001F0D28101210020FBF7F6FE01287FF4B1
:10B790003EAECEE6052901F05780062900F034863A
:10B7A000072901F0618108297FF442AE0122C549D1
:10B7B0009520FCF701FD3BE606297FF439AE002019
:10B7C00002F0FEFD6423206002E6052900F0A68752
:10B7D000062900F05486072901F01C8108297FF40E
:10B7E00027AE0122B849A020FCF7E6FC20E6052997
:10B7F00000F0EF86062900F0F085072901F05E8150
:10B8000008297FF415AE0222B0499E20FCF7D4FC33
:10B810000EE606297FF40CAE002004F0DFF9642365
:10B820002060D5E506297FF403AE7621002004F0E0
:10B830005DFB00F0070020606423C9E5052900F0E6
:10B84000EB8406297FF4F4AD9D4B93F83B30C3F3B2
:10B8500080032360F9E5052900F06E8506297FF451
:10B86000E7AD974B93F83B3003F001032360ECE521
:10B87000052900F0CB86062900F0F585072901F09F
:10B88000A68008297FF4D4AD01229149A820FCF7B5
:10B8900093FCCDE506297FF4CBAD002002F06EFECF
:10B8A0006423206094E5052900F04A87062900F00A
:10B8B000F185072901F0B58008297FF4B9AD01228F
:10B8C00084497A20FCF778FCB2E5052900F0FE8374
:10B8D000062900F08885072901F0498108297FF4AD
:10B8E000A7AD04227C494420FCF766FCA0E50529AD
:10B8F00000F00A87062900F0BC85072901F0838043
:10B9000008297FF495AD012274499720FCF754FC77
:10B910008EE506297FF48CAD4FF0FF3300200093B5
:10B92000022301906D226C2104F028FE644A6423F6
:10B93000927D90FBF2F222604AE506297FF478AD11
:10B9400000234FF0FF321846019300926D226C21C4
:10B9500004F014FE642320603AE506297FF468AD04
:10B9600000204FF0FF320B4601900092DAE70629E3
:10B970007FF45EAD1821002004F0B8FA584B82B273
:10B98000013293FBF2F26423226021E5052900F0E5
:10B990001A85062900F0E085072901F0EF800829C3
:10B9A0007FF446AD01224F497020FCF705FC3FE5CE
:10B9B000052900F0CE83062900F07B85072901F0D8
:10B9C000E48008297FF434AD012247496B20FCF75D
:10B9D000F3FB2DE506297FF42BADFEF7B5FC00B295
:10B9E00020606423F4E406297FF422AD002003F0F4
:10B9F000F3F864232060EBE406297FF419AD0020FE
:10BA000003F0DEF864232060E2E4052900F0AB8651
:10BA1000062900F09D86072900F0AF8708297FF4EA
:10BA200007AD012231495B20FCF7C6FB00E5052983
:10BA300000F0E383062900F05F87072901F02280E8
:10BA400008297FF4F5AC042229496420FCF7B4FBF3
:10BA5000EEE406297FF4ECAC7621002004F046FAEF
:10BA6000C0F3022020606423B2E406297FF4E0AC36
:10BA7000002002F0C9FC64232060A9E4052900F03D
:10BA8000098606297FF4D4AC002002F0C3FC2060B4
:10BA9000DBE406297FF4CCAC002002F0AFFC642389
:10BAA000206095E4052900F0198606297FF4C0ACD2
:10BAB000002002F0D5FC2060C7E400BF5E2100201A
:10BAC0002C210020812100208C2100208A210020AF
:10BAD00094210020662100203021002083210020B5
:10BAE00000E1F5055C2100205721002047210020BE
:10BAF00050210020052900F0DB85062900F0D285C1
:10BB0000072900F0488708297FF492AC0122E14917
:10BB10005920FCF751FB8BE406297FF489AC002007
:10BB200003F054F80546002003F04AF82B1A1BB224
:10BB300023608AE4052900F0C985062900F0C08544
:10BB4000072900F02F8708297FF472AC0122D2491F
:10BB50005A20FCF731FB6BE406297FF469AC002026
:10BB600003F03AF8DEE7052900F0E285062900F047
:10BB70008C84072900F0328708297FF459AC04220D
:10BB8000C6494020FCF718FB52E406297FF450AC6C
:10BB9000002002F073FC6423206019E406297FF47E
:10BBA00047AC002002F064FC6423206010E4052907
:10BBB00000F05A8506297FF43BAC002002F052FCCD
:10BBC000206042E4052900F0F082062900F07C8420
:10BBD000072900F0EF8708297FF42AAC0222B04938
:10BBE0008820FCF7E9FA23E4052900F09A82062967
:10BBF00000F0A586072900F0F88608297FF418AC24
:10BC00000422A8494C20FCF7D7FA11E4052900F0DA
:10BC10003985062900F03085072900F0B586082906
:10BC20007FF406AC0222A0495020FCF7C5FAFFF7CA
:10BC3000FFBB052900F0BF84062900F0B684072960
:10BC400000F0768608297FF4F3AB02229749522050
:10BC5000FCF7B2FAFFF7ECBB052900F06D8206296C
:10BC600000F04E84072900F0B38708297FF4E0AB89
:10BC700002228F496020FCF79FFAFFF7D9BB062903
:10BC80007FF4D6AB854A642392F82A202260FFF71E
:10BC90009FBB052900F07582062900F01B84072947
:10BCA00000F0C78708297FF4C3AB012281495C20DB
:10BCB000FCF782FAFFF7BCBB052900F0CE84062909
:10BCC0007FF4B6AB002002F03BFC2060FFF7BDBB69
:10BCD00006297FF4ADAB4FF0FF33002000930190B5
:10BCE000052333E6052900F06985062900F0608503
:10BCF000072900F0168608297FF49AAB01226E49C5
:10BD00005820FCF759FAFFF793BB052900F08F8400
:10BD1000062900F08684072900F04B8608297FF465
:10BD200087AB012265495720FCF746FAFFF780BB35
:10BD3000052900F08A84062900F08184072900F093
:10BD40003F8608297FF474AB01225D49A120FCF7EE
:10BD500033FAFFF76DBB052900F00982062900F0D0
:10BD6000AE83072900F01F8708297FF461AB042206
:10BD700054494820FCF720FAFFF75ABB052900F088
:10BD80000882062900F0ED85072900F0BF86082902
:10BD90007FF44EAB01224C497720FCF70DFAFFF7F8
:10BDA00047BB052900F01282062900F0CE8507293D
:10BDB00000F0B38608297FF43BAB0122434975208C
:10BDC000FCF7FAF9FFF734BB06297FF431AB4FF0EB
:10BDD000FF330020009301900323B7E506297FF489
:10BDE00027AB1221002004F081F84FF6FE12001458
:10BDF00000F5F9437F33934288BF0020642320601D
:10BE0000FFF7E6BA06297FF413AB1321002004F0F4
:10BE10006DF800B22060FFF718BB06297FF408AB6D
:10BE20001221F3E706297FF403AB00220321104619
:10BE300004F07EF80221002004F058F880B220605F
:10BE40006423FFF7C5BA052900F0CC81062900F06C
:10BE50004A85072900F02B8608297FF4E9AA0122E8
:10BE60001B495620FCF7A8F9FFF7E2BA06297FF430
:10BE7000DFAA002002F0AAFE64232060FFF7A8BA20
:10BE800006297FF4D5AA002002F024FF6423206055
:10BE9000FFF79EBA45210020462100202C210020DA
:10BEA00074210020382100203C2100203E21002068
:10BEB0004C21002048210020442100204321002063
:10BEC0008D210020342100206321002061210020E9
:10BED00042210020052900F0E581062900F02C838D
:10BEE000072900F0598608297FF4A2AA0422D6491E
:10BEF0007C20FCF761F9FFF79BBA052900F09A81D5
:10BF0000062900F01E83072900F05B8608297FF4CC
:10BF10008FAA0422CD498020FCF74EF9FFF788BA9A
:10BF2000052900F0D681062900F0F682072900F0E5
:10BF30008E8608297FF47CAA0222C5496820FCF776
:10BF40003BF9FFF775BA06297FF472AA4FF0FF3369
:10BF50000020009301900123F8E4052900F081847A
:10BF6000062900F04582072900F0858508297FF41D
:10BF70005FAA0222B7497820FCF71EF9FFF758BAEA
:10BF8000052900F09981062900F0BF84072900F0F7
:10BF90005D8508297FF44CAA0122AF497520FCF782
:10BFA0000BF9FFF745BA052900F09A80062900F041
:10BFB0009682072900F0368608297FF439AA0222E2
:10BFC000A6498420FCF7F8F8FFF732BA052900F0FB
:10BFD0005781062900F0AA82072900F03186082936
:10BFE0007FF426AA02229E498620FCF7E5F8FFF797
:10BFF0001FBA052960D0062900F07D82072900F0CC
:10C00000FC8508297FF414AA022296495E20FCF7D9
:10C01000D3F8FFF70DBA052973D0062900F0658221
:10C02000072900F0F88508297FF402AA02228E4928
:10C030008C20FCF7C1F8FFF7FBB906297FF4F8A9BB
:10C040004FF0FF3300200093019004237EE4052984
:10C0500000F0A78306297FF4EBA9002002F0B0FAD4
:10C060002060FFF7F2B9052900F03D81062900F0B4
:10C070005882072900F0C88508297FF4D9A904222D
:10C080007A49A420FCF798F8FFF7D2B9052900F007
:10C090007D81062900F00782072900F047860829DC
:10C0A0007FF4C6A9022272498A20FCF785F8FFF7BF
:10C0B000BFB90323FFF78AB942F2107322689A428C
:10C0C0000BD86C496423CA83FFF78EB9216800201E
:10C0D00002F002FA00287FF4ABA90423FFF784B929
:10C0E0002368B3F5004FF8D2624C9BB21946A4F80E
:10C0F0004430B4F84620002004F024FA6423FFF70B
:10C1000073B92368B3F5004FE7D20022594C9BB2B4
:10C110001946A4F84C30104604F02AFA6423FFF7BD
:10C1200063B94EF6602321689942D6D8002002F008
:10C13000A5FC6423FFF758B922684F4902F5433341
:10C1400003F5A0738B42C8D84A4964230A84FFF7D9
:10C150004BB92368042B01D9C82BBED1454A82F8BC
:10C160002B302078FDF778FF6423FFF73DB94EF6BA
:10C17000602322689A42B0D83E4964238A60FFF760
:10C1800033B92268022AA8D83A4964230A77FFF70C
:10C190002BB92368012BA0D8364A002082F837300B
:10C1A00002F020FD6423FFF71FB92368B3F5004FA9
:10C1B00093D2304C9BB21946A4F84830B4F84A20C8
:10C1C000002004F0CFF96423FFF70EB92368012B98
:10C1D00083D8284A002082F8353002F003FD64231A
:10C1E000FFF702B921684B1EFE2B3FF676AF002009
:10C1F00002F036FC6423FFF7F7B82368B3F1807FC1
:10C20000BFF46BAF1B4C1A4663622621002003F07B
:10C210008FFE6423FFF7E8B823681649002B00F06F
:10C22000B58191F83B20642342F0040281F83B2061
:10C23000FFF7DAB82268114B9A423FF64EAF0D492C
:10C2400064230A64FFF7D0B8682100206C21002025
:10C250005421002064210020622100207021002050
:10C26000722100204A210020782100209021002006
:10C27000762100202C210020801A0600A0860100D3
:10C280002368B3F5004FBFF428AFBC4C9BB21A46ED
:10C29000A4F84630B4F84410002004F053F96423A5
:10C2A000FFF7A2B82268B64B9A423FF616AFB349E1
:10C2B0006423CA63FFF798B82368012B3FF60DAFDC
:10C2C000AE4A002082F8363002F08CFC6423FFF77F
:10C2D0008BB82268B2F5803FBFF4FFAEA749642354
:10C2E0000A85FFF781B82268052A7FF7F6AEA349D1
:10C2F00064234A66FFF778B82168A24AA1F5C343D0
:10C30000283B93423FF6E9AE9C4B9F4A1965236850
:10C31000182192FBF3F20020013A03F009FE642396
:10C32000FFF762B82268012A3FF6D7AE934964232B
:10C3300081F83220FFF758B82368002B40F00184C1
:10C340008E49642391F83B2022F0010281F83B20C2
:10C35000FFF74AB82268072A3FF6BFAE8749642331
:10C3600081F83320FFF740B82368844A03F00703BD
:10C3700082F834306423FFF737B82068002840F093
:10C380000E81FBF787F86423FFF72EB82368B3F517
:10C39000004FBFF4A2AE794C9BB21A46A4F84A30C3
:10C3A000B4F84810002004F0DDF86423FFF71CB84F
:10C3B000216807293FF691AEC9B20020FBF784F946
:10C3C0006423FFF711B822686C49003218BF0122BC
:10C3D000642381F83020FFF707B8684BB3F85E306C
:10C3E0002360FFF732B8654B5B682360FFF72DB819
:10C3F000624BB3F938302360FFF727B85F4B93F8EF
:10C4000069302360FFF721B85C4B93F85530236007
:10C41000FFF71BB8594B93F85C302360FFF715B852
:10C42000564B93F856302360FFF70FB8534B93F8F1
:10C4300058302360FFF709B8504BDB6A2360FFF7E1
:10C4400004B84E4BB3F85A302360FEF7FEBF4B4B97
:10C4500093F86A302360FEF7F8BF484B93F85430E6
:10C460002360FEF7F2BF454B93F868302360FEF778
:10C47000ECBF424B93F857302360FEF7E6BF3F4BCB
:10C4800093F860302360FEF7E0BF3C4B1B682360ED
:10C49000FEF7DBBF394B93F83A30003318BF012366
:10C4A0002360FEF7D2BF354BB3F84A302360FEF766
:10C4B000CCBF324B93F82B302360FEF7C6BF2F4B17
:10C4C0009B682360FEF7C1BF2C4BB3F84830236054
:10C4D000FEF7BBBF294B1B7F2360FEF7B6BF274B80
:10C4E000B3F844302360FEF7B0BF244BB3F84C30B0
:10C4F0002360FEF7AABF214BDB8B2360FEF7A5BFAD
:10C500001E4BB3F920302360FEF79FBF1B4B93F8FF
:10C5100034302360FEF799BF184B1B8D2360FEF764
:10C5200094BF164B5B6E2360FEF78FBF134BB3F8BF
:10C5300046302360FEF789BF104BDB6B2360FEF7AC
:10C5400084BF0E4B1B6C2360FEF77FBF0B4B93F831
:10C5500033302360FEF779BF084B93F83030236007
:10C56000FEF773BF054B1B6D2360FEF76EBF034BD9
:10C5700093F832302360FEF768BF00BF2C21002003
:10C58000400D0300F824010000E1F50591F83B207F
:10C59000642322F0040281F83B20FEF725BF00202F
:10C5A000FAF770FF6423FEF71FBF002003F018FAAC
:10C5B0002060FEF74ABF2168002003F01DFA002822
:10C5C0007EF436AF89E5206804F008F96423FEF7AD
:10C5D0000BBFC84B22680020A3F85E2003F0ACFA22
:10C5E0006423FEF701BF206804F0D4F86423FEF74B
:10C5F000FBBE2368BF4A003318BF0123002082F826
:10C60000543003F00DFA6423FEF7EEBEB94B2268F6
:10C6100093F82B0083F86820FDF71EFD6423FEF7D6
:10C62000E3BE002002F050FA2060FEF70EBF217832
:10C63000002002F039FA00287EF4FAAE4DE5002021
:10C6400002F060FA2060FEF700BF2178002002F0BF
:10C6500047FA00287EF4ECAE3FE52168002002F0A6
:10C660009FF96423FEF7C0BE2168002002F074F930
:10C6700000287EF4DDAE30E5002003F091F9206063
:10C68000FEF7E3BE2168002003F096F900287EF44F
:10C69000CFAE22E52168002002F038F900287EF4B0
:10C6A000C7AE1AE5002002F06BFA2060FEF7CDBE9F
:10C6B0002178002002F054FA00287EF4B9AE0CE58F
:10C6C000002002F075FA2060FEF7BFBE217800203E
:10C6D00002F05EFA00287EF4ABAEFEE42168002092
:10C6E00002F0E4F800287EF4A3AEF6E40022032171
:10C6F000104603F01DFC0221002003F0F7FB000CA4
:10C7000020606423FEF764BE7A4B2268002083F821
:10C71000572003F085F96423FEF766BE754B226847
:10C72000002083F8602003F007FA6423FEF75CBE64
:10C730002168002001F0B0FE00287EF479AECCE440
:10C740002168002001F0E2FE00287EF471AEC4E40E
:10C750002521002003F0CAFB664BC0F30030D876D9
:10C760002060FEF772BE2368624C003318BF0123BD
:10C770002521E376002003F0B9FBE37E20F480520C
:10C780001B0303F480531A432521002003F0D0FB40
:10C790006423FEF729BE206804F008F86423FEF73E
:10C7A00023BE2168002001F029FF6423FEF71CBE90
:10C7B000002002F0CDF92060FEF747BE217800206E
:10C7C00002F0AAF900287EF433AE86E42368494AD1
:10C7D000003318BF0123002082F85C3003F0ACF96D
:10C7E0006423FEF701BE2368424A003318BF0123C9
:10C7F000002082F8563003F013F96423FEF7F4BDED
:10C80000206803F0DFFF6423FEF7EEBD394B22689A
:10C81000002083F8582003F003F96423FEF7E4BDF9
:10C820002368344A98B2D362FDF79AFD6423FEF779
:10C83000DBBD304B226893F82B0083F86920FDF7AD
:10C840000BFC6423FEF7D0BD23682A4A003318BFCF
:10C850000123002082F8553003F0E2F86423FEF74C
:10C86000C3BD244B226800201A8702F0BBF9642361
:10C87000FEF7BABD1F4B22680020A3F85A2003F030
:10C88000CFF86423FEF7B0BD1A4B226893F82B0053
:10C8900083F86A20FDF7E0FB6423FEF7A5BD20685E
:10C8A00003F0B4FF6423FEF79FBD206803F0A2FFEE
:10C8B0006423FEF799BD206803F0D8FF6423FEF7D8
:10C8C00093BD206803F0C6FF6423FEF78DBD20688A
:10C8D00003F0B4FF6423FEF787BD206803F0A2FFD6
:10C8E0006423FEF781BD002002F0AEF82060FEF761
:10C8F000ACBD00BF2C2100202621002003F0F6FA59
:10C90000DA4B58622060FEF7A0BD3321002003F00F
:10C91000EDFAD64BC0F3003083F836002060FEF706
:10C9200094BD0122D2495820FBF7D6FBFEF780BD0B
:10C930000222D0495220FBF7CFFBFEF779BD002041
:10C9400002F0AAF82060FEF780BD3321002003F03A
:10C95000CDFAC64B00F0010283F835202260FEF7C5
:10C9600074BD3321002003F0C1FAC04BC0F3002096
:10C9700083F837002060FEF768BD0122BE495B20C6
:10C98000FBF7AAFBFEF754BD0222BC495020FBF77F
:10C99000A3FBFEF74DBD0122B9495920FBF79CFBD3
:10C9A000FEF746BD0122B7495A20FBF795FBFEF77B
:10C9B0003FBD0122B4495720FBF78EFBFEF738BD7F
:10C9C0000122B249A120FBF787FBFEF731BD01220E
:10C9D000AF49A820FBF780FBFEF72ABD0422A3493C
:10C9E0004020FBF779FBFEF723BD0422A9494C2028
:10C9F000FBF772FBFEF71CBD0122A749AA20FBF73B
:10CA00006BFBFEF715BD0122A4499720FBF764FBE1
:10CA1000FEF70EBD0222A249A020FBF75DFBFEF748
:10CA200007BD01229F497A20FBF756FBFEF700BDA8
:10CA300001229D499820FBF74FFBFEF7F9BC01222C
:10CA40009A499620FBF748FBFEF7F2BC0122984971
:10CA50007620FBF741FBFEF7EBBC022295499A20BA
:10CA6000FBF73AFBFEF7E4BC012293499520FBF764
:10CA700033FBFEF7DDBC022290497820FBF72CFB4C
:10CA8000FEF7D6BC04228E496420FBF725FBFEF797
:10CA9000CFBC01228B499C20FBF71EFBFEF7C8BCD4
:10CAA000012289499420FBF717FBFEF7C1BC012244
:10CAB00086495620FBF710FBFEF7BABC02228449D8
:10CAC0009E20FBF709FBFEF7B3BC0846FAF754FDBE
:10CAD00000283EF42EAD95F83330D9073EF522AD4F
:10CAE000FEF795BC0221FAF747FD00283EF421AD80
:10CAF00095F833305B077EF58AACFEF781BC0422E3
:10CB000074496C20FBF7E8FAFEF792BC01227249E7
:10CB10007720FBF7E1FAFEF78BBC01226F49752005
:10CB2000FBF7DAFAFEF784BC0121FAF725FD0028AD
:10CB30003EF4FFAC95F833309A077EF568ACFEF70B
:10CB400021BE00222821104603F0F2F94749642350
:10CB500091F83B2042F0010281F83B20FEF744BCF3
:10CB600001225F49A920FBF7B7FAFEF761BC042256
:10CB70005C494420FBF7B0FAFEF75ABC01225A493F
:10CB80007020FBF7A9FAFEF753BC012257496B202E
:10CB9000FBF7A2FAFEF74CBC042255497C20FBF7B8
:10CBA0009BFAFEF745BC042252494820FBF794FA51
:10CBB000FEF73EBC022250498820FBF78DFAFEF7B3
:10CBC00037BC04224D498020FBF786FAFEF730BCC3
:10CBD00002224B496020FBF77FFAFEF729BC0122B5
:10CBE00048497220FBF778FAFEF722BC0122464939
:10CBF0007320FBF771FAFEF71BBC022243495E204B
:10CC0000FBF76AFAFEF714BC04224149A420FBF7A3
:10CC100063FAFEF70DBC02223E498C20FBF75CFA5A
:10CC2000FEF706BC02223C498420FBF755FAFEF7CA
:10CC3000FFBB012239495C20FBF74EFAFEF7F8BB37
:10CC4000022237498620FBF747FAFEF7F1BB0222A2
:10CC500034496820FBF740FAFEF7EABB012232496B
:10CC60007420FBF739FAFEF7E3BB00BF2C2100204C
:10CC7000442100203E210020472100203C210020AB
:10CC80004521002046210020432100208D21002045
:10CC900094210020382100209621002083210020AB
:10CCA0008C21002066210020842100208221002088
:10CCB00062210020862100208121002064210020A3
:10CCC00050210020882100208021002042210020C6
:10CCD0008A210020582100206321002061210020AA
:10CCE00095210020302100205C21002057210020C8
:10CCF0006821002034210020742100206C210020B4
:10CD00004C2100205E2100205F2100204A210020CC
:10CD1000902100207821002070210020482100204F
:10CD200072210020542100206021002002220649A7
:10CD30008A20FBF7D1F9FEF77BBB04220349902040
:10CD4000FBF7CAF9FEF774BB762100207C21002096
:10CD500038B57F4CA378002B40F0C7806378403B08
:10CD6000BF2B00F27E82DFE813F06F0211024C024B
:10CD70007C02C5015E02ED012E027C026B017C0289
:10CD8000FF01B601A7017C027C027C0291013C02FA
:10CD9000D5017C0220027C027C027C027C027C02A7
:10CDA0007C027C027C027C027C027C027C027C0293
:10CDB0007C027C027C027C027C027C027C027C0283
:10CDC0007C027C027C027C027C027C027C027C0273
:10CDD0007C027C027C027C027C027C027C027C0263
:10CDE0007C027C027C027C027C024E0184017C017C
:10CDF000600155017C027C027C027C027C027C0288
:10CE00007C027C027C027C027C027C027C027C0232
:10CE10007C027C027C027C027C027C027C027C0222
:10CE20007C027C027C027C027C027C027C027C0212
:10CE30007C027C027C027C027C027C027C027C0202
:10CE40007C027C027C027C027C027C027C027C02F2
:10CE50007C027C027C027C027C027C027C027C02E2
:10CE60007C027C027C027C027C027C027C027C02D2
:10CE70007C027C027C027C027C027C027C027C02C2
:10CE80007C027C027C027C027C027C027C027C02B2
:10CE90007C027C027C027C027C027C027C027C02A2
:10CEA0007C027C027C027C027C027C027C027C0292
:10CEB0007C027C027C027C027C027C027C027C0282
:10CEC0007C027C027C027C027C023E017C027C02B1
:10CED0007C027C027C027C027C027C027C027C0262
:10CEE0007C027C027C023E014501022B13D0032B05
:10CEF0003AD00422174B1A700A280BD1164A12781E
:10CF000042B1164A5B681360154ADBB1136823F01F
:10CF10000803136038BD6278372A5AD80A2800F00F
:10CF20005D8209285AD00B2800F0B9820C28F1D173
:10CF3000BDE838400B499200114402F21A700422F5
:10CF4000FBF73AB9136843F00803136038BD00BF1C
:10CF500008230020FC240020892400202424002011
:10CF6000102300200C25002063782E2B00F27981FD
:10CF7000DFE813F0DC01A3012602770177017701D6
:10CF800077017701770177017701770177017701E1
:10CF900077017701770177017701770177017701D1
:10CFA00077017701770177017701FE011202EA012B
:10CFB0001C0277017701770177017701770177010B
:10CFC0007701F4010802D20199018F0185017B01EB
:10CFD000B1010A2800F0028209289BD16168C34B85
:10CFE00043F8221038BD0A2894D1C14AC14B1278A7
:10CFF0005A6083E70A2800F0318209288AD1227911
:10D00000BD4B1A7038BD0A2884D1BC4AB94B12787E
:10D010005A6073E70A2800F0F48109287FF47AAF98
:10D02000B44AB74B52681A6038BD0A2800F0EE8146
:10D0300009287FF46FAFAF4AB24B52681A6038BD0F
:10D040000A2800F0D68109287FF464AF21790029ED
:10D0500040F03682AC4BD9751720BDE83840FAF75E
:10D060001FBF0A287FF456AFA84AA24B12685A6025
:10D0700044E70A287FF44EAFA04A9E4B1278A2F1F3
:10D080000402B2FA82F252095A6037E70A2800F025
:10D09000AB8109287FF43EAF9B4D2B7D13F0010F30
:10D0A000237902D0DA0740F177822B751946BDE863
:10D0B00038401420FAF7F4BE0A2800F0E681092867
:10D0C0007FF428AF2379904A194653751520BDE89F
:10D0D0003840FAF7E5BE0A2800F0AC8109287FF451
:10D0E00019AF2379884A194693700220BDE8384069
:10D0F000FAF7D6BE0A2800F0BE8109287FF40AAFED
:10D1000063688149042241F81C3F1C20BDE8384077
:10D11000FAF7E2BF0A2800F0838109287FF4FAAE0B
:10D12000794D042229461020636841F8103FFAF730
:10D13000D3FFF9F773FE2A69A9686879BDE838401A
:10D14000FAF7E4BC0A2800F0A58109287FF4E2AED2
:10D1500063686D49042241F80C3F0C20FAF7BCFFCC
:10D16000BDE83840F9F75ABE0A2800F06D81092859
:10D170007FF4D0AE2379644C19460320E370FAF7AC
:10D180008FFEE078BDE83840FBF7BCB90A2800F014
:10D190006D8109287FF4BEAE23795B4A194613706E
:10D1A0000020BDE83840FAF77BBE0A2800F0338142
:10D1B00009287FF4AFAE6368012B40F2E3810422BB
:10D1C0004C4B1A7038BD0A2800F05A8109287FF4A8
:10D1D000A1AE4D4D63682946042241F8083F08205E
:10D1E000A5E70A2800F02B8109287FF493AE636835
:10D1F0004549042241F8203F2020BDE83840FAF795
:10D200006BBF0A2800F0118109287FF483AE2379CF
:10D210003D4C1846637003F011FB61780120BDE8B6
:10D220003840FAF73DBE0A2800F0138109287FF440
:10D2300071AE2379344A194605205371FAF730FE4E
:10D24000BDE83840F9F7EABD0A2800F03281092824
:10D250007FF460AE217940F2FF70BDE83840FAF704
:10D260001FBE0322234B1A7046E60A2800F04381B2
:10D2700009287FF44FAE6268254B9A6238BD0A28B0
:10D2800000F03E8109287FF445AE6268204B5A6267
:10D2900038BD0A2800F0398109287FF43BAE626866
:10D2A0001B4B1A6238BD0A2800F01B8109287FF445
:10D2B00031AE6268164BDA6138BD0A2800F007818A
:10D2C00009287FF427AEFAF7FFFA62681149104B7C
:10D2D00048605A6038BD0A2800F01C8109287FF494
:10D2E00019AE62680A4BDA6238BD00BF0C25002017
:10D2F00098210020FC24002088240020BD24002048
:10D30000B8290020BC2900209C210020582400209E
:10D310008C240020102900200A2800F0E78009282A
:10D320007FF4F8AD62688F4B9A6138BD0A2800F02F
:10D33000058109287FF4EEADFAF7C6FA62688A49DA
:10D34000884B08601A6038BD0A2800F0ED80092873
:10D350007FF4E0AD2279834B5A7338BD0A2800F080
:10D36000F78009287FF4D6AD62687E4B1A6138BD1C
:10D370000A2800F0D48009287FF4CCAD2279794BBB
:10D380001A7338BD0A2800F0DE8009287FF4C2AD88
:10D390006268744B5A6138BD0A2800F0CA800928B7
:10D3A0007FF4B8AD22796F4B9A7338BD0A2800F02C
:10D3B000D48009287FF4AEAD22796A4BDA7338BD88
:10D3C0000A2800F0898009287FF4A4ADFAF77CFAD6
:10D3D00062686549634B88609A6038BD6349644BF5
:10D3E00051F822205A6089E5624A614B127D5A60E9
:10D3F00084E5604A5E4BD27D003218BF01225A603C
:10D400007CE55D4A5A4B12685A6077E55B4A584B97
:10D4100012685A6072E5574A554B127E5A606DE5A4
:10D42000544A534B12695A6068E5524A504B52783D
:10D430005A6063E54F4A4E4B92785A605EE54D4A1A
:10D440004B4B126A5A6059E54A4A494BD2785A60A6
:10D4500054E5484A464B52795A604FE5484A444B96
:10D460001278003218BF01225A6047E5414A404B0A
:10D4700012785A6042E53F4A3D4BD2695A603DE519
:10D480003C4A3B4B92685A6038E53A4A384B527DE9
:10D490005A6033E5374A364BD2685A602EE5334935
:10D4A0009200114402F21A70BDE838400422FAF7E3
:10D4B00013BE40F2FF70FAF7DDFC2D4B58601DE5FE
:10D4C00001232C482A4A1946C3755360C4E5254AEE
:10D4D000274B52685A6011E5224A254B92685A60E0
:10D4E0000CE5204A224BD2695A6007E51D4A204BC1
:10D4F00092695A6002E51B4A1D4B926A5A60FDE42C
:10D50000184A1B4B526A5A60F8E4164A184B126AC2
:10D510005A60F3E4134A164BD26A5A60EEE4114A99
:10D52000134B127B5A60E9E40E4A114B527B5A604E
:10D53000E4E40C4A0E4B927B5A60DFE4094A0C4B40
:10D5400012685A60DAE4074A094B52695A60D5E416
:10D55000044A074B12695A60D0E4024A044BD27B5A
:10D560005A60CBE48C240020102900200C250020D8
:10D57000FC2400209C210020B8290020BC29002088
:10D580008824002023790649012201F8183F182039
:10D59000BDE83840FAF7A0BDFAF7B0FC237984E57E
:10D5A0009C210020074B9A78022A04D15A685878A7
:10D5B0002AB9FAF70DB80422034B1A707047FAF72C
:10D5C00017B800BF08230020FC24002010B51E4C13
:10D5D000A378012B27D01ED3022B06D004221B4B8D
:10D5E0001A7022780F2A08D010BD6078F9F7DEFF94
:10D5F0002278164B0F2A5860F6D1154A1278002A65
:10D60000F2D0144A5B681360134A93B1136823F095
:10D610000803136010BD6078FF280FD0F9F78CFF66
:10D620000A4B5860DDE76078F9F7F2FF074B586066
:10D63000D7E7136843F00803136010BDFAF710F83A
:10D64000024B5860CDE700BF08230020FC240020D7
:10D6500089240020242400201023002010B41E4B15
:10D660005B789BB901241D491D4B08689B781D4AB6
:10D670001D4902F8013B0C70431E073013F8011FCF
:10D68000834202F8011BF9D110BC7047012B10D066
:10D69000052B17D0062B1AD0072BF5D10A240B2007
:10D6A0000C210D22114BDC71987159711A7110BC4B
:10D6B0007047062464200C210C4AD4715371907178
:10D6C0001171E1E7142412200B211D22EAE7002446
:10D6D00011200E212622E5E7082300200400002067
:10D6E0009C2100202C24002028240020FC24002041
:10D6F000642230B5044D054C28786968431E83B018
:10D7000060702270616003E008230020FC24002088
:10D71000FE2B00F2F381DFE813F00F010E01EC01A4
:10D72000E801DC01DC01DC01DC01D901D901D9010E
:10D73000D901F101D601D301F101F101F101D001CB
:10D74000CD01CA01C701C401C101BE01BB01B801BD
:10D75000B501F101B201AF01AC01A901A601A3011C
:10D76000A0019D019A019701940191018E018B0105
:10D77000880185018201F1017F017C017901760137
:10D78000F101F101F101730170016D01F101F1018C
:10D79000F101F101F101F1010C01F101F101F101DE
:10D7A000F101F101F101F101F101F101F101F101E9
:10D7B000F101F101F101F1016A01F101F101F10160
:10D7C000F101F101F101F101F101F101F101F101C9
:10D7D000F101F101F101F101F101F101F101F101B9
:10D7E000F101F101F101F101F101F101F101F101A9
:10D7F000F101F101F101F101F101F101F101F10199
:10D80000F101F101F101F101F101F101F101F10188
:10D81000F101F101F101F1016701640161015E01B2
:10D8200059014F01460143014C012F01F101F10162
:10D83000350132013801F101F101F1012501F10158
:10D840001B01F101F101F101F101F101F101F1011E
:10D85000F101F101F101F101F101F101F101F10138
:10D86000F101F101F101F101F101F101F101F10128
:10D87000F101F101F101F101F101F101F101F10118
:10D88000F101F101F101F101F101F101F101F10108
:10D89000F101F101F101F101F101F101F101F101F8
:10D8A000F101F101F101F101F101F101F101F101E8
:10D8B000F101F101F101F101F101F101F101F101D8
:10D8C000F101F101F101F101F101F101F101F101C8
:10D8D000F101F101F101F101F101F101F101F101B8
:10D8E000F101F101F101F101F101F101F101F101A8
:10D8F000F101F101F101F101F101F101FF00F1018B
:10D90000F101F101F101F101F101F101F101F10187
:10D91000F101F101F10113012B68824A23F07F43E9
:10D9200023F0FF03934204D17F4B994201D1FDF7CD
:10D930008FFA03B030BD4942A87801F00DF8F8E73E
:10D9400040F2D2439942F4D10122784B5A73F0E766
:10D95000A878C20700F1DD806978400802F0C6FAB5
:10D960006060E6E7A878C30700F1CB800A4640086C
:10D97000697802F0DDFADCE7FBF71AF8D9E7FAF785
:10D9800071FED6E7FBF742F9D3E702AA42F8041D7D
:10D99000A8786978FDF73CFB019B20706360C8E7BD
:10D9A000FBF722F8C5E7624B197D9878FBF7D4F8AE
:10D9B000BFE7FFF753FEBCE7FAF7F4FF0020F9F7E3
:10D9C00061FD0021084600F071FFB2E7584B187D59
:10D9D000FAF7D2FFADE7FAF707FEAAE7FAF7FEFD7E
:10D9E000A7E7FAF7E9FDA4E7FAF736FEA1E7FBF7A8
:10D9F00061FF9EE7FBF74EFF9BE7FBF729FF98E7E8
:10DA0000FBF716FF95E7FBF709FF92E7FBF7FCFE34
:10DA10008FE7FBF7E5FE8CE7FBF7A4FE89E7FBF752
:10DA200095FE86E7FBF702FE83E7FBF761FD80E7E3
:10DA3000FBF7B8FC7DE7FBF7F1FB7AE7FBF748FB68
:10DA400077E7FBF78FFA74E7FAF78EFD71E7FBF7DC
:10DA500051FA6EE7FBF73AFA6BE7FAF733FF68E73C
:10DA6000FAF79EFD65E7FAF76FFD62E7FAF7B6FE93
:10DA70005FE7FBF7DFF95CE7FBF7A6F959E7FBF790
:10DA800089F956E7FBF7F0F853E7FBF71FF950E782
:10DA9000FBF704FA4DE7FBF7E9F94AE7FBF7A4F8CF
:10DAA00047E7FBF73FF844E7FAF7DAFF41E7FAF711
:10DAB000E1FF3EE7FAF738FF3BE7FAF731FE38E7D8
:10DAC000FFF784FD35E7FFF76DFD32E7FFF740F91B
:10DAD0002FE702AB43F8041D6A780146A878FDF7EA
:10DAE00069FB019B2070636023E7A878FDF776FA55
:10DAF0001FE7A878002100F02FFF1AE70223237008
:10DB000017E701380A46C0F34700697802F07AFD4A
:10DB10000FE70138C0F34700697802F051FD6060FB
:10DB200007E700BF00819200D6C5B4A350200020B3
:10DB30009C2100202DE9F04FB14B89B01B7863B1D7
:10DB4000B04B1B78063BDBB2192B00F2B880AE4A13
:10DB500022FA03F3DA0740F1B280AC4CA37B5A1EE1
:10DB6000012A40F26781AA4D04AE032B00F0018127
:10DB7000042B00F07B820023627BA3732B70002AAE
:10DB800040F0A7803046FAF717F80546002840F025
:10DB9000AA800DF10F00FAF79DFC9E4F002840F07F
:10DBA000FA803B785A1E012A40F23782042BA27B6E
:10DBB00000F0D180082A40F21981FFF799FDA37B7C
:10DBC000092B40F0D380F9F77FFE934DDFF8608298
:10DBD0002B68D8F80020C31A83EAE370A0EBE37047
:10DBE000904200F2AC81F9F76FFE6B68D8F8042020
:10DBF000C31A83EAE370A0EBE370904208D9874E22
:10DC00007378012B04BF02237370F9F75DFE68601F
:10DC1000F9F75AFEAB68D8F80820C31A83EAE37014
:10DC2000A0EBE370904208D97C4EB378012B04BF7F
:10DC30000223B370F9F748FEA860002001F04AF80B
:10DC400094F820304BB940B10123744E84F8203051
:10DC5000F378012B04BF0223F370002001F03AF89F
:10DC600008B984F820004FF0270B00254FF0020A76
:10DC7000664EDFF8A8910DE0032B00F06D81012BBB
:10DC800000F067810135082D06F101060BF1010B4B
:10DC900000F07081E8B2F9F74FFC33788342F1D09D
:10DCA0002B1D58F823303070022BE5D10028E9D124
:10DCB00019F80B20012AE5D109F80B30E2E700231F
:10DCC000524C534D627B04AEA3732B70002A3FF479
:10DCD00059AF0120F9F7A4FD3046F9F76DFF05466D
:10DCE00000283FF456AF02F0F1FC464B9DF81A2095
:10DCF0009DF818009A709DF8102018709DF8191062
:10DD00009DF81B709DF81C609DF81D509DF81E002D
:10DD1000072A5970DF719E715D7118710CBF012364
:10DD200002233C4FA3733B789DF811105A1E012A21
:10DD3000E17340F20081052B00F0FD800122384B99
:10DD40001A700DF10F00FAF7C5FB18BB3B78A27BE8
:10DD5000042B7FF42FAF2B4B93F90030002BFFF6F1
:10DD600029AF082A40F25081FAF784FF09B0BDE8D4
:10DD7000F08F2B78002B00F0A080012B7FF4FBAEFE
:10DD8000284F07F1090817F8010FFAF785FB4745F7
:10DD9000F9D1F0E60125FAF7BBFB00287DD1227C02
:10DDA0009DF80F10531CDBB22244092B237411750C
:10DDB00078D12074019002F089FC1B4B227D5B78A6
:10DDC00001989342C2D1194BD91D01E013F8012BE0
:10DDD00010449942C0B2F9D1237F834200F0E2811E
:10DDE00004233A78A3739A42B5D01A4640F25113ED
:10DDF000D340DB077FF5E1AE09B0BDE8F08F00BF8F
:10DE00008824002008230020110200025020002056
:10DE100028240020BD24002010290020C824002030
:10DE2000892400202B2400209C2100206520002034
:10DE30008C240020012B0CBF072708270020BA499B
:10DE4000BA4DCE68E37B2A788DF8107005968DF870
:10DE500012008DF811304ABBB54B89681F785E7887
:10DE6000D8798DF818108DF81F2099795A791B7977
:10DE70008DF819708DF81A608DF81B008DF81C1044
:10DE80008DF81D208DF81E3004AE3046F9F740FEA7
:10DE900000283FF46BAFA37B67E601229DF80F30AB
:10DEA00022742375002D7FF451AF7AE6012A00F029
:10DEB0000C81022AE8D104AE5DE6DFF86C92DFF84F
:10DEC000708299F8020099F8017098F8002098F88B
:10DED00001300744174498F807201F4498F806308B
:10DEE000174498F805201F4498F8043017441F443D
:10DEF000FAF7D2FA99F80100FAF7CEFA98F800008A
:10DF0000FAF7CAFA98F80100FAF7C6FA98F8070083
:10DF1000FAF7C2FA98F80600FAF7BEFA98F8050080
:10DF2000FAF7BAFAFFB298F80400FAF7B5FA3846E9
:10DF3000FAF7B2FA1FE600227E4B1A7001E77E4E16
:10DF40003378012B04BF02233370F9F7BDFC28603E
:10DF500049E600283FF496AE19F80B300135012B45
:10DF600008BF09F80BA0082D06F101060BF1010B03
:10DF70007FF490AE01210020F9F7FEFA237A834264
:10DF800011D098F80C302070DBB2022B00F0B88072
:10DF9000032B02D0012B06D128B1674EF37E012B53
:10DFA00001D10223F37600210846F9F7E5FA237B35
:10DFB000834211D098F80E302070DBB2022B00F0B3
:10DFC000A980032B02D0012B06D128B15A4E337FF2
:10DFD000012B01D102233377584B1B7833B3584DB3
:10DFE0002B781BBB1846544E564902E001332F2BA9
:10DFF0001CD0F25C022AF9D151F82320B2F1FF3F84
:10E0000040F0AC80F054F1E740F25113D340DB070D
:10E010007FF5AAAE09B0BDE8F08F4B4B1868B0F59C
:10E02000006F5DD90023A27B3B70C3E5A17B09296A
:10E030007FF49CAE3B78022B44D0444A1068002801
:10E040003FF494AE012B7FF491AE3F4B404A1C68E5
:10E050001368A34218BF002304D133E052F8041F11
:10E06000A1422FD001338342F8D17FE60023012261
:10E07000DFF8B4902E4F99F8020099F801807B7078
:10E08000804490447B603A70FAF706FA99F80100F0
:10E09000FAF702FA3878FAF7FFF97878FAF7FCF924
:10E0A000F879FAF7F9F9B879FAF7F6F97879FAF729
:10E0B000F3F95FFA88F83879FAF7EEF94046FAF79B
:10E0C000EBF958E505233B7050E6224B06AA03F115
:10E0D000080013F8011B984202F8011BF9D1D3E69E
:10E0E000421C1D491A60F9F7BFFF09210122114B9B
:10E0F000A1731A703B78042B7FF45FADA27B2AE6F4
:10E1000000287FF450AF0C4EF27E012A7FF44BAF13
:10E11000F37648E700287FF45FAF074E327F012A8D
:10E120007FF45AAF337757E79C2100202824002042
:10E13000FC24002089240020C8240020FC22002088
:10E14000BC2400206823002058240020C024002084
:10E150005C2400202D240020082300204FF001081B
:10E160004FF0000E224923480E68A17B224C037712
:10E170002368224C85F8008024680660204D214EDB
:10E180002D680194436034681F4B32601F4A8460DD
:10E19000C56012681D78019C05614461826183F845
:10E1A00000E044E71A4B617DA27DE67D257E197073
:10E1B0005A70A17EE27E607E9E70DD7159711A7187
:10E1C0009871F9F781FB00260321124A3B78124D22
:10E1D00010605A1E012A2E70A17305D9052B03D099
:10E1E00001220E4B1A7085E700220C4B1A7081E752
:10E1F00024240020DC220020082500208424002084
:10E200001023002058240020042300200C29002083
:10E2100008230020F8240020042500208924002061
:10E22000F0B50027254B02794478867890F803E012
:10E23000DA7142791C709A7182790D465A71C179EE
:10E240001F4A204C83B05E70197183F802E094E895
:10E25000030017708DE80300FFF74AFA1A4B6E4669
:10E260001B78B3B1012B05D096E8030084E80300C6
:10E2700003B0F0BD154A6B1E073512F8011B03F8F9
:10E28000011FAB42F9D196E8030084E8030003B014
:10E29000F0BD2B706B7063782278EB70AA70E37915
:10E2A00096E803002B71A3796B716379AB712379C5
:10E2B000EB7184E8030003B0F0BD00BF0823002029
:10E2C00089240020FC240020282400202D24002064
:10E2D000074A0849136823F07F4323F0FF038B426A
:10E2E00000D070475268044B9A42FAD1FCF7B0BD97
:10E2F0000823002000819200D6C5B4A340F2D24387
:10E30000034A52689A4202D10122024B5A73704763
:10E310000823002050200020F8B50024FF23002609
:10E3200000271449144A15480C701460144D1549FF
:10E33000154A046015482C600C601460144D154992
:10E34000154A046015482C600C6014601449154D82
:10E35000154A037015482B700B70C2E9006702F074
:10E3600071F9134B20461C804FF48071BDE8F840D2
:10E37000FBF708BBE4290020C0290020C8290020A1
:10E38000D0290020C4290020D4290020182A0020E8
:10E39000202A0020E8290020F0290020EC29002074
:10E3A000CC290020242A0020D8290020F829002088
:10E3B00074200020014B1868704700BFE02900203E
:10E3C000014B53F8200070471C2A002010B504466A
:10E3D000F9F768F800B110BD2046FBF72BFB0028C9
:10E3E000F9D14FF480712046FBF702FB0028F2D1EF
:10E3F0002046BDE81040F9F745B800BF014B53F87F
:10E4000020007047C0290020014B53F820007047BE
:10E41000C02900206C2110B5104C034601FB0041BF
:10E420000A7E012A11D06C2202FB034292F861108D
:10E4300029B1BDE81040918A184601F02DBE18465A
:10E44000918A01F029FE404210BDCA7D012AEAD01E
:10E45000BDE81040898A01F01FBE00BF2C210020BA
:10E46000FFF7D8BF014B53F820007047C4290020A4
:10E47000014B53F820007047182A0020014B53F835
:10E4800020007047D42900206C2303FB00F0014BCF
:10E49000185870472C210020F8B50C4B994201D92F
:10E4A0000020F8BD6C250B4605FB00F5084E094F12
:10E4B0007219927D00EB800401FB02F247F83430C0
:10E4C0006021735101F034FD0120F8BD400D0300BF
:10E4D0002C21002004210020094B99420ED86C22E7
:10E4E00010B4084C084B02FB004200EB800003EB29
:10E4F000C00041615160012010BC7047002070478E
:10E50000A08601002C21002004210020012901D92E
:10E51000002070476C2210B4074C084B02FB0042ED
:10E5200000EB8000C9B203EBC00080F8241082F831
:10E530003A10012010BC70472C210020042100203B
:10E5400038B50C4B044653F8200003F0E9F86C2270
:10E55000094B054602FB0434606E03F0E1F8014606
:10E56000284603F031F94FF05E5103F02DF903F026
:10E570007BFA38BD202A00202C21002038B50E4B14
:10E5800000EB800203EBC2030446986803F0C8F86E
:10E590006C220A4B054602FB0434606E03F0C0F89F
:10E5A0000146284603F010F94FF05E5103F00CF9D4
:10E5B00003F05AFA38BD00BF042100202C210020AE
:10E5C00038B50C4B044653F8200003F0A9F86C2230
:10E5D000094B054602FB0434606E03F0A1F80146C6
:10E5E000284603F0F1F84FF05E5103F0EDF803F028
:10E5F0003BFA38BDE82900202C21002070B50446E4
:10E600006C26084603F08CF84FF08F4103F0DCF8DD
:10E61000194B054606FB0436706E03F081F801467F
:10E62000284603F085F903F01FFA96F86130054695
:10E63000B27DC3B100FB02F26B21204601F078FCF1
:10E640004FF480412046FBF7AFF90C4B04EB8400FC
:10E650000B490C4A03EBC0039D605D6041F82450F8
:10E6600042F8245070BD434202FB03F26B21204666
:10E6700001F05EFCE4E700BF2C2100200421002013
:10E68000E8290020202A0020B1F5007F10B50446BB
:10E6900034D025DDB1F5806F12D0B1F5006F36D1E1
:10E6A000FBF770F94FF48E412046FBF77DF901230B
:10E6B000184A204613551946BDE8104001F082BCA7
:10E6C000FBF760F920464FF49641FBF76DF9032202
:10E6D000104B20461A550221BDE8104001F072BCD3
:10E6E000B1F5807F14D1FBF74DF94FF49C412046E2
:10E6F000FBF75AF90022074B1A5510BDFBF742F9F8
:10E700004FF49A412046FBF74FF90223D0E710BDA2
:10E7100010BD00BFE429002008B51B4B1878F8F79E
:10E7200077FF1A4B00EB800200EB4210A3FB0023A3
:10E73000C01A03EB5000C00A154BB0F5027F1860F9
:10E7400009D278280CD90420FBF738F9BDE8084035
:10E750000220FBF733B90420BDE80840FBF71CB9E1
:10E760000220FBF719F900210846F8F7A5FE4FF43F
:10E7700080710020FFF788FF0020F8F78BFEBDE8CE
:10E7800008400420FBF71AB9010000200101100025
:10E79000E029002038B5424B1878F8F739FF02F02D
:10E7A0008FFB33A3D3E9002302F000FC32A3D3E9AB
:10E7B000002302F025FD02F0A9FE02F0A3FB0246B1
:10E7C0000B4604460D462AA1D1E9000102F03AFAAF
:10E7D0000022344B02F014FD02460B462046294627
:10E7E00002F00EFD02F092FE02F08CFB00222D4B97
:10E7F00002F006FD03F078FB21A3D3E9002302F029
:10E80000D5FB21A3D3E9002302F01EFA02460B46F2
:10E810001FA1D1E9000102F0F3FC1FA3D3E90023FB
:10E8200002F010FA02F072FE03F01EF91E4B63288C
:10E83000186002DC5A2812DD38BD08210020FBF7E1
:10E84000A1F84FF480710020FFF71EFF0021084659
:10E85000F8F732FEBDE838400020F8F71BBE08216B
:10E86000BDE838400020FBF79FB800BFAFF3008041
:10E870006666666666660A400000000000FEAF40FD
:10E88000C3F5285C8FA272400000000000FEAA4081
:10E890009A999999FD6F2F41C3F5285C8F127140A9
:10E8A00000000020000024401C2A00206C22134B92
:10E8B00002FB0032137E3BB1012B1AD001F56A43F3
:10E8C0000F4A6033934201D90020704770B50B4660
:10E8D000044600260B4A0C4D4FF4006142F82030EC
:10E8E00045F82060FFF7D0FE2046FFF76FFD0120BE
:10E8F00070BDD37D012BE1D0002070472C2100207A
:10E90000C0D40100C8290020D02900206C2370B594
:10E910000D4C03FB00431B7E012B05D901F56A4317
:10E920000A4C6033A34201D9002070BD0B4600267B
:10E93000074D084C4FF4006145F8206044F8203042
:10E94000FFF7A2FE012070BD2C210020C0D40100E1
:10E95000C8290020D02900206C2310B50D4C03FBE2
:10E9600000431B7E33B101F543330B4C03F5A07319
:10E97000A34201D9002010BD0B460446074A4FF4BC
:10E98000007142F82030FFF77FFE2046FFF71EFDA2
:10E99000012010BD2C210020801A0600C42900206F
:10E9A00070B56C24144B04FB0034237E03B970BD96
:10E9B0000546084602F0B4FE4FF08F4102F004FF16
:10E9C0000646606E02F0ACFE0146304602F0B0FF33
:10E9D00003F04AF8094B4FF4804143F825002846DC
:10E9E000FAF7E2FF28464FF48061FFF74DFE284614
:10E9F000BDE87040FFF7EABC2C210020202A00204F
:10EA00000F4B70B5044653F820000D4602F088FE07
:10EA10006C230C4A064603FB0423586E02F080FE6A
:10EA20000146304602F0D0FE4FF05E5102F0CCFEBF
:10EA300003F01AF841192046BDE87040FFF7B0BF57
:10EA4000E82900202C21002010B5044601F038FDF3
:10EA50006C22024B02FB0434A07510BD2C21002057
:10EA60006C2310B4044CCAB203FB00439A751146E0
:10EA700010BC01F02BBD00BF2C2100206C2310B472
:10EA80000C460449224603FB0013DC60998A10BC43
:10EA900001F084BB2C2100206C23024A03FB0020E0
:10EAA000C06870472C210020032901D9002070473D
:10EAB00038B56C25034C05FB0042D17501F0F0FC24
:10EAC000012038BD2C21002010B5044601F0E0FCE7
:10EAD0006C22024B02FB0434E07510BD2C21002097
:10EAE000012901D90020704710B403466C24044A60
:10EAF000012004FB032383F8611010BC704700BFA2
:10EB00002C2100206C23034A03FB002090F86100B5
:10EB1000704700BF2C210020042912D86C2270B548
:10EB2000094C012902FB0042117608D00025074E4E
:10EB30002B462A46642146F8205001F027FA01208E
:10EB400070BD0020704700BF2C210020D02900207C
:10EB50006C23024A03FB0020007E70472C2100201A
:10EB6000022909D810B403466C24044A012004FB8E
:10EB70000323597610BC7047002070472C210020D9
:10EB80006C23024A03FB0020407E70472C210020AA
:10EB9000022909D810B403466C24044A012004FB5E
:10EBA0000323997610BC7047002070472C21002069
:10EBB0006C23024A03FB0020807E70472C2100203A
:10EBC00008B5232101F092F900B208BD08B539213A
:10EBD00001F08CF900B208BD08B52A2101F086F9D0
:10EBE000001408BD6C2370B5194E044603FB006386
:10EBF00093F8355093F83630003518BF01250BB126
:10EC000045F480556C2303FB046393F837300BB154
:10EC100045F480753321204601F068F9020C120496
:10EC20002A432046332101F083F93721204601F0A1
:10EC30005DF96C2303FB0463B3F9382080B240EA2A
:10EC4000024237212046BDE8704001F071B900BF93
:10EC50002C2100206C23054A03FB002090F83B3058
:10EC600023EA010180F83B10704700BF2C210020EF
:10EC70006C23054A03FB002090F83B30194214BF77
:10EC800001200020704700BF2C21002010B56C240B
:10EC9000094B04FB003494F83B30D9070AD5002116
:10ECA000FFF7ACFC94F83B305A0744BF23F0010354
:10ECB00084F83B3010BD00BF2C21002010B5282166
:10ECC000044601F013F900B910BD2046BDE810401C
:10ECD000FFF7DCBF08B5FAF79FFEC0F3803008BD30
:10ECE00038B56C233D4A044603FB00231B7E042BEE
:10ECF00046D8DFE803F01D313B3D03006C2303FBE6
:10ED00000022D57D012D3CD001222046522101F068
:10ED10000FF94FF400612046FAF76AFE002818BF89
:10ED200001212046BDE8384008BF022101F04AB960
:10ED30000022242101F0FCF801222046522101F09A
:10ED4000F7F82046082101F03DF92046BDE838409B
:10ED50000022212101F0ECB85221022201F0E8F852
:10ED60002046BDE83840012101F02CB90522CCE74E
:10ED70006C2303FB0022D37D012B19D00322C4E7AF
:10ED800038BD2B460022522101F000F90023204615
:10ED90001A461C2101F0FAF82A462046512101F0BA
:10EDA000C7F82A462046BDE83840502101F0C0B8D7
:10EDB0000022522101F0EAF8002320461A461C21C5
:10EDC00001F0E4F820460322512101F0B1F8204679
:10EDD000BDE838400322502101F0AAB82C210020C0
:10EDE0006C230B4A03FB00235B7E012B0BD006D365
:10EDF000022B03D10122502101F09AB87047002262
:10EE0000502101F095B80322502101F091B800BFC4
:10EE10002C2100206C230B4A03FB00239B7E012B3B
:10EE20000BD006D3022B03D10122512101F080B86F
:10EE300070470022512101F07BB80322512101F0DB
:10EE400077B800BF2C2100206C22F8B5494D4A4903
:10EE500002FB00520E5C137E04469E42474853D08C
:10EE6000032B57D06C2202FB0452927E012A65D0FC
:10EE70004FF0000E042B24D06C2707FB0457BF7EF5
:10EE8000022F1ED00B550255BEF1000F26D1204691
:10EE9000FFF726FF4FF400412046FAF773FD2046A6
:10EEA000FFF7B8FF6C2303FB0455354E6B7E325DD4
:10EEB0009A4205D02046FFF793FF6B7E3355F8BD8D
:10EEC000F8BD042EDED0065D022EDBD06C260127B5
:10EED00006FB04560B55025586F831700022294B6B
:10EEE0004FF40061204623F81420FAF781FD002832
:10EEF0000CBF02210121204601F064F84FF40041CB
:10EF00002046FAF751FDCAE7927E075D9742C9D0C5
:10EF1000032BA7D1032E19D0025D012A4FF06C02FA
:10EF200002FB04521BD0D77D012F94BF4FF0000E7F
:10EF30004FF0010E82F82AE0927E9BE7032EEBD180
:10EF4000042B03D1065D022EC0D105E06C2202FB2A
:10EF50000452927E022A06D00B55025597E74FF0D5
:10EF6000000E927E86E7065D022EAFD10B55065548
:10EF70008DE700BF2C210020EC290020CC290020A7
:10EF8000242A0020742000202DE9F0470D4609783E
:10EF9000044698469DF82070032903D8DFE801F065
:10EFA0006B34060200232B70BDE8F0871646F8F795
:10EFB00079FA002865D0DFF8A09139F814300133D0
:10EFC0009BB2632B29F8143062D9C72B40F296808C
:10EFD000B3F5967FC0F0AF80B3F5C87FC0F0AE80C8
:10EFE000B3F5FA7FC0F0AD80B3F5167FC0F0AC800A
:10EFF000B3F52F7FC0F0AB80B3F5487F4FF2FF7AB7
:10F0000028BF4FF0000A45E000230122292100F02B
:10F01000BDFF012300225221204600F0B7FF00234C
:10F020001C211A46204600F0B1FF0121204600F0C5
:10F03000C9FF6421204600F059FF642182B22046B6
:10F0400000F076FF6421204600F050FF6C21414B18
:10F05000020C01FB04318B68898A1B0293FBF1F3DC
:10F0600012049BB21A432046642100F061FF022380
:10F070002B70BDE8F0870022374B23F81020BDE845
:10F08000F0870122344B2A7023F81400BDE8F08782
:10F090004FF4804A1C21204600F028FF000C000499
:10F0A00040EA0A021C21204600F042FF39F81430E1
:10F0B000B342FFF479AFB8F1000F2FD1DFF894809D
:10F0C000FFB96C2606FB04860022B18A204600F0B8
:10F0D000B7FF0022B18A204601F03EF84FF40061EC
:10F0E0002046FAF785FC00280CBF022101212046AA
:10F0F00000F068FF03232B70BDE8F0874BF6FF7A22
:10F10000C8E70020FBF72CF9FBF71EF90646FBF7D2
:10F1100027F96C2303FB0483DE62D2E70022272158
:10F12000204600F005FF6C230022DFF8288003FB57
:10F1300004831A85C4E74FF4005AABE74DF6FF7A13
:10F14000A8E74FF4805AA5E74EF6FF7AA2E74FF4FE
:10F15000006A9FE72C21002074200020401A00B292
:10F16000704700BF2DE9F0410D780E46012D044691
:10F1700032D02FD3022D2BD15C4B1B5C9A1E012A5F
:10F1800056D9012B6AD000223921204600F0F0FE2A
:10F19000574F02B2B7F902309A421BD09BB2C01A45
:10F1A00005B205EBD57503EB650301222A21204644
:10F1B0009DB200F0DDFEBB880122C31AEB1A9BB2A0
:10F1C0002046292100F0E2FE00233370BDE8F081E3
:10F1D00000230B70BDE8F081332100F087FE33215E
:10F1E00020F48072204600F0A3FE00232A46292145
:10F1F000204600F0CBFE00223921204600F0B8FE68
:10F200000746DFF8EC802A462A212046A8F802703B
:10F2100000F0AEFE3F1ABFB23B462A4620462921E7
:10F22000A8F8047000F0B2FE02233370BDE8F0814C
:10F230006C23304F03FB007393F86130002B46D0F2
:10F240002D4B53F820206C2303FB0477BB7D6621F4
:10F2500002FB03F2204600F06BFE94E76C23254F7F
:10F2600003FB007393F86130B3B3244B53F8205081
:10F270004FF06C0808FB04786421204600F036FE4D
:10F28000B8F814202B0293FBF2F382B242EA034255
:10F290006421204600F04CFE98F861300BBB184BFF
:10F2A00053F824506D426421204600F01FFE6C2369
:10F2B00003FB0477BA8A2B0293FBF2F3020C9BB296
:10F2C00012041A436421204600F032FE5BE70A4B29
:10F2D00053F820205242B6E7084B53F820506D42B5
:10F2E000C6E7074B53F82450DDE700BFE4290020B0
:10F2F000742000202C210020182A0020C82900207A
:10F30000D02900202DE9F04F6C241E464FF0000E4E
:10F3100004FB00F0144B891A1A18B2F84C701B58F1
:10F3200087FB0145002CC3F1000A75F1000283B090
:10F3300037613160C6F814E04FEAEA7B10DB98468B
:10F340004FEAE379200A52465B46CDE9008940EA5C
:10F350000560291201F032FCB06103B0BDE8F08F06
:10F36000FF3445F10005EAE72C2100202DE9F04F9C
:10F370008BB0F8F7A9FA0746F8F7ACFABD4EB368B8
:10F38000984203D00446FAF7FFFBB460F368FB1A17
:10F39000002BB8BF5B42B3F57A7F80F248813369B6
:10F3A0009F4200F02E8101F0DFF90020FFF74CFDB5
:10F3B0006A21002000F09AFDAF4CA37D94F86120F3
:10F3C00090FBF3F302B95B42227EDFF8D4A2012A5C
:10F3D00008BFAA4B4FF0000008BF1B69DFF8C482CA
:10F3E000CAF8003000F02CFFA37D90FBF3F094F8F6
:10F3F0006130C8F8000013B94042C8F80000692124
:10F40000002000F073FDE27D030C012A00F013815F
:10F4100047F6FF414FF6FE15CA1892B2AA4204D829
:10F42000014489B2A94240F29C8294F8345015F00C
:10F43000010300F0E98094F8331011F0010100F0AD
:10F440003C8100210846F8F797F8031C18BF0123F8
:10F4500094F83450049315F0020540F0DA800395D7
:10F460004FF480610020FAF7C3FA002857D0844B8C
:10F4700094F83A000593002840F029811968D8F8DB
:10F480000020804BFFF73EFFDFF8FC91C9F8000039
:10F49000059BD8F800101B68226C5B1A002BB8BFC4
:10F4A0005B42934208DCDAF80030E26B002BB8BF15
:10F4B0005B42934240F3AB81039B1BB1D9F8003010
:10F4C000002B05DB049B8BB3D9F80030002B2DDD1E
:10F4D00000210846FFF794FA4FF400710020FAF774
:10F4E00087FA50B3DFF8C081DFF89091D8F8003088
:10F4F0004846C9F80C3000F02FFC634AD9F81030A8
:10F500001360039A0AB1002B03DB049AAAB1002B03
:10F5100013DD0023C8F80030C9F810300DE0D8F82A
:10F520000020564B56499A600A6018624FF40071E9
:10F530000020FAF75DFA0028D4D14FF400610020D2
:10F54000FAF756FA70B1DAF800304C4A4E49D360F7
:10F550000B601361039B002B40F02281049B002B66
:10F5600040F02A814FF480710020FAF741FA002818
:10F5700044D1217E012900F05081023902293DD871
:10F580004FF40041FAF734FA002800F023813F4B92
:10F590001B789A1E012A40F29081012B2ED194F8FB
:10F5A0006130002B40F0CB81394B1D686D426421E6
:10F5B000002000F09BFCA28A2B0293FBF2F382B2A4
:10F5C00042EA03426421002000F0B2FC94F861306A
:10F5D000002B40F085812F4B1D686D426421002077
:10F5E00000F084FCA28A2B0293FBF2F3020C1204BB
:10F5F0009BB21A436421002000F09AFCFFF78CF8BC
:10F6000037610BB0BDE8F08F049315F002053FF4AD
:10F6100026AF94F83300012110F0020046D00020FC
:10F62000F7F7AAFF031C18BF0123039318E7FFF79E
:10F63000B1F8F760B3E64FF6FE1103F5F9427F32F9
:10F6400092B28A423FF6F1AEA18A1BB203FB01F1EE
:10F650000029B8BFFF31091294F8613003B949425B
:10F6600008230D4D0D482A680093012300F048FB44
:10F670002860DAE6742000202C21002004210020DC
:10F68000202A0020F8290020182A0020E429002040
:10F69000C8290020D0290020C0290020D829002016
:10F6A000D4290020E8290020C4290020F7F764FFAE
:10F6B000B0FA80F35B090393D2E60846F7F75CFFE4
:10F6C000B0FA80F35B0994F8345004939DE7DFF8B7
:10F6D000CC921B684846C9F8043000F077FBD9F893
:10F6E0000810A74BD8F800200020FFF70BFED8F831
:10F6F0000010D9F808207823521A82EAE271A1EBAF
:10F70000E2718B464FEAE17CCDE908BC93464FEAB3
:10F71000E27C6268CDE906BC82FB03BC099B0BFB63
:10F7200003FE01FB0CE3ABFB011213449C46236870
:10F730008B461D46934A6146106000234FF6FF72C8
:10F74000584602F0B7F985FB0523CDE900230022D6
:10F75000002300F04DFA00F05DFADDE906BCBBF1D4
:10F76000010F7CF100022DDB2268514200F038FAD3
:10F7700080EAE072A2EBE0725142824B814D186840
:10F7800001F00CFA03462268D9F8100051421844DF
:10F790002B6001F003FADFF8F891C9F8000077E672
:10F7A0000020FEF737FE0028BFF6D8AE00237649CA
:10F7B000764A0B601360D5E60020FEF72BFE00288A
:10F7C000F4DCCFE6DDE906120A4340F0A580002113
:10F7D0000A46D2E794F82A303BB1237E032B00F08F
:10F7E0009E80A37E012B00F09A8094F831302BB1DB
:10F7F000237E042B77D0A37E022B74D00020FFF74A
:10F800006FFA4FF400410020FAF7BCF8F6E64FF427
:10F8100080410020FAF7B6F84EE600F0D3FBE37D16
:10F82000012B29D0DFF86891D9F800500DB1A568F7
:10F830002D026421002000F059FBA38A020C95FBE5
:10F84000F3F51204ADB22A436421002000F070FBEE
:10F850006421002000F04AFB642182B2002000F005
:10F8600067FB94F86130D9F8002003B95242212196
:10F87000002000F05DFBC1E694F86130002B58D108
:10F88000414B1D686D426421002000F02FFBA28ACD
:10F890002B0293FBF2F382B242EA0342642100207E
:10F8A00000F046FB6421002000F020FB020C120453
:10F8B0006421002000F03CFBA0E694F86130002BAE
:10F8C0003AD1334B1B685B42A27D662103FB02F2F7
:10F8D000002000F02DFB94F86130002B3FF47BAE4C
:10F8E0002A4B1D687AE694F832305BB3012B7FF423
:10F8F00085AEA08DFAF734FD4FF400610020FAF7D1
:10F9000077F800280CBF02210121002000F05AFBEB
:10F91000002384F8313071E62268404225E7207FD9
:10F92000C0B102287FF46AAE1A490020FFF71AFC22
:10F9300064E6154B1D68A6E7154B1B68C4E7124B20
:10F940001D6834E60121E28B184600911249FFF749
:10F950001BFB53E6E28B012300900E49FFF714FBDB
:10F960004CE64FF4807201B21BB20B44A18A01FB3A
:10F9700003F1237E91FBF2F1012B7FF46DAE6FE674
:10F98000F8290020F0290020C8290020D0290020D3
:10F99000182A0020562100205D210020042100208B
:10F9A00010B5044600F0A2FD6C22024B02FB0434A9
:10F9B000208210BD2C210020B1F5803F01D3002012
:10F9C000704738B56C25054C8BB205FB00421946D3
:10F9D000138200F091FD012038BD00BF2C210020D2
:10F9E00010B5044600F098FD6C22024B02FB043473
:10F9F000608210BD2C210020B1F5803F01D3002092
:10FA0000704738B56C25054C8BB205FB0042194692
:10FA1000538200F087FD012038BD00BF2C2100205B
:10FA2000F8B56C231A4E044603FB006393F8545058
:10FA300035B3184F3B5C43B36C2505FB046595F863
:10FA4000551095F856600031204618BF012176B157
:10FA5000F7F792FC95F857102046F7F783FC022140
:10FA6000B5F85A200C4B395523F81420F8BDF7F798
:10FA700083FC31462046F7F775FC01233B55F8BD62
:10FA8000F7F786FC034B1D55F8BDF7F70DFCD3E7E0
:10FA90002C2100202C2A0020282A00200021024AA4
:10FAA0001154FFF7BDBF00BF2C2A00200C4A125C86
:10FAB000022A06D10B4931F810201AB1013A21F877
:10FAC0001020704730B46C240325074A21F81050E9
:10FAD00004FB002330BC93F85810F7F743BC00BF79
:10FAE0002C2A0020282A00202C21002038B5F7F7E6
:10FAF000EBFE0546FAF7DAFB40B90E4C23689D424F
:10FB000002D00020FFF7D2FF256038BDFAF704FCD1
:10FB10000028F2D04FF400410020F9F769FF0028D7
:10FB2000EBD0FAF711FC002203461C21104600F02E
:10FB30002DFAE2E79020002070B56C241C4B04FBEA
:10FB4000003494F85C3033B9BDE870404FF0FF32B8
:10FB5000752100F0EDB90546B4F85E20154EC2EBF4
:10FB6000023286FB0231D3170A44C3EBE213A3F53A
:10FB7000DE43143B9BB20122752100F007FA94F892
:10FB80006020B4F85E3028469B1AC3EB033386FB33
:10FB90000326DA173344C2EBE313A3F5DE43143B29
:10FBA0009BB20022BDE87040752100F0EFB900BFA4
:10FBB0002C210020C12787CB10B50024044B204600
:10FBC0001C70FFF72DFF2046BDE81040FFF7B4BFC3
:10FBD0002C2A0020FFF7B0BF704700BF00207047FD
:10FBE000904203DC8842B8BF084670471046704711
:10FBF00030B5DDE90345844275EB010E07DB904229
:10FC000071EB030400DB30BD1046194630BD2046C1
:10FC1000294630BD021E37DBFF2A1FDDB2F5803FCB
:10FC200036490CDBB2F1807F1CDBB2F1805F3ADB3E
:10FC3000B2F1804F5ADB1316CB5C1B0239E0B2F5F0
:10FC4000805F19DBB2F5804F3EDB1312C85C0130D8
:10FC500000FB00F39A4219DA01387047274B985C91
:10FC600000097047B2F5801F11DBB2F5800F41DB50
:10FC70001314CB5C1B0110E0B2F5806F29DB13116C
:10FC8000C85C8308581CE3E74FF0FF307047B2F5BB
:10FC9000802F27DA9312CB5C5B0092FBF3F00133E9
:10FCA00003445810D4E7B2F1806F17DA9314CB5C99
:10FCB0005B0192FBF3F101330B445B1092FBF3F019
:10FCC000013303445810C3E79311C85C4008013066
:10FCD000BEE79310CB5CDB08581CB9E71315CB5C6F
:10FCE0009B01E6E71313CB5C9B00D6E79315CB5C37
:10FCF000DB01DEE79313CB5CDB00CEE708240108D1
:10FD0000D0B4D0E900679DF80C40891AE31A9940F5
:10FD1000761847EBE177C4F1200226FA04F307FADC
:10FD200002F2203C43EA02035CBF47FA04F4234397
:10FD3000C0E90067D0BC1846704700BF00234FF6EB
:10FD4000FF72036002834360C36003614361C36168
:10FD5000036280F824307047F8B590F824300446E8
:10FD600033B36369184EC56886FB03760069D917FB
:10FD70002A1A002AB8BF5242C1EBA6118A42B8BF64
:10FD80004FF47A734FF47A71B8BF5343E6690E4A61
:10FD9000334482FB0362DE179211971B01FB17337A
:10FDA0008542E3610CDC05DAB21A1044206101E0FF
:10FDB000C068206122685142FFF712FF2061F8BD40
:10FDC00038442061F6E700BFD34D621090F824302C
:10FDD00013B9436883607047F0B50446836845688B
:10FDE0007820ED1A636985EAE57283FB0001A2EBD6
:10FDF000E572D71700FB07F3266802FB0133A0FB6F
:10FE00000201A6FB066783B0228B1944002301F090
:10FE100051FE00220023CDE90067FFF7E9FEFFF75E
:10FE2000F9FE002D52DD22680021FFF7D9FE0546BC
:10FE300063692D4E216986FB03766A1AD817002A5A
:10FE4000B8BF5242C0EBA6108242B8BF4FF47A73DB
:10FE50004FF47A70B8BF5343E669234A334482FBB8
:10FE60000362DE179211971B00FB17338D42E3618B
:10FE700035DD39442161208B3C22002380FB0101C8
:10FE800001F018FE4FF47A72236A174EC01841EB46
:10FE9000E371A368C2FB030180EAE075A5EBE0759E
:10FEA00086FB0576002871F100034FEAE573C3EB8A
:10FEB000A61302FB1353B8BF5B4223624FF47A725E
:10FEC000002301F0F7FDA06003B0F0BDB0D02168C1
:10FED000404249420022FFF783FE0546A8E7CADAFE
:10FEE000B21A11442161C6E7D34D621038B501F052
:10FEF0007F0100220546FAF7DBFF00222846114663
:10FF0000FAF7D6FF0022040211462846FAF7D0FF7E
:10FF10000022044311462846FAF7CAFF24020122B0
:10FF2000044300212846FAF7C3FF2402204338BDCA
:10FF300038B51546044641F080010022FAF7B8FFB3
:10FF4000290E20460022FAF7B3FFC5F307412046E9
:10FF50000022FAF7ADFFC5F3072120460022FAF789
:10FF6000A7FFE9B22046BDE838400122FAF7A0BF5A
:10FF700010B51446FFF7BAFF2CB1012C01D1000CCB
:10FF800010BD002010BD80B210BD00BFF8B51446F2
:10FF90001F4605460E46FFF7A9FF54B1012C01D1BB
:10FFA00067F31F40024631462846BDE8F840FFF798
:10FFB000BFBF67F30F00024631462846BDE8F84050
:10FFC000FFF7B6BF38B50D4663210446FFF78EFF35
:10FFD00020F0FF0045EA000263212046BDE83840DA
:10FFE000FFF7A6BF70B50D4604460121FFF7EAFFF3
:10FFF000ABB22046BDE8704001226421FFF7C6BFC6
:020000040801F1
:1000000070B56F210446FFF771FF002206466F218D
:100010002046FFF78DFF20466E21FFF767FF05465C
:10002000324620466F21FFF783FF284670BD00BF90
:1000300008B56921FFF75AFF001408BD002070477A
:1000400070B514460E46240201210546FFF7BAFF9B
:1000500094FBF6F32846BDE870409BB20122642170
:10006000FFF794BF10B50C46FFF7CAFF00FB04F082
:100070000028B8BFFF30001210BD00BF10B50C46FD
:100080006921FFF733FF001404FB00F00028B8BF1C
:10009000FF30001210BD00BF2DE9F0410D466F2169
:1000A0000446FFF723FF002280466F212046FFF71A
:1000B0003FFF20466E21FFF719FF012206466F2100
:1000C0002046FFF735FF20466E21FFF70FFF07465A
:1000D000424620466F21FFF72BFFF01905FB00F089
:1000E0000028B8BFFF300012BDE8F08110B50C4603
:1000F0006921FFF7FBFE03B203EB204004FB00F095
:100100000028B8BFFF30001210BD00BF00207047AC
:100110008BB200226421FFF739BF00BF70B56F2199
:100120000446FFF7E3FE012206466F212046FFF753
:10013000FFFE20466E21FFF7D9FE054632462046D7
:100140006F21FFF7F5FE284670BD00BF08B5692195
:10015000FFF7CCFE00B208BD130293FBF1F30022BF
:100160009BB26421FFF712BF10B50C46FFF7D6FF14
:1001700000FB04F00028B8BFFF30001210BD00BF24
:1001800010B50C466921FFF7B1FE00B200FB04F088
:100190000028B8BFFF30001210BD00BF130293FB50
:1001A000F1F300229BB25E21FFF7F0BE10B50C46C2
:1001B0005E21FFF79BFE80B204FB00F0001210BD31
:1001C00038B504460D460221FFF7FCFE2A462046BC
:1001D000BDE838406621FFF7ABBE00BF6621FFF7E0
:1001E00085BE00BF6A21FFF781BE00BF00207047B7
:1001F00038B504460D460321FFF7E4FE2A462046A3
:10020000BDE838406821FFF793BE00BF38B504460B
:100210000D460321FFF7D6FE20466B21FFF766FE51
:10022000682142192046BDE83840FFF781BE00BF73
:100230006821FFF75BBE00BF0A466B21FFF778BE5F
:100240006B21FFF753BE00BF00207047F8B50D4685
:1002500009780446BDF81860032903D8DFE801F0E7
:100260005625050200232B70F8BD1988013189B28B
:1002700091421980F8D3274E002227212046FFF70C
:1002800057FE726824212046FFF752FE3389002270
:100290001C212046FFF77AFE338820460022522197
:1002A000FFF774FE03232B70F8BD52212046FFF7A1
:1002B0001DFE184F242138802046FFF717FE1C2111
:1002C00078602046FFF712FE0023388101222921A1
:1002D0002046FFF75BFE0123002252212046FFF754
:1002E00055FE0023012224212046FFF74FFE33460E
:1002F000002224212046FFF749FE002320461A460B
:100300001C21FFF743FE02232B70F8BD00221A8048
:10031000F8BD00BF94200020401A00B2704700BF13
:100320002DE9F0410C780D46012C06462DD028D33E
:10033000022C03D000230B70BDE8F0813921FFF7B8
:10034000D5FD274F02B2B7F90A309A42F4D09BB2DA
:10035000C01A04B204EBD47403EB64032A213046C0
:100360009CB2FFF7C3FDBB890122C3EB1043E31A24
:100370009BB230462921FFF709FE00232B70BDE810
:10038000F08100231380BDE8F0813321FFF7AEFD3B
:10039000332120F480723046FFF7CAFD0023224645
:1003A00029213046FFF7F2FD39213046FFF79EFD47
:1003B0000746DFF82C802A213046A8F80A70FFF79C
:1003C00095FDA7EB1047BFB23B4622463046292198
:1003D000A8F80C70FFF7DAFD02232B70BDE8F0815E
:1003E000942000202DE9F0430E46114D83B0296979
:1003F0001446B1421F468146BDF82820DDF82C8006
:10040000BDF8303001D02CB12E61022C08D003B0E1
:10041000BDE8F083009339464346FFF717FFF3E743
:1004200042463946484603B0BDE8F043FFF778BF7F
:100430009420002070B4BDF80C60BDF81440039601
:10044000059470BCFFF7CEBF137813B910B1022822
:1004500000D07047012308701370704791420BD091
:1004600038B5144652211D46FFF762FD032C02D118
:10047000049B1B780BB138BD704715F0FD0FFAD106
:100480000123049A1370F6E700221A21FFF750BDEA
:1004900008B51B21FFF72AFDC0F3074008BD00BFC8
:1004A00038B50D461B210446FFF720FD20F47F00E0
:1004B00040EA05421B212046BDE83840FFF738BD21
:1004C00008B51B21FFF712FDC0B208BD38B50D46B7
:1004D0001B210446FFF70AFD000C000440EA050258
:1004E0001B212046BDE83840FFF722BD08B5092191
:1004F000FFF7FCFC80B208BD38B50D460921044663
:10050000FFF7F4FC000C000440EA05020921204634
:10051000BDE83840FFF70CBD08B50821FFF7E6FC41
:1005200080B208BD38B50D4608210446FFF7DEFC51
:10053000000C000440EA050208212046BDE83840CE
:10054000FFF7F6BC38B5054642EA0144224654217D
:10055000FFF7EEFC22462846BDE838405621FFF75B
:10056000E7BC00BF42EA01425821FFF7E1BC00BFEF
:1005700042EA01425A21FFF7DBBC00BF2DE9F047F8
:10058000894611469A4616460546089C9DF82480E1
:10059000FFF7ACFC5246074631462846FFF7C8FC39
:1005A00049462846FFF7A2FC044024FA08F42846EE
:1005B0003A463146FFF7BCFC2046BDE8F08700BF55
:1005C00038B501F07F0100220546FAF773FC0022DE
:1005D00028461146FAF76EFC00220402114628460E
:1005E000FAF768FC0022044311462846FAF762FC39
:1005F00024020122044300212846FAF75BFC24026E
:10060000204338BD38B51546044641F0800100222C
:10061000FAF750FC290E20460022FAF74BFCC5F3EE
:10062000074120460022FAF745FCC5F30721204682
:100630000022FAF73FFCE9B22046BDE8384001222B
:10064000FAF738BC30B40023002400250360C0E969
:10065000024530BC83617047114B1A68821A002A28
:10066000B8BF5242B2F57A7F18DB0022F0B49F681F
:10067000996A1860186B1E699D691C6A5F609F6BA0
:100680009A601A619A611A629A6259621A63D86210
:100690009A63DE605D61DC615F63F0BC704700BF40
:1006A000A8200020024A936801339360704700BF7E
:1006B000A8200020014B9868704700BFA8200020A8
:1006C000014B5868704700BFA8200020024A1369F8
:1006D00001331361704700BFA8200020014BD86888
:1006E000704700BFA8200020024A9369013393613C
:1006F000704700BFA8200020014B5869704700BF19
:10070000A8200020024A136A01331362704700BF19
:10071000A8200020014BD869704700BFA820002006
:10072000024A936A01339362704700BFA8200020F9
:10073000014B586A704700BFA8200020024A136B83
:1007400001331363704700BFA8200020014BD86A13
:10075000704700BFA8200020024B186B00EB800000
:1007600040007047A8200020024A936B0133936336
:10077000704700BFA8200020014B586B704700BF96
:10078000A8200020024B986B00EB800040007047CF
:10079000A8200020014B1860704700BF542A002099
:1007A000014B1868704700BF542A0020014B1860A5
:1007B000704700BF4C2A0020014B1868704700BFEB
:1007C0004C2A0020014B1860704700BF482A0020C7
:1007D000014B1868704700BF482A0020014B186081
:1007E000704700BF402A0020014B1868704700BFC7
:1007F000402A0020014B1860704700BF502A00209B
:10080000014B1868704700BF502A0020014B186048
:10081000704700BF342A0020014B1868704700BFA2
:10082000342A0020014B1860704700BF3C2A00208A
:10083000014B1868704700BF3C2A0020014B18602C
:10084000704700BF382A0020014B1868704700BF6E
:10085000382A0020014B1860704700BF442A00204E
:10086000014B1868704700BF442A0020014B1860F4
:10087000704700BF302A0020014B1868704700BF46
:10088000302A002010B400220124044B18705C723E
:100890001A725960DA6010BC704700BFEC2000206B
:1008A0000022024B5A721A72DA607047EC20002064
:1008B000014B187A704700BFEC200020014B587A9A
:1008C000704700BFEC200020014BD868704700BF84
:1008D000EC2000200021064B0068DA681961013223
:1008E0008242DA6002D159721972D960704700BF32
:1008F000EC20002084B0F0B4144D154E2C693768FC
:10090000013405AEBC422C6186E80E0016DB2B7A62
:10091000A3B10168EB68994210DD00274268059E8B
:100920001801165001330244069C079E089899420C
:10093000EB6054609660D0602F6102D0F0BC04B0D0
:1009400070476F722F72EF60F8E700BFEC20002055
:10095000180000200068704700680001704700BF61
:100960000420704710B404688C420DDD032A02DDB8
:10097000022010BC70474468002004EB011151F8BC
:10098000222010BC1A607047012010BC704700BFC5
:100990000A2807D8DFE800F00611150A0E0E060631
:1009A00006060E000022094B5A6170470322074BCE
:1009B0005A617047054B586170470122034B5A61D9
:1009C00070470222014B5A61704700BFEC200020A3
:1009D000014B5869704700BFEC200020014B1860A4
:1009E000704700BF18000020014B1868704700BF17
:1009F0001800002010B5144B1C78062C08D8DFE82E
:100A000004F00713171B1F0C04005A68904207DDFF
:100A100001221A7200225A7210BD5A688242F7DC13
:100A20001A7A002AF6D110BD59689142F8DDEFE735
:100A300059688A42ECDCF3E75A688A42E8DCEFE75F
:100A40005A689142E4DCEBE7EC200020B0F5803FEF
:100A50001CDBB0F1807F31DBB0F1805F39DAB0F1BF
:100A6000806F394A4DDB0315D35C9B0190FBF3F299
:100A7000013313445B1090FBF3F2013313445B101A
:100A800003FB03F2904217DA581E7047FF2805DC7B
:100A9000002856DB2C4B185C00097047B0F5805FCE
:100AA000294A26DBB0F5804F2FDB0312D35C0133DC
:100AB00003FB03F29042E7DB18467047B0F5801F56
:100AC000214A0FDBB0F5800F32DB0314D35C1B012E
:100AD000D1E7B0F1804F22DB1C4B98422CDD4FF662
:100AE000FF707047B0F5802F1EDB0313D35C9B00B3
:100AF000C1E7B0F5806F0DDB0311D35C9B080133B8
:100B0000D6E78314D35C5B01B0E78311D35C5B0849
:100B10000133CDE78310D35CDB080133C8E70A4A11
:100B20008315D35CDB01A1E78312D35C5B00A2E7F2
:100B30008313D35CDB009EE7034A0316D35C1B02DE
:100B400094E74FF0FF307047082501080080FE7FD2
:100B5000B0F5806F14D2B0F5007F08D2FF2895BFA2
:100B60000A4B0B4BC018181A90F800017047B0F5EB
:100B7000407F07D3074B181A90F800014042704796
:100B800000207047044BC05C4042704708250108B4
:100B9000072701080729010808240108904203DCFF
:100BA0008842B8BF0846704710467047904203D845
:100BB000884238BF084670471046704730B5DDE9B7
:100BC0000345844275EB010E07DB904271EB030491
:100BD00000DB30BD1046194630BD2046294630BDE9
:100BE00070B514460E4600F09BFD0546204600F009
:100BF00093FD04460146284600F09AFE0146284629
:100C000000F0D8FC0546304600F08AFD214600F091
:100C10008FFE0146284600F0CFFC00F025FF70BD96
:100C200010B4019C891AE31A026801FA03F3134411
:100C3000036043FA04F010BC704700BF81F000412C
:100C400002E000BF83F0004330B54FEA41044FEAB1
:100C5000430594EA050F08BF90EA020F1FBF54EA4C
:100C6000000C55EA020C7FEA645C7FEA655C00F0E8
:100C7000E2804FEA5454D4EB5555B8BF6D420CDDB9
:100C80002C4480EA020281EA030382EA000083EA3C
:100C9000010180EA020281EA0303362D88BF30BDDC
:100CA00011F0004F4FEA01314FF4801C4CEA113132
:100CB00002D0404261EB410113F0004F4FEA033391
:100CC0004CEA133302D0524263EB430394EA050F1C
:100CD00000F0A780A4F10104D5F1200E0DDB02FA8B
:100CE0000EFC22FA05F2801841F1000103FA0EF21F
:100CF000801843FA05F359410EE0A5F120050EF1E5
:100D0000200E012A03FA0EFC28BF4CF0020C43FA15
:100D100005F3C01851EBE37101F0004507D54FF022
:100D2000000EDCF1000C7EEB00006EEB0101B1F572
:100D3000801F1BD3B1F5001F0CD349085FEA3000B8
:100D40004FEA3C0C04F101044FEA445212F5800FC3
:100D500080F09A80BCF1004F08BF5FEA500C50F160
:100D6000000041EB045141EA050130BD5FEA4C0C43
:100D7000404141EB010111F4801FA4F10104E9D1CC
:100D800091F0000F04BF01460020B1FA81F308BFC3
:100D90002033A3F10B03B3F120020CDA0C3208DD8F
:100DA00002F1140CC2F10C0201FA0CF021FA02F16A
:100DB0000CE002F11402D8BFC2F1200C01FA02F1DA
:100DC00020FA0CFCDCBF41EA0C019040E41AA2BFFF
:100DD00001EB0451294330BD6FEA04041F3C1CDAC7
:100DE0000C340EDC04F11404C4F1200220FA04F0E7
:100DF00001FA02F340EA030021FA04F345EA030191
:100E000030BDC4F10C04C4F1200220FA02F001FA52
:100E100004F340EA0300294630BD21FA04F02946D4
:100E200030BD94F0000F83F4801306BF81F480116D
:100E30000134013D4EE77FEA645C18BF7FEA655CE0
:100E400029D094EA050F08BF90EA020F05D054EAB2
:100E5000000C04BF1946104630BD91EA030F1EBFB7
:100E60000021002030BD5FEA545C05D140004941BB
:100E700028BF41F0004130BD14F580043CBF01F5AE
:100E8000801130BD01F0004545F0FE4141F4700194
:100E90004FF0000030BD7FEA645C1ABF194610466F
:100EA0007FEA655C1CBF0B46024650EA013406BF70
:100EB00052EA033591EA030F41F4002130BD00BF2F
:100EC00090F0000F04BF0021704730B54FF48064EC
:100ED00004F132044FF000054FF0000150E700BF6D
:100EE00090F0000F04BF0021704730B54FF48064CC
:100EF00004F1320410F0004548BF40424FF00001B9
:100F00003EE700BF42004FEAE2014FEA31014FEAFB
:100F100002701FBF12F07F4393F07F4F81F060514A
:100F2000704792F0000F14BF93F07F4F704730B5B9
:100F30004FF4607401F0004521F0004120E700BF4C
:100F400050EA010208BF704730B54FF000050AE0D3
:100F500050EA010208BF704730B511F0004502D5D4
:100F6000404261EB41014FF4806404F132045FEAD6
:100F7000915C3FF4DCAE4FF003025FEADC0C18BF7B
:100F800003325FEADC0C18BF033202EBDC02C2F171
:100F9000200300FA03FC20FA02F001FA03FE40EA03
:100FA0000E0021FA02F11444C1E600BF70B54FF003
:100FB000FF0C4CF4E06C1CEA11541DBF1CEA1355E5
:100FC00094EA0C0F95EA0C0F00F0DEF82C4481EA4D
:100FD000030621EA4C5123EA4C5350EA013518BF6D
:100FE00052EA033541F4801143F4801338D0A0FB5A
:100FF00002CE4FF00005E1FB02E506F00042E0FB07
:1010000003E54FF00006E1FB03569CF0000F18BF0C
:101010004EF0010EA4F1FF04B6F5007F64F54074B4
:1010200004D25FEA4E0E6D4146EB060642EAC62147
:1010300041EA55514FEAC52040EA5E504FEACE2EB4
:10104000B4F1FD0C88BFBCF5E06F1ED8BEF1004FB7
:1010500008BF5FEA500E50F1000041EB045170BD33
:1010600006F0004646EA010140EA020081EA030177
:10107000B4EB5C04C2BFD4EB0C0541EA045170BD73
:1010800041F480114FF0000E013C00F3AB8014F1ED
:10109000360FDEBF002001F0004170BDC4F1000436
:1010A000203C35DA0C341BDC04F11404C4F12005B7
:1010B00000FA05F320FA04F001FA05F240EA020012
:1010C00001F0004221F0004110EBD37021FA04F648
:1010D00042EB06015EEA430E08BF20EAD37070BD02
:1010E000C4F10C04C4F1200500FA04F320FA05F061
:1010F00001FA04F240EA020001F0004110EBD37063
:1011000041F100015EEA430E08BF20EAD37070BDD2
:10111000C4F1200500FA05F24EEA020E20FA04F3AB
:1011200001FA05F243EA020321FA04F001F000415A
:1011300021FA04F220EA020000EBD3705EEA430ECB
:1011400008BF20EAD37070BD94F0000F0FD101F0FA
:101150000046400041EB010111F4801F08BF013C33
:10116000F7D041EA060195F0000F18BF704703F071
:101170000046520043EB030313F4801F08BF013DF8
:10118000F7D043EA0603704794EA0C0F0CEA1355B4
:1011900018BF95EA0C0F0CD050EA410618BF52EA6E
:1011A0004306D1D181EA030101F000414FF0000074
:1011B00070BD50EA410606BF1046194652EA430682
:1011C00019D094EA0C0F02D150EA013613D195EAF6
:1011D0000C0F05D152EA03361CBF104619460AD13E
:1011E00081EA030101F0004141F0FE4141F4700148
:1011F0004FF0000070BD41F0FE4141F4780170BD38
:1012000070B54FF0FF0C4CF4E06C1CEA11541DBF9C
:101210001CEA135594EA0C0F95EA0C0F00F0A7F89E
:10122000A4EB050481EA030E52EA03354FEA0131CB
:1012300000F088804FEA03334FF0805545EA1313DE
:1012400043EA12634FEA022245EA111545EA1065A6
:101250004FEA00260EF000419D4208BF964244F13D
:10126000FD0404F5407402D25B084FEA3202B61A5C
:1012700065EB03055B084FEA32024FF480104FF430
:10128000002CB6EB020E75EB030E22BFB61A7546A4
:1012900040EA0C005B084FEA3202B6EB020E75EB37
:1012A000030E22BFB61A754640EA5C005B084FEA9F
:1012B0003202B6EB020E75EB030E22BFB61A75466C
:1012C00040EA9C005B084FEA3202B6EB020E75EB77
:1012D000030E22BFB61A754640EADC0055EA060E38
:1012E00018D04FEA051545EA16754FEA06164FEA7B
:1012F000C30343EA52734FEAC2025FEA1C1CC0D127
:1013000011F4801F0BD141EA00014FF000004FF0B3
:10131000004CB6E711F4801F04BF01430020B4F174
:10132000FD0C88BFBCF5E06F3FF6AFAEB5EB030C2C
:1013300004BFB6EB020C5FEA500C50F1000041EB29
:10134000045170BD0EF0004E4EEA113114EB5C04F6
:10135000C2BFD4EB0C0541EA045170BD41F48011C9
:101360004FF0000E013C90E645EA060E8DE60CEAD1
:10137000135594EA0C0F08BF95EA0C0F3FF43BAFEE
:1013800094EA0C0F0AD150EA01347FF434AF95EAA5
:101390000C0F7FF425AF104619462CE795EA0C0F89
:1013A00006D152EA03353FF4FDAE1046194622E756
:1013B00050EA410618BF52EA43067FF4C5AE50EA30
:1013C00041047FF40DAF52EA43057FF4EBAE12E720
:1013D0004FF0FF3C06E000BF4FF0010C02E000BF01
:1013E0004FF0010C4DF804CD4FEA410C7FEA6C5CE4
:1013F0004FEA430C18BF7FEA6C5C1BD001B050EA87
:10140000410C0CBF52EA430C91EA030F02BF90EA71
:10141000020F0020704710F1000F91EA030F58BF30
:10142000994208BF90422CBFD8176FEAE37040F092
:10143000010070474FEA410C7FEA6C5C02D150EA30
:10144000013C07D14FEA430C7FEA6C5CD6D152EAEB
:10145000033CD3D05DF8040B704700BF84461046B0
:1014600062468C461946634600E000BF01B5FFF7AF
:10147000B7FF002848BF10F1000F01BD4DF808ED7F
:10148000FFF7F4FF0CBF012000205DF808FB00BF50
:101490004DF808EDFFF7EAFF34BF012000205DF8AA
:1014A00008FB00BF4DF808EDFFF7E0FF94BF0120F7
:1014B00000205DF808FB00BF4DF808EDFFF7CEFFF8
:1014C00094BF012000205DF808FB00BF4DF808ED37
:1014D000FFF7C4FF34BF012000205DF808FB00BF08
:1014E0004FEA410C7FEA6C5C02D150EA013C0AD120
:1014F0004FEA430C7FEA6C5C02D152EA033C02D112
:101500004FF0000070474FF0010070474FEA410272
:10151000B2F1E04324BFB3F5001CDCF1FE5C0DD951
:1015200001F0004C4FEAC0024CEA5070B2F1004F9B
:1015300040EB830008BF20F00100704711F0804F9E
:1015400021D113F13872BCBF01F00040704741F463
:1015500080114FEA5252C2F11802C2F1200C10FA67
:101560000CF320FA02F018BF40F001004FEAC1234B
:101570004FEAD32303FA0CFC40EA0C0023FA02F3EF
:101580004FEA4303CCE77FEA625307D150EA0133C5
:101590001EBF4FF0FE4040F44000704701F0004095
:1015A00040F0FE4040F40000704700BF80F0004073
:1015B00002E000BF81F0004142001FBF5FEA41032B
:1015C00092EA030F7FEA226C7FEA236C6AD04FEA2B
:1015D0001262D2EB1363C1BFD21841404840414070
:1015E000B8BF5B42192B88BF704710F0004F40F422
:1015F000000020F07F4018BF404211F0004F41F43E
:10160000000121F07F4118BF494292EA030F3FD009
:10161000A2F1010241FA03FC10EB0C00C3F120031C
:1016200001FA03F100F0004302D5494260EB4000AB
:10163000B0F5000F13D3B0F1807F06D340084FEA16
:10164000310102F10102FE2A51D2B1F1004F40EB0B
:10165000C25008BF20F0010040EA03007047490073
:1016600040EB000010F4000FA2F10102EDD1B0FA3E
:1016700080FCACF1080CB2EB0C0200FA0CF0AABF33
:1016800000EBC25052421843BCBFD04018437047D1
:1016900092F0000F81F4000106BF80F400000132D7
:1016A000013BB5E74FEA41037FEA226C18BF7FEAAE
:1016B000236C21D092EA030F04D092F0000F08BFF0
:1016C0000846704790EA010F1CBF0020704712F0D7
:1016D0007F4F04D1400028BF40F00040704712F116
:1016E00000723CBF00F50000704700F0004343F07B
:1016F000FE4040F4000070477FEA226216BF0846B1
:101700007FEA23630146420206BF5FEA412390EA73
:10171000010F40F4800070474FF0000304E000BF69
:1017200010F0004348BF40425FEA000C08BF70471A
:1017300043F0964301464FF000001CE050EA0102DE
:1017400008BF70474FF000030AE000BF50EA0102F3
:1017500008BF704711F0004302D5404261EB4101E0
:101760005FEA010C02BF84460146002043F0B64305
:1017700008BFA3F18053A3F50003BCFA8CF2083A2A
:10178000A3EBC25310DB01FA02FC634400FA02FC33
:10179000C2F12002BCF1004F20FA02F243EB02003A
:1017A00008BF20F00100704702F1200201FA02FC9C
:1017B000C2F1200250EA4C0021FA02F243EB02008F
:1017C00008BF20EADC7070474FF0FF0C1CEAD052D3
:1017D0001EBF1CEAD15392EA0C0F93EA0C0F6FD094
:1017E0001A4480EA010C400218BF5FEA41211ED072
:1017F0004FF0006343EA501043EA5111A0FB01315E
:101800000CF00040B1F5000F3EBF490041EAD37132
:101810005B0040EA010062F17F02FD2A1DD8B3F1AE
:10182000004F40EBC25008BF20F00100704790F01D
:10183000000F0CF0004C08BF49024CEA502040EA6F
:1018400051207F3AC2BFD2F1FF0340EAC250704735
:1018500040F400004FF00003013A5DDC12F1190F73
:10186000DCBF00F000407047C2F10002410021FAE5
:1018700002F1C2F1200200FA02FC5FEA310040F1FD
:10188000000053EA4C0308BF20EADC70704792F076
:10189000000F00F0004C02BF400010F4000F013AAE
:1018A000F9D040EA0C0093F0000F01F0004C02BFA9
:1018B000490011F4000F013BF9D041EA0C018FE718
:1018C0000CEAD15392EA0C0F18BF93EA0C0F0AD01E
:1018D00030F0004C18BF31F0004CD8D180EA010044
:1018E00000F00040704790F0000F17BF90F0004FDD
:1018F000084691F0000F91F0004F14D092EA0C0FBF
:1019000001D142020FD193EA0C0F03D14B0218BF51
:10191000084608D180EA010000F0004040F0FE4097
:1019200040F40000704740F0FE4040F44000704733
:101930004FF0FF0C1CEAD0521EBF1CEAD15392EAB2
:101940000C0F93EA0C0F69D0A2EB030280EA010CA2
:1019500049024FEA402037D04FF0805343EA11113B
:1019600043EA10130CF000408B4238BF5B0042F199
:101970007D024FF4000C8B4224BF5B1A40EA0C003E
:10198000B3EB510F24BFA3EB510340EA5C00B3EB70
:10199000910F24BFA3EB910340EA9C00B3EBD10F5E
:1019A00024BFA3EBD10340EADC001B0118BF5FEAB0
:1019B0001C1CE0D1FD2A3FF650AF8B4240EBC250D9
:1019C00008BF20F0010070470CF0004C4CEA50209A
:1019D0007F32C2BFD2F1FF0340EAC250704740F4E9
:1019E00000004FF00003013A37E792F0000F00F0DB
:1019F000004C02BF400010F4000F013AF9D040EA59
:101A00000C0093F0000F01F0004C02BF490011F4EC
:101A1000000F013BF9D041EA0C0195E70CEAD153E4
:101A200092EA0C0F08D142027FF47DAF93EA0C0FCB
:101A30007FF470AF084676E793EA0C0F04D14B02AF
:101A40003FF44CAF08466EE730F0004C18BF31F061
:101A5000004CCAD130F000427FF45CAF31F000435B
:101A60007FF43CAF5FE700BF4FEA4002B2F1FE4FA8
:101A70000FD34FF09E03B3EB12620DD94FEA002350
:101A800043F0004310F0004F23FA02F018BF404229
:101A900070474FF00000704712F1610F01D1420210
:101AA00005D110F0004008BF6FF0004070474FF0C4
:101AB000000070477BB972B90029BEBF00204FF00B
:101AC000004106E008BF00281CBF6FF000414FF046
:101AD000FF3000F0ADB9ADF1080C6DE904CE00297E
:101AE00009DB002B1ADB00F035F8DDF804E0DDE956
:101AF000022304B07047404261EB4101002B1BDB25
:101B000000F028F8DDF804E0DDE9022304B04042EB
:101B100061EB4101524263EB43037047524263EB76
:101B2000430300F017F8DDF804E0DDE9022304B018
:101B3000404261EB41017047524263EB430300F0C6
:101B400009F8DDF804E0DDE9022304B0524263EB5A
:101B5000430370472DE9F0478C460E460446089D26
:101B6000002B50D18A4217466CD9B2FA82FEBEF1E0
:101B7000000F0BD0CEF1200C01FA0EF620FA0CFC6F
:101B800002FA0EF74CEA060C00FA0EF43A0CBCFB13
:101B9000F2F9BBB202FB19CC09FB03FA4FEA144875
:101BA00048EA0C46B2450AD9F61909F1FF3180F02E
:101BB0002581B24540F22281A9F102093E44A6EBFB
:101BC0000A06B6FBF2F002FB106600FB03F3A4B2B8
:101BD00044EA0644A34209D9E41900F1FF3280F037
:101BE0000B81A34240F2088102383C440021E41AF0
:101BF00040EA0940002D62D0002324FA0EF42C6044
:101C00006B60BDE8F0878B4207D9002D55D00021CD
:101C100085E841000846BDE8F087B3FA83F1002962
:101C200040F08F80B34202D3824200F2FC80841ADB
:101C300066EB03060120B446002D40D085E8101065
:101C4000BDE8F08712B90127B7FBF2F7B7FA87FEB4
:101C5000BEF1000F35D10121F61B4FEA174C1FFAD8
:101C600087F8B6FBFCF20CFB126608FB02F0230CB3
:101C700043EA0646B04207D9F61902F1FF3302D211
:101C8000B04200F2D2801A46361AB6FBFCF00CFBCA
:101C9000106608FB00F8A3B243EA0644A04507D942
:101CA000E41900F1FF3302D2A04500F2B9801846D2
:101CB000A4EB080440EA02409CE729462846BDE818
:101CC000F08707FA0EF7CEF1200326FA03F24FEA67
:101CD000174CB2FBFCF11FFA87F80CFB112206FA35
:101CE0000EF620FA03F301FB08F933431E0C46EA13
:101CF0000246B14500FA0EF409D9F61901F1FF3296
:101D000080F08C80B14540F2898002393E44A6EBD8
:101D10000906B6FBFCF00CFB106200FB08F99EB252
:101D200046EA0246B14507D9F61900F1FF3371D2F0
:101D3000B1456FD902383E44A6EB090640EA01419D
:101D40008FE7C1F1200722FA07F88B4048EA030326
:101D500026FA07F44FEA134EB4FBFEF91FFA83FC90
:101D60000EFB19448E4020FA07F809FB0CFA48EAEA
:101D700006084FEA184646EA0444A24502FA01F270
:101D800000FA01F608D9E41809F1FF3044D2A2455F
:101D900042D9A9F102091C44A4EB0A04B4FBFEF0E9
:101DA0000EFB104400FB0CFC1FFA88F848EA0444C0
:101DB000A44507D9E41800F1FF3E29D2A44527D94C
:101DC00002381C4440EA0940A0FB0289A4EB0C0C39
:101DD000CC45C246CE4615D312D055B1B6EB0A0358
:101DE0006CEB0E0606FA07F7CB401F43CE402F6080
:101DF0006E600021BDE8F0871046F7E68946DEE612
:101E00004645EAD2B8EB020A69EB030E0138E4E773
:101E10007046D7E718468FE78146BDE7114676E75B
:101E200002383C4444E7084606E7023A3E442BE7C2
:101E3000704700BF2A4C08B5F5F7A8FCF4F746FF39
:101E4000F4F760FFF4F7ECFFF5F7AAF9F5F724FDD6
:101E5000F8F76AF8F8F7DAF8F5F7E8FFF6F7CEF9E9
:101E6000F4F7DAFFF5F764FC2078F6F701FAE0788A
:101E7000F6F748FB2269A1686079F5F747FE00266E
:101E8000F9F72AF80125FCF747FA164CFDF794FEFE
:101E9000F5F78AF80BE0F5F735FB2571F5F714FD3A
:101EA0002060F5F711FDFEF7D7FBF5F73FFCFEF7D5
:101EB000F9FBFBF73FFEFDF759FAFDF717FEF5F7C3
:101EC00003FD2368C01A0028B8BF4042B0F57A7FEE
:101ED000E7DD2379002BDED0F5F70CFB2671DDE77B
:101EE0009C210020882000202DE9F0438BB004467F
:101EF0000D4600F079F8374B804693F9006089462B
:101F0000731C0DD022462B4620462946FFF7E8FADF
:101F100030B90022002320462946FFF7D7FA20B126
:101F2000404649460BB0BDE8F0832B4B0890CDE905
:101F30000245CDE904450193DEB94FF06046274FD5
:101F40002046294600220023CDE90667FFF796FACE
:101F5000002837D002230093684600F039FAC8B150
:101F6000089BE3B9DDE90689404649460BB0BDE868
:101F7000F0834FF00008DFF86C90204629460022DD
:101F80000023CDE90689FFF779FA68B102239E4262
:101F90000093E1D100F024FA22230360E0E700F08F
:101FA0001FFA089B0360DDE70123022E00930BD18B
:101FB00000F016FA21230360094800F00BFACDE97E
:101FC0000601CDE701230093684600F001FA0028DE
:101FD000F2D1EDE78000002014270108FFFFEFC7D2
:101FE000102701080000F0FF2DE9F04FB1F5801F28
:101FF00085B006460F460B465ADA024621F00044E9
:10200000224300F0F8800029C0F27A810022D64BEA
:10201000FEF7CCFF0B46D54A064693420F466FF0BB
:10202000350C4ADCC3F3130505F5152E0EF6647E58
:102030000EF4801E8EF07F5282F440121C1542EA8C
:102040000507A4F2FF3464440022C94B30463946E8
:1020500004EB1E54FEF7F6FDAB1CC3F31303022B77
:1020600082468B464FF0000230DC0023FFF706FA71
:10207000002800F0C980002C00F04B812046FEF7BC
:102080002FFFA5A3D3E9002306460F46FEF78EFFD8
:10209000A3A3D3E9002304460D4630463946FEF794
:1020A00085FF02460B4620462946FEF7CDFD0AE095
:1020B000AE4A4FF0000C9342B4DD32463B46304608
:1020C0003946FEF7C1FD05B0BDE8F08F4FF0804303
:1020D000FEF7BAFD02460B4650465946FFF790F808
:1020E000064620460F46FEF7FBFE3246CDE90001CC
:1020F0003B4630463946CDE90267FEF757FF0246B8
:102100000B4680468946FEF751FF87A3D3E900239B
:1021100006460F46FEF74AFF85A3D3E90023FEF7E4
:1021200093FD32463B46FEF741FF83A3D3E90023EC
:10213000FEF78AFD32463B46FEF738FF80A3D3E91F
:102140000023FEF781FD42464B46FEF72FFF7EA39C
:10215000D3E900238046894630463946FEF726FFFC
:102160007BA3D3E90023FEF76FFD32463B46FEF723
:102170001DFF79A3D3E90023FEF766FD32463B46F7
:10218000FEF714FF0B46024649464046FEF75CFD4B
:10219000A5F5C223C5F5D725A3F27A4351351D43D2
:1021A000002D8046894656DD0022724B5046594626
:1021B000FEF7FCFE52465B46FEF7F8FE06460F466B
:1021C000002C68D132463B4640464946FEF73CFD6E
:1021D000DDE90223FEF7EAFE02460B4630463946A9
:1021E000FEF730FD02460B4650465946FEF72AFDE3
:1021F00005B0BDE8F08F0022002300205E49FEF705
:10220000FFFF05B0BDE8F08F55A3D3E9002350468A
:102210005946FEF7CBFE02460B4600205549FEF715
:1022200011FD524606460F465B4650465946FEF79C
:10223000BDFE02460B4630463946FEF7B7FE06465F
:102240000F46002C40F09A8002460B4650465946F5
:10225000FEF7F8FC37E7002C00F0A4802EA3D3E9AA
:102260000023DDE90001FEF7A1FE42464B4604468D
:102270000D4650465946FEF7E5FCDDE90223FEF720
:1022800095FE27A3D3E9002306460F46DDE90001AA
:10229000FEF78CFE21E020A3D3E90023DDE9000155
:1022A000FEF784FE32463B4604460D46404649460C
:1022B000FEF7CAFCDDE90223FEF778FE18A3D3E996
:1022C000002380468946DDE90001FEF76FFE0246E5
:1022D0000B4640464946FEF7B7FC02460B463046E1
:1022E0003946FEF7AFFC52465B46FEF7ABFC0246B2
:1022F0000B4620462946FEF7A5FC05B0BDE8F08F49
:1023000002460B46FEF79EFC00220023FEF778FFF4
:10231000D9E600200021D6E60000E0FE422EE63F8E
:10232000763C7935EF39EA3D44523EDF12F1C23F47
:10233000DE03CB966446C73F599322942449D23F8B
:10234000935555555555E53F9FC678D0099AC33FDB
:10235000AF788E1DC571CC3F04FA97999999D93FF2
:10236000555555555555D53F00005043FFFFEF7F5C
:102370000000F03F0000E03F000050C32046FEF7A1
:10238000AFFD0FA3D3E9002380468946FEF70EFE7A
:102390000DA3D3E9002304460D4640464946FEF707
:1023A00005FE9AE702460B4650465946FEF74AFCA0
:1023B000DDE90223FEF7FAFD14E700BFAFF300806A
:1023C0000000E0FE422EE63F763C7935EF39EA3DEB
:1023D0000020704700200149704700BF0000F87FCF
:1023E000014B1868704700BF1C000020020000006D
:1023F00000000001000000000102030401020304C8
:1024000006070809020406080010161B2023272AC5
:102410002D30323537393B3D4041434547494B4CE0
:102420004E505153545657595A5B5D5E606162631A
:10243000656667686A6B6C6D6E70717273747576C1
:102440007778797A7B7C7D7E8080818283848586A3
:102450008788898A8B8C8D8E8F909091929394959A
:1024600096969798999A9B9B9C9D9E9FA0A0A1A2AF
:10247000A3A3A4A5A6A7A7A8A9AAAAABACADADAED5
:10248000AFB0B0B1B2B2B3B4B5B5B6B7B7B8B9B909
:10249000BABBBBBCBDBDBEBFC0C0C1C1C2C3C3C44B
:1024A000C5C5C6C7C7C8C9C9CACBCBCCCCCDCECE93
:1024B000CFD0D0D1D1D2D3D3D4D4D5D6D6D7D7D8E4
:1024C000D9D9DADADBDBDCDDDDDEDEDFE0E0E1E13D
:1024D000E2E2E3E3E4E5E5E6E6E7E7E8E8E9EAEA9D
:1024E000EBEBECECEDEDEEEEEFF0F0F1F1F2F2F300
:1024F000F3F4F4F5F5F6F6F7F7F8F8F9F9FAFAFB6C
:10250000FBFCFCFDFDFEFEFF0010161B2023272A0E
:102510002D30323537393B3D4041434547494B4CDF
:102520004E505153545657595A5B5D5E6061626319
:10253000656667686A6B6C6D6E70717273747576C0
:102540007778797A7B7C7D7E8080818283848586A2
:102550008788898A8B8C8D8E8F9090919293949599
:1025600096969798999A9B9B9C9D9E9FA0A0A1A2AE
:10257000A3A3A4A5A6A7A7A8A9AAAAABACADADAED4
:10258000AFB0B0B1B2B2B3B4B5B5B6B7B7B8B9B908
:10259000BABBBBBCBDBDBEBFC0C0C1C1C2C3C3C44A
:1025A000C5C5C6C7C7C8C9C9CACBCBCCCCCDCECE92
:1025B000CFD0D0D1D1D2D3D3D4D4D5D6D6D7D7D8E3
:1025C000D9D9DADADBDBDCDDDDDEDEDFE0E0E1E13C
:1025D000E2E2E3E3E4E5E5E6E6E7E7E8E8E9EAEA9C
:1025E000EBEBECECEDEDEEEEEFF0F0F1F1F2F2F3FF
:1025F000F3F4F4F5F5F6F6F7F7F8F8F9F9FAFAFB6B
:10260000FBFCFCFDFDFEFEFF000203050608090BB6
:102610000D0E101113141617191B1C1E1F21222436
:102620002527292A2C2D2F303233353638393B3C9B
:102630003E3F4143444647494A4C4D4F5051535405
:102640005657595A5C5D5F606263646667696A6C7D
:102650006D6E707173747577787A7B7C7E7F808203
:1026600083848687888A8B8C8E8F9092939495979B
:1026700098999A9C9D9E9FA1A2A3A4A5A7A8A9AA48
:10268000ABACAEAFB0B1B2B3B4B5B7B8B9BABBBC0E
:10269000BDBEBFC0C1C2C3C4C5C6C7C8C9CACBCCF2
:1026A000CDCECFD0D0D1D2D3D4D5D6D7D7D8D9DAF2
:1026B000DBDCDCDDDEDFDFE0E1E2E2E3E4E4E5E613
:1026C000E7E7E8E8E9EAEAEBECECEDEDEEEEEFF057
:1026D000F0F1F1F2F2F3F3F4F4F4F5F5F6F6F7F7BE
:1026E000F7F8F8F8F9F9F9FAFAFAFBFBFBFCFCFC4D
:1026F000FCFCFDFDFDFDFDFEFEFEFEFEFEFEFFFF01
:10270000FFFFFFFFFFFFFFFF313633365631313217
:08271000000000006C6F67007F
:04271800F8B500BF51
:04271C00F8B500BF4D
:0827200034F4FF7F010000000A
:1027280003020000082701080100000000480040DB
:1027380001000000D0070000010000002000002078
:102748000000000000000000000000000000000081
:102758000000000000000000000000000000000071
:102768000000000000000000000000000000000061
:102778000000000000000000000000000000000051
:102788000000000000000000000000000000000041
:102798000000000000000000000000000000000031
:0427A800010000002C
:04000005080041109E
:00000001FF
